:020000040800F2
:100000000050002005730108A1730108D5EE000817
:10001000A1730108A1730108A17301080000000089
:10002000000000000000000000000000A1730108B3
:10003000A173010800000000A1730108DB1701088B
:10004000A1730108A1730108A1730108A17301083C
:10005000A1730108A1730108611B0108751B010848
:10006000711B01086D1B0108691B01081194000830
:1000700001940008F1930008E1930008D19300086F
:10008000BD930008AB930008A1730108A173010898
:10009000A1730108A1730108A1730108651B010880
:1000A000A173010821F80008A173010811F80008E4
:1000B00001F80008F1F70008E1F7000885390108A8
:1000C000893901087D39010881390108A1730108C6
:1000D000A1730108191801080D180108A17301087E
:1000E0005D1B0108A1730108A17301080000000055
:1000F0000000000000000000000000000000000000
:0C01000000000000000000005FF808F1A3
:100110002DE9F04F0B4B0C4D0C4AC5F8B8340023B9
:1001200010680B499FB08842C5F8BC3416D11360E3
:1001300062B6084B18680BF05DF9074B1B689847CF
:10014000FEE700BFDFCD000820060020F04F0020B2
:10015000EFBEADDE00F0FF1F04F0FF1F0893099310
:100160000A934FF4E013BD4C0B93236843F48033A0
:100170002360A36943F01003A361236803F40033F1
:100180000993089B01330893099B1BB9089BB3F59E
:10019000A06FF2D1236813F4003300F0A58202238C
:1001A0000A93AF4BAF4F1A6842F010021A601A68F8
:1001B00022F003021A601A6842F002021A606368B1
:1001C000636063686360636843F480636360A64B45
:1001D0001A68043B22F070425A60A44A3A6062688E
:1001E00022F47C1262605A6842F000425A60DA6877
:1001F00022F40042DA609B681E0449BF9C4B4FF416
:10020000E0133B604FF480130B930A9B012B00F02B
:100210008382022B05D10B9B6268134343F4803326
:100220006360236843F08073236023689801FCD5E2
:10023000636823F003036360636843F00203636051
:10024000636803F00C03082BFAD16368DFF8688257
:1002500003F00C03042B00F06382082B00F0628291
:10026000824BC8F800306368DFF85092C3F3031381
:1002700019F80320D8F80030DFF844B2D340C8F8AA
:1002800000307C4B4FF6FF72CBF80C30A3690DF1B8
:10029000780A43F00103A361636A636A764E43F010
:1002A00080736362A369304643F01C03A3614FF07F
:1002B00000032AF82C2D51468DF84E3009F03AF8FB
:1002C00051466E4809F036F851466D4809F032F84B
:1002D00010228DF83E2002228DF83F204FF400724C
:1002E0001EA921F83C2D3046326109F023F86549FA
:1002F00050464A6842F000724A600AF0DFFE139BE3
:10030000614A3046B3FBF2F34FF47A72C5F8C03459
:10031000D8F800304FF0010CB3FBF2F35B4A013B1D
:100320005360F0238BF82330002393600723DFF81A
:1003300094E11360564A09F10E01002331F8026F6F
:1003400046FA03F818F0010F18BF0CFA03F803F18E
:1003500001031EBF1060A2F804800832102BEFD1F9
:1003600000F580607045E8D13B68404A934240F018
:10037000EB81012385F8C4340DF08EF918B90FF024
:10038000F5F80EF0F5FD0EF01FFF95F8C534414F5E
:1003900043F0010385F8C5343F4BDFF82C819A7890
:1003A0003E4B08F1050A1A703D4B1B683B6095F8FF
:1003B000CA3485F8C634002313F808004FEA830BCB
:1003C0005E1C002800F0C681029311F099FA029B8E
:1003D0004AF8230010B10523C671837112215AF81F
:1003E0000B0011F0B3FA032E3346E5D10021084685
:1003F00011F050FB0021012011F04CFB00210220E4
:1004000011F048FB0121022011F044FBA3690021F7
:1004100043F00103A3614022224819F038FE4FF057
:10042000FF33214AC5F818356420C2F8033011F0B3
:10043000CAF9A02200211D4819F029FE00241C4DF4
:100440001C4E0023605956F83310DA00884240F001
:10045000848109EB0203187F38E000BF00100240DE
:1004600000200240D80000200410014000127A0051
:10047000001BB7000005FA0500080140000C014010
:10048000001001400000014040420F0010E000E079
:10049000341600200C3600200816002024250020E9
:1004A00068180020F80A0020380B0020081C0020E3
:1004B00090BE010800A2010810000020E8A1010878
:1004C00000ED00E000140140E70A0020103414F0B1
:1004D0007BFEE02CB5D1B44AB44C0021A046914635
:1004E000B34E00250B5D01F10F00204406EB030A1B
:1004F00010F801CFBCF1000F05D09AF80CE0E645EA
:1005000008BF82F858E090F803C0BCF1000F05D096
:1005100016F803E0E64508BF82F859E00135032DDF
:10052000E6D1B2F8580040B108EB010009EB8303B3
:100530005065C3F8202502F517721C313829D0D137
:100540000424994E302200219A483D6886F82C45B3
:1005500019F09DFD964B224693F80BC093F80A9034
:100560000023944C1846A2464FF0FF0BDFF89CE2A4
:1005700005F040081EF9011F1E29195540F0F380AF
:10058000B8F1000F00F0F980B9F1000F00F0F5802C
:100590000C33302BEED108B186F82C25864B874CD6
:1005A00093F800B0864E874B15F4805214BFA08894
:1005B000B08A83F800B00292994616F059FADFF833
:1005C0005082DFF850A2C8F80000308A16F04CFACA
:1005D0007D4B1860708A16F047FA7C4B1860608873
:1005E00016F042FA7A4B1860208816F03DFA794BE3
:1005F000BAF81A101860C1F5FA60039116F038FACB
:10060000754A03991060BAF81820B4F806A0501A79
:10061000A0EB0A00039216F02BFA039A6F490860C8
:10062000C2F5FA60A0EB0A0016F022FA6C4B6D4A94
:1006300018606D4B2B40002B40F0A5806B4B03EBFB
:10064000CB0B9BF80130136040F2DC510023684A69
:1006500022F813100133082BFAD1029BB6F814B01C
:100660000BB1B4F804B0B378042B05D14FF480502B
:100670000CF08EFD4FF0000B002599F800205D4C2A
:10068000A2F11703022B257000F2C880DFF88891D1
:10069000002155F8090005EB090A16F0D1FB0028E6
:1006A00073D03B68DA0400F1DA800023D8F8001038
:1006B000514A42F823100133082BFAD12378C02283
:1006C00000214E48049319F0E2FC3779B3780037E3
:1006D00018BF0127042B00F2E780DFE813F0900138
:1006E000E5009201E8008A01226842F001022260DE
:1006F0000893236803F002030993089B01330893CE
:10070000099B1BB9089BB3F5A06FF2D123689F0723
:1007100001D5012344E5FEE7636843F460137FE5F8
:100720003B689EE563686268C3F38343D10303F1CA
:10073000020302D4324A534393E5626812F4003F45
:100740003A6818BF5208F6E72E4A93427FF414AE77
:1007500002230FE64AF8230045E60133042B7FF419
:1007600072AE0020B2E61F297FF412AFB8F1000F7D
:1007700003D0BCF1000F7FF40BAF013A0AF803B0CD
:10078000D2B2012004E701235DE71F4B05EB030E06
:100790009AE80F008EE80F00237810350133802D82
:1007A00023707FF475AF7CE72006002020A20108AB
:1007B0007C210020584100202C250020A42D002061
:1007C0007823002094110020902300203411002071
:1007D000BC110020B0110020C8110020B811002069
:1007E000C4110020541200202000100010AC010899
:1007F00054230020042300205825002080250020B9
:1008000000093D00001BB700D011002057A20108CD
:10081000C82600203836002064170020B44B13F897
:10082000321003EBC2030829217088BF0821D3F8D6
:1008300004C088BF2170BCF1000F3FF432AF002527
:10084000DFF8109323789D42BFF62BAF2B0103EB0B
:10085000090E63440FCB01358EE80F00F2E72378D1
:10086000012B7FF622AF4FF07C59A24D05EB03130D
:1008700003F110071035BD423FF417AF494655F854
:100880000C0C16F049F9494645F80C0C55F8100CBB
:1008900016F042F9494645F8100C55F8080C16F0C8
:1008A0003BF945F8080CE5E7934CA04602E0934C71
:1008B000DFF8A482924A934B21461A60924A934BE6
:1008C0004046002F18BF1346914A0025136016F0CA
:1008D0001BF801464FF07A5016F0D2F98D4903907B
:1008E000204616F019F98C4CDFF870A20590049B95
:1008F000AB4240F3E58005EB0A035E790021304608
:100900000EF054FF029000287DD1844A7D4B1A607E
:100910007D4A7F4B1A60824C82482368002B40F04E
:100920001F81037803F0EF02082A7F4A40F03A81E2
:100930001178182B41F01001117001D10FF08AFECF
:100940002368002B40F03781784A794C136806926F
:1009500013F0010640F078819B0440F1C28194F8C5
:100960001826744B04F5A8651A7004F5C26816F8C9
:100970000890002148460EF019FF074698B3002260
:100980004FF0010A5FFA86FB05F80FBC45F8040C2E
:1009900005F80E2C05F8062C05F810AC484610F0AA
:1009A000AFFFD3445FFA8BFB18B180F806A080F844
:1009B00007B04FF0000B2A2110F0C8FF5E4A00215B
:1009C000384610F005FE5D4B2A1D2B605C4B294616
:1009D00038466B60C5F808B010F04EFE5A4679797B
:1009E00038680BF02DFC0136082E05F11C05BED130
:1009F00077E10024A04601274FF0000B5AE7454C51
:100A0000F8E7504C51E7304610F07AFF6B1C6061FC
:100A1000DBB210B10322C37182711A2110F096FF6C
:100A2000002F51D0BAF8000016F022F816F076FA2E
:100A3000454B4FF6FF791E68B6FBF0F34B441B0C99
:100A4000B6FBF3F60FB1B6FBF0F99AF80230042BBF
:100A50003ED1484616F008F82E4916F05DF8A06021
:100A60000790304616F000F8414616F055F8079BFF
:100A700006903649184616F04FF8069A0146104679
:100A800015F040FF9AF80330E06032460193029976
:100A90001FFA89F3CDF800B0204615F085F9002340
:100AA00018221D49AB4218D1002383F0010323749F
:100AB00001231D44082D637404F118047FF417AF5B
:100AC0000122234B1A7026E7039816F08BFFADE73F
:100AD000304615F0C9FF0599BFE702FB03104668D1
:100AE0006068864201D00133DCE70123DDE700BF07
:100AF00010AC0108D41100206F120339ACC5A73720
:100B00006DBD000838310020EDBA000899BD00081D
:100B10003C3100206F12833A80250020EFBA000894
:100B20005412002094110020ED2600200C360020E5
:100B300020060020A021002040420F007DC20008B6
:100B400063B90008282930381000002000007A44DA
:100B500058120020D0110020ACC5A7367823002001
:100B60000278334B334913F8325003EBC2035E680B
:100B70000D70002E3FF4D5AE00232F4FAB42BFF6D1
:100B8000D0AEC3EBC3017218D2F800C001EB070E60
:100B900041F807C091880133AEF8041092798EF8BD
:100BA0000620EBE70E2B3FF4C3AE1178192B21F092
:100BB00010011170C1E600254FF0040B1F4F204EAD
:100BC000DFF880A0A7F1030917F8018FB8F1000F33
:100BD0003FF4BAAE404610F093FE01350446706112
:100BE000EDB210B180F806B0C571002140460EF09C
:100BF000DDFD80461A21204610F0A8FEB8F1000F56
:100C00003FF4A2AE0022B9F8023001929AFBF3F34E
:100C1000B9F800209BB2009230460A4A414615F0CE
:100C2000C3F80123082D737406F11806CCD18BE6A6
:100C30005CAA0108152B0020162B00207D2C00201B
:100C4000A421002040420F000025FF2294F82D75BA
:100C5000CF4B294638461D705D609D60DD601D6488
:100C600083F8442083F8452083F8465083F84750A2
:100C700083F848500EF09AFD064690B30368C549C4
:100C80006A18507C18B15268934200F03F841835BE
:100C9000C02DF5D10025C4F83C6584F830553846A0
:100CA00010F02EFE10B10223C571837100252A2198
:100CB00010F04CFEB84A0021304610F089FCB74BCA
:100CC000B74AC4F84035B74B111F3046C4F8443515
:100CD000C4F8485510F0D0FC2A46717930680BF002
:100CE000AFFA94F8C534B4F81E6643F0040384F8F0
:100CF000C534A4F8206694F81A06002E40F011843A
:100D000010F0FEFD94F81B26C4F82406003218BF2C
:100D1000012284F8282650B1242294F81C368271CE
:100D2000002BC6710CBF1221162110F00FFE0020FF
:100D300010F084FE4FF000089B4B0020C4F84836AA
:100D400008F0DAFA012008F0D7FA984A02F1200CEC
:100D500052F8055CA5B312F9093CE11891F84C660C
:100D600091F84E7691F850E604EB0310911E11F8BD
:100D7000019FB14591F8029008BF80F85866B945C7
:100D800091F8049008BF80F85976F14508BF80F8C3
:100D90005AE68A42EBD104EB031393F8581679B163
:100DA00093F8591661B193F85A1649B15179C3F8BD
:100DB000545683F85B16917983F8608683F85C1645
:100DC00010326245C4D114F04BFB14F049FB94F887
:100DD0006C0614F0F9F9012394F86C2602F01F0157
:100DE0005209022A03FA01F300F0CA83032A00F031
:100DF000CC8394F8680610F083FD054618B11223E1
:100E000083710223C37194F8690610F079FD18B15B
:100E1000132383710223C37194F86A0610F070FDE6
:100E200018B1142383710223C3711B21284610F0CB
:100E30008DFD94F8690610F063FD072110F086FD22
:100E400094F86A0610F05CFD1B2110F07FFDD4F8C9
:100E50006426574B9A4240F09D8303F56043D9685E
:100E600041F48051D960D96821F48051D96094F857
:100E70007036002B00F0AA8300231846118801F475
:100E8000415141F445710B4303431380938B23F489
:100E900000631B041B0C93830723138213889BB2EC
:100EA00043F04003138094F8C434032B11D11F2066
:100EB00007F037FC00233F4A02EBC30191F902100F
:100EC000022901F016820133042BF5D1022007F02C
:100ED00028FC0CF03EF8012012F0E6FB2C2010F06C
:100EE0000FFD9F238DF83C300023C4F87406322098
:100EF0008DF83D308DF83E308DF83F3010F063FCBA
:100F0000D4F8740610F086FD04230FAA13A92A480A
:100F10000BF0A9FFD4F8740610F081FD9DF84E3057
:100F20009DF84D201B0243EA02439DF84F201343D6
:100F3000224A93421FD0322010F045FCD4F87406A8
:100F400010F068FDF5211C480BF0BBFFFF211A488B
:100F50000BF0B7FF8DF84C00D4F8740610F05FFD6D
:100F60009DF84C30702B06D194F8C434022B02D17A
:100F7000032384F8C434124B00211E791148751ED6
:100F80006A426A415D7984F878266F1E1CE000BFD2
:100F9000BC1B00208025002040420F0089B90008BA
:100FA000640B0020BDBA00087C21002065A2010866
:100FB0000030014032410020003800401520200060
:100FC000FE350020A00C00207B427B4184F87C365B
:100FD000069B14221B6803F40047C3F3C03384F854
:100FE0007A3619F054F8012E04BF94F8793684F853
:100FF00080361FB194F87B3684F88F3694F87E36AD
:101000001BB194F87F3684F88A36012D08BF94F816
:101010007D36C14D08BF84F8853600232E464FF03B
:10102000070B1F469946DFF83C8308F1940A307895
:10103000E8B110F065FC18B180F806B080F80790B0
:10104000002110F083FC002331781AF813005A00B5
:10105000884240F0BE8208EB020393F8953073702B
:101060000723337101237A1CB770F370D7B20BF1E9
:10107000010B5FFA8BFBBBF10B0F06F10506D6D116
:10108000002B00F0BB80A54E4920736843F4404319
:10109000736014F099F8A24AA24900234FF01C0E85
:1010A000104688460EFB032CDCF804C08C4540F04B
:1010B0009682DBB21C2101FB0303726919694FF0B0
:1010C00000090A437261062283F819901A7695483E
:1010D00009F07BFF13A809F04DFF934B022F1393E8
:1010E00034BF4B46802318934FF4807319934FF409
:1010F00080631A9320231B934FF400538B4E13A944
:10110000884816971C931496CDF85490CDF85C90AF
:10111000CDF8749009F03BFF012F94BF002201220B
:10112000D8F80030824943F00103C8F800304B681A
:101130004FF0070E23F4702323F4807343EA022355
:101140004B608A687B4B134043F4602343F00203F7
:101150008B60CA6A7B1E22F47002DBB242EA035340
:10116000CB621F270123EA784AB395F80180581C07
:10117000B8F1090FC0B295F804C040F23682A8F168
:101180000A02D1F80C9002EB42020EFA02FA29EAA6
:101190000A090CFA02F242EA0902CA60062B00F2BE
:1011A000318203F1FF3C4A6B0CEB8C0C07FA0CF319
:1011B00022EA030308FA0CF21A434A630346053590
:1011C000AE42D0D15A4B9A6842F480729A609A68C3
:1011D00042F001029A609A6842F008029A609A68A6
:1011E0001007FCD49A6842F004029A60504B9A6847
:1011F0005107FCD49A6842F4A0029A60D4F89C0685
:10120000002841F0BD80D4F8A036002B41F0B88012
:10121000D4F8A436002B41F0B3800DF0A1F930B919
:101220000120022110F074FC012014F0A9FE01211C
:1012300094F8C534084643F0020384F8C53410F02E
:1012400029FC0021084610F025FC0021022010F0A6
:1012500021FC0A25384E012010F043FB002010F03D
:1012600040FB192010F0AFFA3368DA0302D40120F2
:1012700010F0E4FB192010F0A6FA002010F0DEFBBD
:10128000013DE8D12946284610F004FC29460120FA
:1012900010F000FC294B2A4F18680FF01FFABA898A
:1012A000002A40F0F981274B0DF14C08587A15F0CF
:1012B000DFFB254915F030FC244915F025FB0CF027
:1012C00038FA234B1860234B188A15F0D1FB0146DE
:1012D000214815F0D5FCC4F8A80611F087FB0123BE
:1012E0001393069B1A68530201D41C4B1393D70027
:1012F0005EBF139B43F010031393194B19680293BD
:1013000011F0020F1EBF139B43F0C60313934E0749
:1013100048BF139B28E000BFA00C00200010024033
:1013200014000020080002404C240140B40C0020AE
:1013300000240140FDF7F1FF741800202025002053
:101340007A2C00207431002035FA8E3CDB0FC93F27
:1013500094310020B8220020A889803A01000010B2
:1013600028250020E8A1010844BF43F00803139397
:10137000D40542BF139B43F000631393B04B19781D
:10138000039301F0EF00082801D00E2903D1139B2D
:1013900043F480531393139BD00354BF43F400537F
:1013A00043F420431393139BD7044CBF43F064438F
:1013B00043F044431393960642BF139B43F4807358
:1013C0001393540742BF139B43F400331393139BAF
:1013D00043F400201390500505D59A4A127912B1B2
:1013E00043F4C0131393182908BF139B4FF0010651
:1013F00004BF43F0607313930723149329464046B8
:10140000ECB209F0AEFA70B120460DF02BFD50B9E8
:101410006A0958F8223004F01F0406FA04F423EA9B
:10142000040448F822400135242DE7D1864D98E880
:10143000030005F2AC6383E803004FF41972002146
:1014400005F2B46018F023FE07F08AFB00227F4FFC
:101450007F4C049767607F4F7F4BBE461A809A701F
:101460007E497F4B7F4E80481960338BDFF824A282
:10147000A06085F8182919B2059005F61C1CDAF849
:10148000000027F8121000F596704CF82200013287
:10149000122AF4D1754FDFF8BCC13868C20458BFB6
:1014A000B6F92610AEF80610714901F1500E0A780F
:1014B000AAB98A7891F803A0524510D2002A00F008
:1014C000FF80013A02EB820202EB820202F56172B6
:1014D00091F801A092B20AF1040A2CF81A20043102
:1014E0008E45E4D1020740F16D81307A0A2800F27E
:1014F0006281DFE810F0F300F300D50351047504B6
:1015000095049504D90460011605F3001B8D594A12
:101510009BB212680133B2FBF3F3574A1370FFF723
:10152000B9BB10F0EDF94021C4F82406C4F8400618
:1015300005461C200EF03AF90746CDB1C0B1242370
:10154000AB7101231A21EB71284610F0FFF900213D
:10155000A4F8446601914949494A91FBF6F192FB8E
:10156000F6F389B200919BB23946464814F01CFC50
:101570000023D4F82C26138084F83D36FFF7DABB1D
:10158000414AD1680B43D36033E43F4A11690B43AE
:1015900013612EE43D4B9A420AD103F5EC331969ED
:1015A00041F480411961196921F4804119615EE4B7
:1015B000374B9A427FF45BAC03F5EA33196941F487
:1015C00000411961196921F40041EFE7012302206C
:1015D00054E401330A2B7FF438AD00233FE5013397
:1015E000072B7FF45FAD002364E50A6908EB480A26
:1015F0000EFA0AF922EA09090CFA0AF242EA090289
:101600000A61CBE50C2B0DD8DA1FD1F830C002EB04
:10161000820207FA02F32CEA030308FA02F21A43E1
:101620000A63CBE50D3BCA6A03EB830307FA03FCAD
:1016300022EA0C0208FA03F31343CB62BEE500BFB3
:101640002C250020361A00202006002079FE0008F4
:10165000D8290020CC35002010360020A0860100BB
:10166000B82900203836002075FE00080C3600200E
:101670007C180020100000201C04002020A107007E
:1016800040420F004C0C0020001002400038004087
:10169000003C0040901B00202E46DFF83890DFF819
:1016A0003880B88915F0E0F9D9F80020014608EB38
:1016B00006002C3609F010F9B6F5B07FF1D1F2E54D
:1016C0000AF1010A0AEB8A0A0AEB8A0A0AF5617230
:1016D000FEE600BF082500207C120020B64B40200B
:1016E0001C6007F01BFA8346002864D04FF0000905
:1016F000B24A82F80090069213F09EF9317A82463F
:101700000129069A0CD0C0F0B9820A2916D1AC4B37
:101710001B6813F480631CBF80F00103DBB21370FD
:101720000322A84B1A700722A74B1A700122A74B5D
:101730001A700C23237042F6F8236380A44B9F4A4F
:101740006360A44BA3609BF90200BAF1000F40F064
:10175000A3821378002B0CBF012303231278002AE5
:1017600040F09C82B27A002A0CBF0022082201922B
:101770000093994A4FF4E133402107F019F8974B51
:101780001860BAF1000F01D0954B1860737D217875
:10179000013BDBB2934A994213709CBF0023137044
:1017A00028B1864B1B7813B1012385F864390030CA
:1017B00018BF012030B908200BF0EAFC049B6360DD
:1017C000059BA3607E4B1B6858040BD51222227028
:1017D00044F620626280844A84496260844AA2603E
:1017E000844A116042F20102134209D044F6206299
:1017F0009904628040F1C083082222707E4A6260B0
:101800004FF0000A7D4CDB0384F800A040F18D818D
:1018100013F0C0F901232370794B40F22A3293F878
:10182000F1B05146774818F032FCBBF1000F00F0E0
:101830006F81514658460DF0B9FF734B026804465C
:101840001A6082689946002A00F06281584610F0BA
:1018500057F8C5F8680918B1282380F807A08371E4
:101860001B2110F073F80023684AD9F8001002F128
:10187000180E5EF833004FEAC30C814240F08383B8
:101880006244107F13F0A0FCD9F80000604A03887E
:101890004FF0000A23F001031B041B0C03805D4B77
:1018A000DFF880E11B68ADF836A0934281BF03F1F9
:1018B000B772594902F55852B2FBF1F292BF0022B9
:1018C00002F1FF3292B2511CB3FBF1F35349ADF870
:1018D00032A0B3FBF1F303219BB2B3FBF1F14FEA6A
:1018E000410CAEF800C0DFF840E18DF838A0AEF84A
:1018F00000101EA921F8482DADF8343013F069FD11
:101900006023ADF83EA0ADF840A0ADF842A0ADF820
:1019100044A0ADF848A0ADF846A0ADF84AA0ADF897
:101920003C30E3794FF0000B580757BF01220422E7
:10193000ADF83E204FF4807203F002034CBFADF8C7
:101940004020ADF84820ADF84430ADF842B00FAAC1
:101950006179D9F800000DF035FE6179D9F8000001
:1019600013F00AFDD9F800200121B2F84430DFF865
:10197000BCA06FEA43436FEA53439BB2A2F84430E2
:1019800013889BB243F0800313806379108C01FAB3
:1019900003F39BB280B220EA03001084108C80B263
:1019A00003431C20138413889BB20B431380237BB7
:1019B0001B4A00FB03233BE0802A0020852A0020ED
:1019C0000C3600207F2A0020842A0020B328002023
:1019D000F1F900083D0101085D020108E42A002038
:1019E0007C1B00207E2A0020F1FE0008400D030031
:1019F000D9FE0008B8290020C9FE0008AB35002038
:101A0000243400209C370020CC3A0020E8A10108B3
:101A1000FF6BDC0210000020006CDC0200350C00C3
:101A2000140000209A37002098370020C83A002080
:101A3000BB4A1869D2F814E040EA0E0EC2F814E06E
:101A40004FF0280E83F819B083F818E0D2F814E0AC
:101A500040EA0E005061B34AC3F814B09A605B7B51
:101A600013A88DF84D108DF84F108DF84C308DF86F
:101A70004EB013F0C7FBA068CAF8000009F0A5FA41
:101A8000DAF80000036823F001031B041B0C036059
:101A900009F09BFA13A809F06DFAD9F800306279C1
:101AA00034331344139340F22A331693802318934C
:101AB0009D4B13A91493102315934FF4007319939E
:101AC0004FF40053DAF800001C93CDF85CB0CDF869
:101AD00068B0CDF874B0CDF86CB009F058FA6279FE
:101AE000D9F800100C2A8EBF5B46904B03EB4203E3
:101AF0008A8998BFB3F8A83092B21343DAF800206D
:101B00008B81136843F0020313600122884B1A7023
:101B10000023FF211C4687481A181C520433802BCF
:101B20009170D170F8D113F0A5F8834B1B6859055B
:101B30003FD5042006F0F2FF804B0421186006F028
:101B4000E3FF7F4B1870082006F0E8FF7D4B08216B
:101B5000186006F0D9FF7C4B2C22187000217B48BE
:101B600018F095FA7C2385F86C398E2385F86D3949
:101B7000E02385F86F397D23202085F8973906F01A
:101B8000CDFF734B2021186006F0BEFF714B18701B
:101B90004FF4805006F0C2FF6F4B4FF48051186035
:101BA00006F0B2FF00226D4B18706D4B1A7009F0F1
:101BB00083FD6C4CB4F80090B9F1000F40F0448202
:101BC00095F89809002800F03F820FF099FEC5F8BB
:101BD0009C0918B11A2380F80790837113210FF024
:101BE000B5FED5F89C090FF01AFF00BF02215E4830
:101BF0000BF01AF94FF000099F2332208DF83C308A
:101C00008DF83D908DF83E908DF83F900FF0DBFD04
:101C10008DF84D9000BFD5F89C090FF0FBFE042312
:101C20000FAA414650480BF01EF9D5F89C090FF059
:101C3000F6FE00BF9DF84E309DF84D201B0243EA92
:101C400002439DF84F201343484A934200F04283D9
:101C500000F39F81464A934200F0A48101329342EF
:101C600000F0E581A2F51A42033A934200F02D8379
:101C7000002323806380A360E360E5E102213D4A05
:101C80000723117003213C4A237011703B4A45F22F
:101C9000F05382F8009050E503235FE5082266E5E3
:101CA0000A221B0193FBF2F300223549A3F5B0632E
:101CB00041F822300132122AFAD142F6F823638029
:101CC000304B40206360304B2270A36006F026FF4B
:101CD000824600283FF46FAD12F0AEFE737AB17AFF
:101CE00000280CBF01220322002B0CBF0623072370
:101CF00000290CBF002108219AF902E082460B431B
:101D00008DE80C00214B224A4021704606F050FD20
:101D1000BAF1000F3FF44BAD1E4B186047E500BF12
:101D200000100240DF8C00089C370020E8A1010869
:101D3000C63A0020183500200C360020741B002005
:101D4000801B0020701B0020811B00208C0F0020B6
:101D5000881B0020831B0020981B0020941B002060
:101D6000951B002038040020003800401620C200D7
:101D700017BA20007F2A0020842A0020B3280020E0
:101D8000E428002019FA000835FA0008A0860100AE
:101D9000A90201087C1B00201023237042F6F823BF
:101DA0006380814B40206360804BA36006F0B6FEE9
:101DB000824600283FF4FFAC12F03EFEB27A0028C3
:101DC0000CBF01230323002A0CBF002208229AF92A
:101DD00002E00192009382464FF4E133744A93E7A4
:101DE0000823237042F6F8236380724B402063601F
:101DF000714BA36006F092FE824600283FF4DBACF4
:101E000012F01AFE002200280CBF012303239AF9C6
:101E100002E00192009382464FF4E133674A73E790
:101E200000234FF00C0E664A66491370664A062876
:101E300084F800E00B7013702BD01B22634B4FF41F
:101E4000E13B1A700522624B83F800E0614B1A7087
:101E500042F6F8236380604B402063605F4BA360D1
:101E600006F05CFE824600283FF4A5AC12F0E4FDCB
:101E7000B27A00280CBF01230323002A0CBF0022E2
:101E800008229AF902E00192009382465B46544A86
:101E90003AE721224D4BDFF884B11A704C4B83F89E
:101EA00000E04C4B1870D3E74FF0000B4D4B402037
:101EB00083F800B00E23237044F6206363804A4BFE
:101EC00063604A4BA36006F029FE00283FF473AC20
:101ED000B0F800A0464B0AF4825A83F800B0B37AF7
:101EE000BAF5825F90F9020014BF01220322B3B950
:101EF000BAF5825F14BF5B4608238DE80C004021D1
:101F00004FF4E1333B4A06F053FCBAF5825F7FF4AD
:101F10004EAC0022384B1860384B1A7047E4082347
:101F2000EBE70A221B0193FBF2F300223449A3F5ED
:101F3000B06341F822300132102AFAD142F6F82378
:101F40006380304B402063602F4B2270A36006F00B
:101F5000E5FD00283FF42FACB37A90F90200002B86
:101F60000CBF0023082301930323284A0093402138
:101F7000274B06F01DFC1AE4DA077FF541AC0C2272
:101F80002270244A3BE40133042B7FF472AC00201E
:101F900078E4214A934200F09F8141DC023A934267
:101FA0007FF466AE802391E155F9000869F90008D5
:101FB00099000108CDF80008E5F800085100010873
:101FC0004D2A0020E42600204C2A00200C28002066
:101FD000302800204E2A00203FE4000855E4000885
:101FE00079FF0008A72A002001FF00082904010842
:101FF000A52A002055030108241A0020301A0020C9
:1020000048290020B5FB0008E5FB0008FD02010897
:10201000A0680600B9FE00081920C20090D0030095
:10202000B94A9342BED0013293427FF421AE4FF4BD
:10203000807323806380A38822881B02A36053439C
:10204000E360012385F8A039E468C4B14FF0000AC9
:10205000E40A0DF14C0BA2450CDA0AEB04094FEA35
:102060006909102241464FEAC92008F07BFE0F287B
:1020700000F3358108F01AFEA44BE4021C60A44B67
:102080009A78A44B02B101221A70039BA2481B78D4
:10209000052B02BF4FF4C872A04B1A800CF0BEFD96
:1020A000C8229F4B00211A809E4AA5F8A2191378D6
:1020B000A5F8A41943F00803137003239A4A85F87E
:1020C000A1391370994B9A4A19805980994B117014
:1020D0001A799946012A0AD13022974817F0D7FF7A
:1020E0004CF250324FF07E51944808F0F5FB00213D
:1020F000934B85F8D81919605960996099F80530A3
:10210000012B09D110228F4817F0C1FF4CF2503239
:102110008D498E4808F0E0FB8D4B8E4A1B684FF0CE
:1021200001083B608C4B00211B688C489B1A18BF30
:1021300001238B4A85F8188A1370442217F0A7FFF1
:102140000023884C884A20461360C5F81C3A06F0E4
:10215000EDF9029B1B68DA0709D5844B41461B68E1
:102160004046642B38BF6423636406F017FA804B43
:102170001A68984612F0020F09D00121022006F0D9
:102180000DFA7C4B1B6B642B38BF6423A367D8F814
:1021900000100320C1F3400106F000FA01210520E0
:1021A00006F0FCF9744B99F804B01A8C734B0720B5
:1021B00093FBF2F3642B38BF64231BF10001C4F8D6
:1021C000143118BF012106F0E9F999F805A008209B
:1021D0001AF1000118BF012106F0E0F999F8083062
:1021E000002B40F0588199F80930002B40F05381C2
:1021F0003968C1F38041BBF1000F03D1BAF1000F80
:1022000000D15146092006F0C9F90121042006F049
:10221000C5F995F86419062006F0C0F901210A20D5
:1022200006F0BCF9D8F800100B20C1F3800106F0CD
:10223000B5F9D8F800300C2013F0140F14BF0121A9
:10224000002106F0ABF939680D20C1F3802106F0BA
:10225000A5F939684B0507D5337A083B012B9CBF9C
:102260004FF4FA63C4F8B4320E20C1F3004106F013
:1022700095F94FF4804006F051FC68B10022032329
:1022800090F902004FF48041009301924FF4E13342
:1022900006F08EFAC5F8200AD5F8203A63B101217C
:1022A000022385F8241A85F8251A85F8261A0F20A6
:1022B00085F8273A06F072F995F8C53463F07F0384
:1022C00085F8C5341FB0BDE8F08F202323804FF47C
:1022D0008073AFE64023F9E74FF40073F6E700237D
:1022E0005BF8232001320BD10133042BF8D14C468B
:1022F000B1E632F83330002B7EF4F0ADFEF7E6BDE8
:1023000009F1010AA146F2E71740EF00E43A002084
:10231000D43A002070230020743C0020AA1C002026
:10232000A81C0020ED260020F9350020321A0020DC
:10233000441A0020FE350020C80F0020CC0F0020DA
:1023400028230020FC0F0020CDCCCC3E0C10002018
:1023500068180020EFBA000838310020C4150020AA
:1023600058120020DC000020C01500202041002071
:1023700028250020B82200203241002040420F00D2
:102380000022464B00B21A7014F072FB444914F05C
:10239000C3FB0746B4F9A00614F06AFB404914F0E9
:1023A000BBFB0646B4F9A40614F062FB3C4914F0EA
:1023B000B3FB3C490546384614F0A6FA0BF0B9F9D0
:1023C000814638460BF0B5F936490746304614F0D9
:1023D0009BFA0BF0AEF9804630460BF0AAF9314972
:1023E0000646284614F090FA0BF0A3F983462846D7
:1023F0000BF09FF949468246584614F08DFB49463A
:102400000290504614F088FB59460390384614F069
:1024100083FB51460490384614F07EFB41460590FC
:10242000584614F079FB204D5146286008F10040D1
:1024300014F072FB04996860AE60304614F06CFBD7
:10244000039914F061FA0599E860304614F064FBD2
:102450000146029814F056FA4146286107F10040FF
:1024600014F05AFB02996861304614F055FB01469E
:10247000059814F047FA0399A861304614F04CFB14
:10248000049914F041FA4946E861404614F044FBCF
:102490002862FEF7C2BE0121ADE600BF1D04002088
:1024A00035FA8E3CDB0FC93FC0270020000000003A
:1024B0002DE9F047B0F908308CB0DDB2382D064672
:1024C0000C460B8100F0CC8100F2B380042D00F0AB
:1024D0004A8171D8022D00F0318100F23581012D41
:1024E00000F01D815C2D00F0E38401F22D83362D78
:1024F00001F0C28401F2AB822C2D00F0888301F23E
:102500005A82222D01F0CA8401F247820A2D00F07E
:10251000AA82742D336800F00C85772D00F01685A3
:10252000472D40F0208572683046D51A0AF04CFFDE
:10253000052D074640F2138530460AF05BFF002662
:10254000054694E80C009B1A103BAF4AAB42A846E4
:10255000B8BF9DB2D3683946DB1B9D42204688BF79
:102560009DB291460AF05BFF3EB9294620460AF02B
:102570006AFF23685A1C22601E70D9F80C307A1941
:102580009A42D4F800A088BFDD1B08F08FFB2A46D2
:102590005146384608F0E6FB236803442360002ECA
:1025A00000F0AC800022804540F3A8802368013011
:1025B000591C21601A70F6E7202D00F0758111D8A2
:1025C000052D8FD120460B2290490AF01EFF204690
:1025D00008228F490AF019FF07228E4920460AF087
:1025E00014FF8BE0242D00F0DE80282D7FF47AAFDD
:1025F00001250B68884E5A1C0A601D700B68204626
:102600005A190A6006221A700B685A190A600A22BF
:102610001A700B685A190A601D7031880AF013FF8E
:10262000718820460AF00FFF68B265810CB0BDE8E2
:10263000F087802D64D02FD8522D00F0548107D818
:10264000442D7FF44FAF002A58D0744B136055E0EF
:10265000542D00F04E816E2D7FF444AF704B0A680C
:102660001B88511CFF2BA8BFFF236E4D21601370E8
:10267000A968204681F3100189B20AF0E4FE6A4B92
:10268000204619880AF0DFFE2968204601F30F0171
:1026900089B20AF0D8FE31E0822D00F08A800FD393
:1026A000A02D70D0FE2D7FF41DAF00255F4E36F8B3
:1026B0001510204601350AF0C6FE042DF7D11DE0A5
:1026C0004FF6FF765A4B0A2519689F68B142A8BF9A
:1026D0003146236821EAE1715A1C226089B2204602
:1026E0001D700AF0B0FE05FB07F1B142A8BF3146EC
:1026F00021EAE17189B220460AF0A5FE012593E79F
:102700000A684C4B511C1B8821600A21FF2BA8BF73
:10271000FF2311702268511C21601370EEE70B68D3
:102720005A1C0A6000221A700B685A1C0A601D703D
:102730000B685A1C0A6024221A7075E704223E496D
:1027400020460AF062FED9E70B6801255A1C0A6090
:1027500002221A700B685A1C0A601D700B685A1905
:102760000A600022E8E72A46344920460AF04DFE76
:10277000334B204619780AF066FE23685A1C226003
:1027800000221A70BAE72F4B204619680AF047FE5C
:102790002D4B204619680AF042FE2C4B2046196842
:1027A0000AF03DFEAAE72A4B204619680AF037FED8
:1027B000A4E7284B20461A780B681A4D591C216053
:1027C0001A70254BD9880AF03EFE154B22681B88EB
:1027D000511CFF2BA8BFFF2321601370A96820465E
:1027E00081F3100189B20AF02EFE2968204601F318
:1027F0000F0189B20AF027FE184B1A782368591C7A
:1028000021601A707AE700BF3804002086BF0108F3
:1028100092BF01089BBF01083C11002023EE000875
:10282000321A002028230020F4350020FC2200204A
:10283000FC0F0020C80F00207CBF010881BF0108E9
:10284000E40A0020E8F7FF1FECF7FF1FF0F7FF1F77
:1028500068180020441A0020FE350020F9350020B9
:1028600001250B685A1C0A601D700B685A190A6012
:1028700005221A700B685A190A600A221A700B682E
:102880005A190A6000221A70B14B2268197850193F
:1028900020601170226859785019206011709A7860
:1028A00023685919216047E7AA4D0B686A78591CBB
:1028B00021601A7023682A78591C21601A702368D5
:1028C000AA78591C21601A70E98820460AF0BBFDDD
:1028D00023682A79591C21601A7023686A79591C67
:1028E00021601A700AE70B685A1C0A6000221A70ED
:1028F00004E70B685A1C0A6000221A700B68591C06
:1029000021601A70FAE600264FF6FF78924FDFF842
:1029100084920196029603960496F157481C0BD0B8
:1029200048FA06F3DA0707D5B9F800303341DB0778
:1029300002D503A808F009F801360B2EEDD10026C8
:102940000FF20429D9E9008932464046494613F07E
:1029500027FB002100F0010050EA010307D0F0B28C
:102960000FF0B2FD18B1314603A807F0EEFF0136B3
:10297000242EE9D1794BDFF820821B78DF074FF056
:1029800000073E4642BF039B43F0010303933946D1
:10299000404607F0E6FF48B1394603A807F0E1FFDB
:1029A00018B1314601A807F0D0FF01360137242FB6
:1029B000EDD16B4B2046B3F850100AF044FD694B43
:1029C00020461988684F89B20AF03DFD674B2046C2
:1029D00019684A01C1F3400302F020021343C1F316
:1029E000800243EA4203C1F3C00243EA8203C1F317
:1029F000401243EAC20301F0100119430AF023FD1B
:102A0000042220460DEB02010AF0FFFC23683A780D
:102A1000591C21601A70564B204619886429A8BF9A
:102A200064210AF010FD962D18D123685A1C2260EB
:102A300003221A7023687A78591C21601A700822C0
:102A4000193E96FBF2F2236882F30402591C2160BE
:102A500020461A7002A90AF0D8FC4FE60021204651
:102A60000AF0F1FCEBE7434813F092FA00233E49E9
:102A700098427FF743AE5A18157922680133561CE5
:102A800026601570F4E710223B4920460AF0BDFC91
:102A900034E600251826394FDFF8008106FB057360
:102AA000597C31B9204601350AF0CDFC082DF5D10D
:102AB00024E658F8250015F01FF881B2F2E736F841
:102AC000151020460AF0BFFC01353B789D42F6DB2D
:102AD00014E62B4D204629880AF0B5FC698820466B
:102AE0000AF0B1FC0A23B5F90410204691FBF3F17A
:102AF00089B20AF0A8FC01E6224B204619680AF0C8
:102B00008EFC214B204619880AF09DFCF6E51F4DEE
:102B1000204629880AF097FCA98820460AF093FCF1
:102B2000298920460AF08FFCE8E5194B226899783C
:102B3000501C206011705A782368591C21601A704B
:102B4000DCE500BFAFF3008090E33FF40800000035
:102B500038110020FE350020AAA20108A43500206B
:102B6000DC000020B83B00200816002028250020AB
:102B70002E1600200C160020542300208025002053
:102B80008C310020A01000201C150020BC0C00205F
:102B900070110020F6350020CC0C00200823002006
:102BA0000021AC48036801EB41029D5C23680131C0
:102BB0005E1C26601D7003680A2913445D78236833
:102BC00003F1010626601D70036813449A78236898
:102BD00003F1010525601A70E4D18FE52168481CD6
:102BE00020600A7013F8012F002AF7D186E501252D
:102BF00023685A1C22601D7016E5974D2046A9894E
:102C00000AF021FC698920460AF01DFC76E5934D07
:102C100023682A7A591C21601A70A98B20460AF071
:102C200012FC298B20460AF00EFC698B20460AF024
:102C30000AFC2368EA7C591C21601A70E98C204642
:102C40000AF001FC298D20460AF0FDFB2368AA7FCB
:102C5000591C21601A70236895F82020591C2160A6
:102C60001A70A98C20460AF0EEFB2368EA7A591CF8
:102C700021601A70E96820460AF0D1FB23682A7C9B
:102C8000591C21601A70236895F82120591C216075
:102C90001A7033E5724D23682A78591C21601A7026
:102CA00023686A78591C21601A70698820460AF0E6
:102CB000CAFB23682A79591C21601A70E9882046CA
:102CC0000AF0C1FB23682A7A591C21601A7015E5A5
:102CD000236816F81510581C06EB45022060197081
:102CE0005178204601EB810101EB810101F2EE21D7
:102CF00089B20AF0A8FB01353B789D42E8DBFDE490
:102D0000564B5A7D2368591C21601A70F6E4002541
:102D1000544E56F82510204601350AF080FB202D30
:102D2000F7D1EBE44F4D002306272846002107FB8F
:102D300003F6226802F1010EC4F800E01370226865
:102D400002F1010EC4F800E011708A192A4492F8C9
:102D5000C0E02268013102F1010C0629C4F800C06C
:102D600082F800E0E5D10133062BDFD10022216893
:102D70004D1C25600B7021684D1C25600A70811860
:102D800091F8E450216801324E1C0B2A26600D7028
:102D9000EDD123685A1C226007221A7023685A1C3E
:102DA000226000221A70236890F8F020591C2160DC
:102DB0001A70A3E407F09CFE002814BF032202222D
:102DC0002368294D591C21601A70298820460AF071
:102DD00026FBE96820460AF022FB07F069FE01465F
:102DE00020460AF01CFB89E4012523685A1C226056
:102DF0001D701E4B2268997850192060117022684E
:102E000019785019206011705A7849E50025236817
:102E100029465A1C22601D70236820465A1C2260D5
:102E20001D7023685A1C22601D700AF0F8FA2946AA
:102E300020460AF0F4FA61E40D4D204629880AF094
:102E400002FB698820460AF0FEFAA98820460AF0AB
:102E5000FAFA53E420250020F0260020383600201E
:102E6000B83100202434002038040020D43A002057
:102E7000A42D0020AB4B1A782368591C21601A70CE
:102E8000A94B9A782368591C21601A70A74B9A782D
:102E90002368591C21601A7030E4B278591C2160F3
:102EA0001A70A34B1A782368591C216000F010BED9
:102EB0009C4E236872799F4D591C21601A702B68B3
:102EC0002046198C0AF0BFFA2B682046598C0AF06C
:102ED000BAFA718920460AF0B6FAB18920460AF09A
:102EE000B2FA2B682046998C0AF0ADFA2B6820467E
:102EF000D98C0AF0A8FAF18920460AF0A4FA318A9E
:102F000020460AF0A0FAFFF7F9BB874BDA7823686E
:102F1000591C21601A70884B1A782368591C21604B
:102F20001A70824BDA782368591C21601A70FFF7F7
:102F3000E5BB72689A420FBF00215A1C32601978B3
:102F40007E4A20460BF0A2FFFFF7D8BB72689A4278
:102F50001DBF5A1C326019780021794AF1E7012619
:102F60008025FFF7EEBA292D2AD0392D1ED0212D2C
:102F700035D15A1C32601A46724D12F8021B304687
:102F8000697032605A782A70DA1C32609B78AB70B4
:102F90000AF030FA3368E8805A1C32601A4612F898
:102FA000021B297132605B786B7105E05A1C32603C
:102FB0001A780A2A00F0AE874FF0FF35FFF734BBCE
:102FC0005A1C32601B780A2BF6D130460AF012FAEE
:102FD0005D4D288030460AF00DFA6880ECE777688E
:102FE0005D2DA7EB030700F0B78300F25C81352D60
:102FF00000F0B58200F2B2802B2D00F067842FD84C
:10300000232D00F0948217D80B2DD5D10021112249
:103010004E4817F03CF8102F4FF0000328BF102740
:103020004B49BB42BFF46AAB3268501C3060107829
:103030005A1810710133F4E7252D00F03C84272D38
:10304000BAD130460AF0D6F9424D286030460AF02F
:10305000D1F9686030460AF0CDF9A860FFF74EBBA1
:103060002F2D00F05D844FD82D2DA5D15A1C326034
:103070001B78394D30462B720AF0BCF9A8833046D4
:103080000AF0B8F9288330460AF0B4F93368688347
:103090005A1C32601B78082FEB747FF62FAB30463A
:1030A0000AF0A8F9E88430460AF0A4F90C2F288524
:1030B0007FF624AB336830465A1C32601A4612F849
:1030C000021BA97732605B7885F820300AF092F90C
:1030D000102FA8847FF612AB336830465A1C32603A
:1030E0001B78EB720AF070F93368E8605A1C3260A2
:1030F0001A78162F2A747FF601AB9A1C32605B781F
:1031000085F82130FFF7FABA312D00F02284332DF3
:103110007FF452AF5A1C32601A780F4B5A75FFF782
:10312000EDBA00BFBA3B0020F02600206411002059
:10313000582C0020202500208827002001EE0008C0
:1031400065ED0008FE3500203C1100200C16002023
:1031500008160020BC0C002038360020482D00F056
:10316000A68339D83C2D3FF4C9AA23D8372D7FF444
:1031700023AF0723B7FBF3F3C3EBC302BF1A7FF4FC
:103180001BAFDFF874A35FFA83F8FBB298453FF4F6
:10319000B5AA002533685A1C326093F900300AEB57
:1031A000C50999F902209A4200F0DE860135042D06
:1031B000F5D101E73E2D00F0AE81412D7FF4FCAE4C
:1031C0000023C2493268501C306012785A540133CF
:1031D000082BF7D1FFF792BA4E2D00F07E8320D84E
:1031E0004C2D7FF4E9AE5A1C32601A46B84D12F8E5
:1031F000021B3046297032605B786B700AF0FAF877
:10320000336868805A1C32601B7830462B710AF094
:10321000F1F83368E8805A1C32601B782B72FFF794
:103220006DBA512D00F02E835B2D7FF4C5AE5A1C74
:1032300032601A46A74D12F8021BA74FA9703260E0
:103240005978A64A30461170DA1C32609A783A7181
:103250001A1D3260DB78042BA8BF0423BB700AF070
:10326000C9F896E80C009B1A012B388003DD304624
:103270000AF0C0F8F881336872689A4206D05A1C86
:1032800032601B78003318BF0123EB710BF022FF73
:10329000336872689A423FF431AA5A1C32601B7834
:1032A000FB70FFF72BBAD42D00F0C98100F28980A2
:1032B000CC2D00F07B8168D8612D00F0928241D83E
:1032C0005F2D7FF479AE30460AF094F830460AF06C
:1032D00091F830460AF08EF83368814D9A1CD5F883
:1032E000008032605A78304688F82F20DA1C32602D
:1032F0009A7888F83A201A1D3260DA78073388F80D
:103300003B2033600AF076F8A8F83E003046D5F846
:1033100000800AF06FF8112FA8F83C002B460CD95A
:1033200032682868511C3160114611F8025B80F840
:1033300031503160527880F8322018680FF092F9DD
:10334000FFF7DCB9C82D00F09880CA2D7FF434AEA9
:10335000634B1868034600F11E0532680333511CA5
:103360003160114611F8027B03F8037C316051781B
:1033700003F8021CD11C3160927803F8012C9D42A5
:10338000EBD10FF06FF9FFF7B9B9CE2D00F06E82D7
:10339000C0F06182D02D00F05182D22D7FF40CAEAE
:1033A0005A1C3260187806065ED44E4B1B78DD0737
:1033B0003FF5A4A9032828BF00200BF0C3FDFFF7A9
:1033C0009DB9DC2D00F0B68125D8D92D00F08E8175
:1033D00013D8D62D7FF4F0AD0025434FDFF81C81C4
:1033E0003B789D42BFF68AA930460AF003F813F0F5
:1033F0003BFB48F825000135F2E7DA2D00F0858126
:10340000DB2D7FF4D9AD364B4A223849186814F0C9
:103410000DFAFFF773B9EF2D72D014D8DD2D00F03F
:10342000AB82DE2D7FF4C8AD304609F0E3FF2A4DB4
:103430002882304609F0DEFF6882304609F0DAFF64
:10344000A882FFF75BB9F22D00F02581FA2D7FF4F9
:10345000B3AD244B1B78DB073FF5AEAD0BF088FD19
:103460000BF0B2FEFFF74AB900F07F00032828BF37
:10347000002012F0FBFCFFF741B9C7F34707122FFA
:103480003FF69AAD00250DF10C08BD420CDB002380
:10349000174A03A99F420ED10021154A122B10D1C1
:1034A0000125144BFFF7A7BB304609F0A3FF28F80E
:1034B00015000135E9E731F8130022F81300013354
:1034C000E8E722F813100133E8E700BF38360020A0
:1034D000B8310020BA3B002078230020582C00206F
:1034E00020250020A435002004230020DCB00108A2
:1034F000EA290020E8290020324100205825002038
:10350000304609F077FFC04DA881304609F072FFC0
:103510006881FFF7F3B85A1C32601A46BB4912F8AB
:10352000020B887032605B784B70FFF7E7B85A1C6B
:1035300032601D78132D3FF63FAD00210C279A1CF9
:1035400032605A78DFF8ECE207FB01E090F808C03F
:10355000944500F0EE8401312429F5D12CE55A1C64
:10356000326019780E293FF627AD9A1C32605D78DB
:10357000032D3FF621AD06224A43A54881184D711F
:10358000DD1C35609D7885541A1D3260DA784A70EA
:103590005A1D32601A798A709A1D32605A79CA703F
:1035A000DA1D32609B790B71FFF7A8B8092F7FF6FF
:1035B00003AD98495A1C0D6832601A4612F8020B86
:1035C0008846287032605B78681DAB700023022B40
:1035D0000CBF4FF0FF0E4FF0640E316801334A1CF0
:1035E00032600A787245A8BF7246032B00F8012B9F
:1035F000EDD18B1C33604B783046642B28BF64239D
:103600002B72CB1C33608B78EB700B1D3360CB7847
:103610002B7109F0EFFE0A2F68810CD03368D8F8BF
:103620000020591C316019780B2F51721FBF991C53
:1036300031605B7853700EF097FFFFF75FB80F2F84
:103640007FF4BAAC5A1C32601D78072D3FF6B4AC3B
:103650000C27304609F0CEFE6F43DFF8DC8108EB23
:103660000705A880304609F0C5FEE880304609F01D
:10367000C1FE336828815A1C32601A4612F8021BB8
:103680003046A97232605B78EB7209F09DFE48F813
:103690000700FFF733B85A1C32601A780F2A3FF63A
:1036A0008BAC991C31605D785B48C2EBC2028554DB
:1036B0008118DA1C32609A784A701A1D3260DA7802
:1036C0008A705A1D32601A79CA709A1D32605A790E
:1036D0000A71DA1D32609A794A7103F10802326088
:1036E000DB798B710CF0B6FFFFF708B8304609F0B4
:1036F00081FE4A4D2880304609F07CFE68803046C5
:1037000009F078FEA880FEF7F9BF19465A1C32600E
:1037100011F8020B424A10703160597830465170EE
:10372000D91C31609B78937009F064FE3B4BD880C4
:10373000FEF7E4BF5A1C32601A463A4912F8020BEF
:10374000087032605978304A9170DA1C32609A7889
:10375000354B9A70FEF7D2BF5A1C32601B78334D3E
:10376000DFF8C0803046D5F8009088F8053009F0C1
:1037700041FEA9F820003046D5F8009009F03AFE45
:10378000052FA9F8220023D9304609F033FEA8F806
:103790000A00304609F02EFEA8F80C003046D5F895
:1037A000009009F027FEA9F824003046D5F80090D3
:1037B00009F020FE0D2FA9F8260009D9304609F09E
:1037C00019FEA8F80E00304609F014FEA8F8100003
:1037D0000BF080FC11F06CFE28680FF001F8FEF78A
:1037E0008DBF5A1C32601A46074912F8020BC87086
:1037F000326059780E4A1170DA1C32609A780A4B9E
:10380000DA70FEF77BBF00BFF026002070110020A9
:103810001C190020AC2D0020862B0020A42D002098
:1038200080100020BA3B00206411002020250020D9
:103830008827002024AF0108F82B0020B44B1B7808
:10384000D8073EF55BAF0BF091FE0BF091FB0BF050
:10385000BBFCFEF753BFAE4B1B78D9073EF54EAF0E
:103860004FF4C872AB4B1A80FEF748BFA84B1B78C9
:10387000DA073EF543AFA84A137843F00403137008
:10388000FEF73CBFA54A1278012A3EF637AF19462B
:103890005A1C326011F8020BA14A907031605978BD
:1038A0001170D91C31609B785370FEF727BF07F069
:1038B0003BFAFEF723BF00239A4D30462B6009F0F8
:1038C00083FD2B6818432860FEF718BF5A1C32602E
:1038D0001A78954B1A70FEF711BF5A1C32601F7888
:1038E000112F3FF669AB9A1C32605B788F4D3046E2
:1038F00005F8173009F07EFD40F6CA039842A8BFCC
:10390000184640F2EE239842B8BF18461923A0F299
:10391000EE2090FBF3F005EB47056870FEF7EEBE76
:10392000834D05F14007304609F064FD3368A5F882
:1039300080005A1C32601A4612F8021B043585F8C2
:103940007E1032605B7885F87F30AF42EBD1FEF7B6
:10395000D5BE5A1C32601D781F2D3FF62DAB052FAA
:103960007FF42AAB304609F02FFD714B43F8250058
:1039700011F010F9FEF7C2BE5A1C32601A4612F856
:10398000020B3260DA1C597832609A7811F082F8B2
:1039900000287EF4B3AEFFF70FBB262D3FF4B7A887
:1039A0002A2D7EF4B6AD604B1A782368591C21602D
:1039B0001A70FEF7A3BE302D3FF4A9A91BD82E2DF7
:1039C0007EF4A7AD5A4D05F14006B5F880102046AB
:1039D00009F039FD236895F88220591C21601A707E
:1039E000236895F883200435591CB54221601A706C
:1039F000EBD1FEF783BE322D3FF482A9342D7EF445
:103A000088AD4C4B03F15A0122685879551C25604A
:103A1000107022681878551C25601070226858783C
:103A2000551C2560107022689878551C2560107010
:103A30002268D878551C25601070226818790633E2
:103A4000551C994225601070DED1FEF757BE462DF9
:103A50003FF4B0A919D83B2D3FF4C9A808D83A2D96
:103A60007EF457AD0021204609F0D9FCFEF746BE92
:103A70003D2D3FF45AA8402D7EF44BAD08222E492F
:103A8000204609F0C2FCFEF739BE4F2D3FF4BEA917
:103A90000AD84B2D3FF4FEA84D2D7EF43AAD0025FB
:103AA000264F224EFFF728B9502D3FF49DA95A2DDD
:103AB0007EF42FAD224E2368F278002A3FF4EDA960
:103AC0005A1C226008221A7023685A1C22600122A4
:103AD0001A701C4D23682A79591C21601A702368BA
:103AE000AA78591C21601A702988204609F0ABFC7D
:103AF000E989204609F0A7FC2368F279591C216066
:103B00001A702368EA78591C21601A70FEF7F6BD16
:103B1000A4350020AA1C0020ED26002070230020E0
:103B2000D43A0020681800202C250020E92A002023
:103B3000243400201C19002038360020D829002009
:103B4000BA3B002078230020702D3FF429A800F212
:103B5000E180672D3EF497AF00F28A80602D3FF43C
:103B6000D4A94FD85E2D7EF4D4AC0021204609F0B4
:103B70006AFC0021204609F066FC0021204609F07D
:103B800062FC2368AE4D5A1C226000221A702B681A
:103B900093F82F102368581C206019702B6893F835
:103BA0003A102368581C206019702B6893F83B105A
:103BB0002368581C2060197023682046591C216016
:103BC0001A702368591C21601A702368591C2160DF
:103BD0001A702B68D98F09F036FC2B682046998F14
:103BE00009F031FC2B6893F831202368591C2160BF
:103BF0001A702B6893F832202368591C21601A70C0
:103C0000FEF77CBD652D3EF47EAE662D7EF481AC64
:103C10008C4E0025328AB2F5007F8CBF0427012725
:103C20007319596B204691FBF7F1043589B209F0FD
:103C30000AFC0C2DF4D10125834E844F396A56F8C5
:103C4000250013F01DF813F057FF013581B220460F
:103C500009F0F9FB042DF1D100257D4E36F8251031
:103C60002046013509F0EFFB032DF7D1FEF746BDE5
:103C70006C2D3EF42EAF0AD8682D3EF40AAF692DA4
:103C80007EF447AC0025734F734EFEF71EBF6D2DBB
:103C90003EF432AF6F2D7EF43CAC704D2B681A7839
:103CA0002368591C21601A702B689A782368591C64
:103CB00021601A7000232A681A445179226801335E
:103CC000501C032B20601170F5D12B6820461A7A06
:103CD0002368591C21601A702B68DA782368591CF4
:103CE00021601A702B681A792368591C21601A7098
:103CF0002B68598909F0A7FB2B685A7A2368591C4D
:103D000021601A702B685A782368591C21601A7038
:103D1000FEF7F4BC7E2D3FF4ADA825D8782D6DD0EC
:103D200005D8752D7EF4F5AB4D4BFEF75BBF7C2DB2
:103D30003FF482A87D2D7EF4ECAB4A4B22681978C3
:103D4000501C2060117022685978501C206011703E
:103D50009A7823682046591C21601A70424BD988F2
:103D600009F071FBFEF7CABC962D3EF4CCAD14D819
:103D70007F2D3EF4D7AF832D7EF4CBAB3B4D204659
:103D8000298A09F060FB698A204609F05CFBA98A50
:103D9000204609F058FBFEF7B1BCF02D3EF42DAFE4
:103DA000F12D7EF4B6AB324B03F170012268187826
:103DB000551C2560107022685878551C25601070BD
:103DC00022689878551C256010702268D878551C98
:103DD0002560107022681879551C256010702268C3
:103DE0005879551C25601070226898790733551C46
:103DF0008B4225601070D9D1FEF780BC1D4D05F1B6
:103E00006006A988204609F01EFBE988204609F0D3
:103E10001AFB2989204609F016FB2368AA7A591C47
:103E200021601A702368EA7A591C21601A7055F8CB
:103E30000C1B204609F0F3FAB542E2D1FEF75EBC56
:103E400020250020B822002020410020CC3B00206B
:103E500088330020D8290020CC350020AC2D00204C
:103E6000B4A2010880100020A42D00207823002097
:103E7000862B0020F82B00204B4D4C4F05F12006DF
:103E8000002395F90220D957914226D00C33302BCC
:103E9000F9D10835B542F3D1FEF730BC444D05F1F8
:103EA000500628780AF0DEFF2368027A591C216048
:103EB0001A7023686A78591C21601A702368AA78DE
:103EC000591C21601A702368EA780435591CAE42E7
:103ED00021601A70E5D1FEF711BC23682046591CF9
:103EE00021601A70298809F0AEFA2368EA78591C13
:103EF00021601A7023682A79591C21601A7023687E
:103F0000AA79591C21601A7023686A79591C2160AA
:103F10001A70BEE79A1C32605978264A1170D91C73
:103F2000316099785170191D3160DB789370FFF71B
:103F300043B801781E4A002002F82510D91C3160D0
:103F4000997802EB85025170191D3160D978917012
:103F5000591D31601B79D3700EF07CFA164B80F03E
:103F600001001870FEF7CABB89F80230304609F02C
:103F700041FA33682AF8350019465A1C326011F8A4
:103F8000022B013789F8032031605A7889F8042020
:103F9000DA1C32609A7889F806201A1D3260DB78C4
:103FA00089F80530FFF7F1B8324100205841002070
:103FB0007C18002038110020000000202DE9F04F6F
:103FC000B34B9DB01B780690012B07D1B149B24A83
:103FD0000968C9691180B14909885180B04D2A78B2
:103FE000002A00F0D384072B40F0F8810DF098FBF5
:103FF0000790AC4F3B68059713F4806F05D0AA4833
:10400000836813B100F144019847A84BA8491B6885
:10401000B1F906405A890891944280F2E2814FF04A
:104020007E536B6095F90C304FF00009002B14BFE4
:1040300001234FF0FF339F4A95F809B0168B95F88E
:1040400008A09D4F04930992089B33F91980A8EBAF
:1040500006000028D8BFA6EB0800B0F5FA7F82F270
:104060003D83B9F1020F02F03F83824580F2CC819B
:10407000A0EB0A0012F0FCFCB04547F82900C2F2A0
:10408000418309F10109B9F1030FDDD1059B1F68D7
:1040900017F4805800F0BA81B4F5FA6F2046A8BF33
:1040A0004FF4FA60B0F57A7FB8BF4FF47A70A0F59C
:1040B0007A724FF0640C92FBFCF38049581C31F982
:1040C00013E031F91000DFF8F091A0EB0E016FF072
:1040D000630000FB0320484390FBFCF0704400B2F7
:1040E00012F0C6FC8246C9F80C00B8F1000F1DD0D2
:1040F0001D200EF0E9F9C8B1714BDB78B3B97149F5
:10410000504612F0FFFB12F0E3FE4FF47A7300B258
:10411000000390FBF3F3C6F5FA6000B2584340F396
:104120000F30304412F0A4FCC9F80C00664B1E8816
:1041300072063BD5654BB3F904000A2390FBF3F0FC
:10414000EB89C01A00B212F093FC614912F0E4FC52
:104150006049054612F0D8FB09F0EBFA8346284681
:1041600009F0E7FA544D81462B68594618460593E5
:1041700012F0D2FCD5F804A004905146484612F043
:10418000CBFC049A0146104612F0BCFB594628604D
:10419000504612F0C1FC059B82461946484612F073
:1041A000BBFC0146504612F0AFFB68604A4B3C4DE9
:1041B0001B6813F0140F1AD016F4027F17D0474B68
:1041C000DFF8F490197811F0100100F034812B7CA5
:1041D0006869002B0CBF01234FF0FF33584312F0E6
:1041E00047FCD9F8041012F08FFBC9F804003C4BCF
:1041F000DFF8C0901A780593A2B1B9F81A30A3423B
:1042000010DB384B1B78012B01D0192B02D1364A19
:10421000927B3AB90E2B05D0082B1FBF0023264AEC
:10422000EB63936095F84240002C65D0B30763D0F0
:104230002E4B2F491E6A304612F016FE002840F021
:104240004A81304613F0D0FC696C12F065FC13F023
:1042500053FCB0F5617FA8BF4FF4617012F008FC09
:10426000244912F059FC09F064FA0646204612F07F
:10427000FFFB314612F050FC13F03EFC00B212F08E
:10428000F7FB0D4C0146E06812F03EFBE06033E0C6
:1042900024250020B41B0020FC2200202E16002024
:1042A000781000200C360020CC3B0020AC2D0020E4
:1042B000CC35002038360020481A0020B02D0020D0
:1042C0001036002000007A44F63500208C310020A2
:1042D00035FA8E3CDB0FC93F28250020ED26002053
:1042E000000000202C2500207A2C00204C310020DA
:1042F0008FC2753CD06D393A95F848A099F81F40A7
:10430000BAF1000F5CD0794B0420D3F8EC6044F68E
:1043100020639E42A8BF1E46B6F57A7FB8BF4FF411
:104320007A76B6B2A5F84A600EF0CEF808B9FF006A
:1043300046D54FF47A73B6FBF3F6642393FBF6F697
:10434000DFF8BCB1142EA8BF1426DBF80030B8F19A
:10435000000F00F0C280DF8E7F086549EB6CD1F85A
:104360000C805A1CEA6405EB430340460892049310
:1043700012F0AEFD089A049BB242A3F85000A4BF0D
:104380000023EB64EB6C05EB4303B3F9500012F030
:104390006FFB0146404612F0B5FA12F099FD00B2EB
:1043A0000028B8BF4042B84240F39A80DBF80030A2
:1043B000188F12F05DFB4F4912F0AEFB059B586061
:1043C00099F81E30002B00F0BE81022B00F09A807D
:1043D000032B00F08C81484B588898E0002307930A
:1043E00007E6B4F5FA6F187ABFBFA31A5843C2F5AF
:1043F000FA6290FBF2F0C0F1640012F039FB3F4921
:1044000012F08AFB68600DE6002033E6099B598BA9
:104410008C420EDBB4F5FA6F2046A8BF4FF4FA6069
:104420004FF47A72401A5043C1F5FA61B0FBF1F2D1
:104430003FE60846F4E7B5F9183095F80BE0A87A9E
:10444000E21ABEF1000F2BD0002AB8BF52428242BE
:1044500010DD01229C42E96185F82020C8BF40425E
:1044600012F006FB0146D9F80C0012F04DFAC9F81B
:104470000C00BCE695F820201AB1AA6A85F8201035
:104480006A6268691844B0F5FA6FA8BF4FF4FA6021
:10449000B0F57A7FB8BF4FF47A7012F0E9FAE6E728
:1044A00082EAE271A1EBE271814209DD022192FB15
:1044B000F1F2EA62012285F8302085F82020E0E759
:1044C00095F82020002ADCD0AA6A85F830E06A62DC
:1044D00085F820E0D5E70020D0E6B3F936703CE758
:1044E0004FF07E53059A53606AE700BFDC0000205E
:1044F000481A00206F12833AD82900200AD7233C9B
:1045000020250020B5F84A0000F57A7080B2023408
:10451000E4B2BAF1000F00F0FF80002800F0FC8048
:104520008D4B00261B688D4FB0FBF3F000B2A5F851
:10453000780012F09DFA01464FF07E5012F0A0FB79
:104540008046DFF8209207F1100AA642C0F2D78019
:10455000834B1B78092B11D1824B834E186813F0C3
:10456000CBFA824B3080D3F8EC004FF47A7390FB97
:10457000F3F012F07DFA12F0ABFC7080B5F97830F0
:10458000002B40F3E28000273E46DFF81482DFF87C
:10459000D4A1A8F11009A742C0F2C48095F8483010
:1045A0000024002B18BF0226714BDFF8F891D3F8D6
:1045B00000806B4B1B78089308F105030993B44204
:1045C00040F3F280089B6B4C092B07D1664EB4F880
:1045D0007830606BB38012F07BFCF080664B93F810
:1045E0002160002E60D01E200DF06EFF00285BD0F1
:1045F000624B1B88580657D494F8B430B34214D099
:1046000084F8B460304612F033FA5D4912F084FA4F
:104610005C49064612F078F909F08BF85A4B98601D
:10462000304609F086F8C4F8B800059B6E6BD3F8E5
:1046300008903046494612F06FFAD5F83C80D5F81C
:10464000B87082463946404612F066FA0146504636
:1046500012F058F94D49824612F006FC08B9DFF80D
:104660002CA14B49504612F009FC08B9DFF820A1F3
:1046700049464046C5F834A012F04EFA3946804605
:10468000304612F049FA0146404612F03DF93F49E2
:10469000064612F0E9FB00B93C4E3D49304612F0A7
:1046A000EDFB00B93A4EEE63002384F84830394BF5
:1046B0001B78002B40F05D81374DAA78002A00F06E
:1046C0005881364C2378013B0D2B00F23F81DFE807
:1046D00013F0110124012E0123023D013D013D0291
:1046E00051026C0589059A05B905C405CD0599F8EF
:1046F0002000C0EB401300EB8300C00006E75AF82F
:10470000261059F8260012F0FDF8414612F004FA7E
:1047100047F82600013618E7B5F87830013BA5F8D0
:1047200078302BE758F8270059F8271012F0ECF8EA
:10473000022F3E46B8BF022648F827004AF8270055
:10474000F6B2013727E7A5F8783095F84830002B06
:10475000ADD0002622E700BF08250020F41000207D
:1047600024250020481A0020FC220020DC00002024
:10477000AC2D00207810002038360020F6350020BF
:1047800035FA8E3CDB0FC93F0000002000C0F94421
:1047900000C0F9C4C4260020D43A002070230020B1
:1047A000041100200AD7233C022C15BF98F8000002
:1047B00098F8010098F802B098F809B012F058F98A
:1047C000494612F0A9F94FF08041074612F060FB0C
:1047D00060B14FF08041384612F094F8AA4912F0C7
:1047E0009BF90146384612F08FF80746A300049360
:1047F000A64BA74953F8240012F08EF920F000438D
:10480000A44A0493049B42F824000C32824642F8E6
:104810002430BBF1000F20D0584612F029F9494648
:1048200012F07AF983465146504612F075F9049910
:1048300012F072F9594612F06FF959460A904FF08A
:104840007E5012F05FF80A9A0146104612F05CF8AA
:104850000146504612F060F982468F49384612F000
:104860005BF9514612F058F9099B074613F8010B02
:10487000099300B312F0FCF8494612F04DF904997F
:1048800012F04AF98549824612F002FB68BB00210A
:10489000504612F0DFFA50BB51464FF07E5012F0F6
:1048A00031F801464FF07E5012F0EAF901463846E1
:1048B00012F032F90746089B0C2B05D1384612F04E
:1048C00007FB774B23F814007649384612F0CCFAF0
:1048D00000B9744F7449384612F0D0FA00B9724FDB
:1048E000724BA200D750013469E64946DAE74FF02F
:1048F0007E51D7E76E4B1B78D90707D5802010F083
:1049000067FF08B103F03CFF12F01AFE1F200DF004
:10491000DBFDD8B10C23237018E00022654B1A6030
:10492000654B1A60654A12685A600323F3E710F07A
:10493000DBFA614E614B1A6873686433934205D2A7
:10494000402010F0A9FA002800F0C28010F0F4FA1C
:104950000646002800F0918423780C3B022B08D9EE
:1049600001232370564B93F8FB2012B1002283F8E9
:10497000FB20544B1B78072B05D10CF0D1FE079B75
:10498000C01A474B988000224D4B1A704D4F3B7810
:10499000072B40F0CC840CF0C3FE07904A4C6368B0
:1049A00020469847A246002855D00026B4F8A850C3
:1049B00084F84960DFF81491002D40F00185E26A27
:1049C000B4F9243094F84A109B1AA363226BB4F90B
:1049D000263004F138009B1AE363626BB4F9283087
:1049E00004F134089B1A23640AF028F94C46DFF8D6
:1049F000B0900AF5707658F8040F12F039F8DAF82A
:104A0000201012F089F83B788346082B03D113F06D
:104A100073F829F815005946DAF8BC333046984740
:104A2000DAF84434014606F1880098473B7883461B
:104A3000032B03D113F060F829F81500DAF8AC3035
:104A40005946D8F8780398470135032D44F8040FE8
:104A500006F12C06CFD11B4C2278072A05D10CF089
:104A60005FFE079BC01A0E4B1880154B93F801216F
:104A70001D460592002A00F07185013A83F8012154
:104A80001DB0BDE8F08F00BFD7A36841481A0020D1
:104A90006F12033B1411002000004843A4707D3FB7
:104AA000FC22002000C0F94400C0F9C4AC10002072
:104AB000A4350020D03A0020FC240020901B0020C8
:104AC0007810002024250020CC3B0020204100202D
:104AD000DFF864834027C246DFF86093336818F834
:104AE000030068B110F0A6FAD9F80030013F03F1D5
:104AF000FF33C9F80030336803F101033360EDD1AF
:104B000033681AF80330002B7FF420AF33604FF086
:104B1000FF3373600423FEE610F0E6F9934A502158
:104B2000A2F10C0301932623029200934920A2F1E3
:104B30000A03163A07F07AFF00287FF407AF4FF018
:104B4000FF328B4B18605A600723E4E610F0CCF973
:104B5000052300210093874B02910191A3F10802E4
:104B6000532007F063FF00287FF4F0AE804B1860FD
:104B70000823D0E610F0B8F97F4B804E186812F089
:104B8000BBFF8046D6F8BC0012F0B6FF814640203D
:104B900010F082F9314600287FF4D8AE744E784F79
:104BA00033687878492B01F28D85DFE813F04A00ED
:104BB00050005E00650069006E00730078007D00A3
:104BC0008400890095009F00A400AF00B400B900E4
:104BD000BE00C600CE00D600490151015901610155
:104BE000690176017F01880191019A01A301AC015D
:104BF000B501BE01C401CD01D301D901DF01E50139
:104C0000EB01F201F901000206020C0213021A0282
:104C1000200226022C02320236023A023F024402ED
:104C200049024F02AB02B802BD02C202C702CC0267
:104C3000D102D702DC02E102E602EB02F002F50249
:104C4000F902504A5049514807F000FC09E0504B26
:104C50004C4A01934F4B504900935048504B07F03A
:104C6000F5FB33680133336070E64E4B4E4A4F49D3
:104C70004F4807F0EBFBF4E74E4A43494E48E3E761
:104C80006B782A784D494E48F3E74E4B4E491A8AC5
:104C90004E48D9E74B4B4C495A8A4D48D4E74FF020
:104CA0007E524C494C48CFE71FFA89F31FFA88F22D
:104CB0004A494B48DDE74B4B4B491A8A4B48C3E7FF
:104CC0004B4B1B68DA0404D591F8C020494846498B
:104CD000BAE70C233360C4E7474948488B784A78E1
:104CE00009780091464907F0B1FBBAE7454B3E49C8
:104CF0001A884548A8E7404B5B79012BB1D1B1F93F
:104D0000C430B1F9C62041483449B2E7404B2E497E
:104D10001A68404898E7404B2B499A783F4893E7F8
:104D20003F4B29491A783F488EE70C2303FB0011BB
:104D30003D4891F8C820244986E70C2303FB001165
:104D40003A4891F8CA2020497EE70C2303FB001162
:104D5000374891F8C9201C4976E70C2303FB001162
:104D6000344891F8D12018496EE700BF5EA30108CE
:104D7000FC24002018A501089023002078100020B2
:104D800008160020A5BF01081ECD0108B1BF01080B
:104D9000E5BF01089BBF0108C5BF0108D3BF0108DB
:104DA000BFBF010892BF010886BF010830CF0108CC
:104DB000EEBF01080C160020FCBF010807C0010867
:104DC0000DC001087823002081CF010818C0010818
:104DD00024C0010837C6010830C0010807C1010816
:104DE0003BC00108B82200201FCF010847C00108BE
:104DF000742300204EC00108FE35002062C0010867
:104E000059C001088E23002072C001087AC0010831
:104E10002041002088C00108BA3B002091C0010851
:104E2000582C0020A1C00108B3C00108BBC0010874
:104E3000C3C00108CFC00108E8A20108D03A002091
:104E40000C2303FB0011844891F8CB208349FBE637
:104E50000C2303FB0011824891F8CC207F49F3E634
:104E60000C2303FB00117F4891F8D0207B49EBE62F
:104E70000C2303FB00117C48B1F8D2207749E3E60C
:104E80000C2303FB001191F8CE3091F8CD2091F85E
:104E9000CF1076480091764925E7764B7648196819
:104EA0004B780A788978009171491CE7714B7348F7
:104EB00019680B79CA78497900916D4913E76D4BF0
:104EC0006F481968CB798A79097A009168490AE7AD
:104ED000684B6C4819688B7A4A7AC97A00916449A0
:104EE00001E7644B684819684B7B0A7B897B00911A
:104EF0005F49F8E65F4B654819680B7CCA7B497CC3
:104F000000915B49EFE65B4B61481968CB7C8A7C7A
:104F1000097D00915649E6E6564B5E4819688B7D3F
:104F20004A7DC97D00915249DDE6524B4B491B68D1
:104F300059481A7E88E64F4B584819680B7FCA7E3D
:104F4000497F00914A49CEE64A4B44491B68544880
:104F50009A7F79E6474B41491B6852481A8C73E6A1
:104F6000444B3E491B6850485A8C6DE6414B3B49C7
:104F70001B684E489A8C67E63E4B38491B684C4884
:104F8000DA8C61E63B4B35491B684A4893F8282088
:104F90005AE6384B31491B68474893F82F2053E6AF
:104FA000344B2E491B68454893F830204CE6314B72
:104FB0002A491B684248DA8E46E62E4B27491B6871
:104FC00040481A8F40E62B4B24491B683E4893F813
:104FD0003A2039E6274B21491B683C4893F83B208F
:104FE00032E6244B1D491B6839489A8F2CE6214B29
:104FF0001A491B683748DA8F26E61E4B17491B688B
:1050000035485A8D20E61B4B14491B6833489A8D4E
:105010001AE60A7A3248114916E64A7A31480F49A7
:1050200012E6314B0D49DA7830480DE62E4B0B492C
:105030001A792F4808E62C4B08495A792D4803E67F
:10504000294A2D49D3892D48528912E6264A2A49F0
:10505000138A2B4892890CE6DBC0010881CF010836
:10506000E3C00108ECC00108F5C001080DC101084A
:1050700004C101082025002013C101081BC101083B
:1050800024C101082BC1010832C1010839C101083E
:1050900041C1010849C1010852C101084BC10108C1
:1050A00059C101086BC1010878C1010883C1010819
:1050B00092C10108A5C10108B2C10108C0C101081F
:1050C000D1C10108E8C10108FAC1010814C20108F0
:1050D0002AC2010838C2010842C201084FC20108B1
:1050E00058DA010860C20108BA3B00206DC201080D
:1050F00076C2010888C2010807C1010898C20108E8
:10510000A6C201088C4B188811F0B2FC8B4911F033
:1051100003FD11F0DDFE8A4902468A4894E5864B7C
:105120008749DA7888488FE5884B85491A78884816
:105130008AE591F8EF208748814985E591F8F820C4
:1051400085487F4980E5854B7D499A7F84487BE58A
:10515000824B7B4993F82020824875E57F4B784944
:105160009A8C814870E57D4B75491A7A7F486BE5CA
:105170007F4B73491A797F4866E57D4B70499A7871
:105180007D4861E57A4B6E491A887C485CE5784B2E
:105190006B49DA897A4857E5BA786949794853E51D
:1051A000794B67491A6879484EE51A200DF08CF959
:1051B000A0B1774B1B888BB9764B14A91B680E20C6
:1051C0001493069B159307F08DF94FF48052724BA0
:1051D0001A800A232370069807F0D2F907F062F9C3
:1051E000FFF7B4BB6D4B1B78002BF4D01A200DF0E9
:1051F0006BF90028EFD16A4B93F8FB30002BEAD112
:1052000009232370EAE7674B1A68674B5B68C8336A
:10521000934211D2AB78032B0BD1644E306803F06C
:105220009BFA00233360624B1B78022B01D103F001
:1052300097FC0123FFF76FBB12F0BEFA0028E9D1FB
:10524000FFF784BB012A01D105F06EFD0D23132069
:10525000237010F03BFEFFF779BB012A04D105F063
:1052600047FC00283FF472AB0E23F0E71F200DF03F
:105270002BF900287FF46AABDBE7EB78002B3FF4D7
:1052800078AB00274FF0010AB9464A4B1B68DB0494
:105290004BBF494B364BB3F804B0B3F814B0584683
:1052A00011F0E6FB454B014653F82700D04611F0BC
:1052B000C7FD00B1C846013746EA0806082FF6B216
:1052C000EDD1384B364F1B68BEB103F59C53083304
:1052D000C7F8FC302378012B7FF44BAB97F8FB30F9
:1052E000002B7FF446ABAB78032B19D012F028F9D2
:1052F000012387F8FB30FFF73CBBD7F8FC209A422C
:10530000E8D82378012B3FF434AB97F8FB30002B1F
:105310003FF42FAB07F042FC87F8FB60FFF729BB97
:10532000802010F055FA00287FF423ABDEE700233D
:105330000793FFF733BB00BFF02600200000C842F0
:1053400081CF0108B8C20108C3C201088827002024
:10535000D0C20108DEC20108EBC2010838360020C5
:1053600001C3010812C301082CC3010846C3010888
:105370007823002058C3010869C301087CC30108D1
:105380008BC301089CC3010868180020A7C301084B
:105390006C23002068230020642300202E25002099
:1053A00078100020901B0020FC240020DC3A002014
:1053B000052500200C360020A42D002058250020B3
:1053C0005E4BD9F800205B78059608934FF47A730A
:1053D000B3FBF2F3C3EB431203EB8203DB009BB29C
:1053E00004933B7804F12C070993554BB3F90690CD
:1053F000049B5B080A93049B9D4201BF00237B63CF
:10540000E3673B604F4BF318B3F924007B6B034415
:105410007B6311F02DFBE26F02F10108B8F1010F7F
:10542000C4F87C8007D10023012D2067E066636704
:105430005DD1002030E0D4F86CA00C9251460B9066
:1054400011F060FA8346404611F012FB01465846BF
:1054500011F016FC514611F057FA0B9B014682469B
:105460002067184611F04EFA594611F055FB616F4E
:1054700011F04AFA012D8346A067C4F86CA060675A
:105480000C9A34D1B8F1010FD3DD104611F0F0FAC7
:105490000146584611F0F4FB12F0EEFD099B8046E0
:1054A000032B05D112F028FB01230FFA80F9059395
:1054B000089BABB1184611F0DBFA414611F0CAFC6B
:1054C00070B1059B13B11E4BA3F806901E4809F05E
:1054D000A5FB00221D4B5A609A60DA60FFF7BBBA49
:1054E0000A9A7B6B1344049A93FBF2F33B600236F7
:1054F000062E07F1040704F114047FF47CAF059B2A
:1055000013B10F4BA3F80690012D0FD10022104BC1
:105510001B689A621A63DA620E4B93F8003113B17A
:105520000D4B1B8813B9012010F0D0FC054AB2F8CE
:10553000A830013BA2F8A830CBE700BFBA3B00205F
:10554000FC220020CC3B0020743C002020410020A5
:10555000B41B00207810002034360020AC4B5B795F
:10556000002B00F03184AB4B1B78013BDBB285F89C
:1055700001312378072B40F02A840CF0D1F80B90EE
:10558000A54B4FF07E501B6807936B680D93D5F8C1
:10559000043119460A9311F0B5F9A04B196811F0BE
:1055A000BBFA4FF07E510C9011F05EFC10B94FF039
:1055B0007E530C939A4B002509939A4B9A4C08936F
:1055C00000230493049BDFF8B0929E0059F82370E7
:1055D000049A964B294653F82280404611F030FC3D
:1055E000E8B9049B09F1D40959F823903846494693
:1055F00011F088F9824620F00041404611F02AFC63
:1056000058B12946504611F043FC002800F0E383CE
:105610004946404611F078F90746854BF750854BCF
:10562000B3F800A01AF0030F3DD0049B022B3AD030
:10563000079B93F8320011F01BFA7F4BF15811F0E1
:105640006BFA079B814693F831B0CBF1000011F063
:105650000FFA80460146484611F0FCFB40B9584617
:1056600011F002FA4946804611F0FEFB00B9C84627
:10567000049A724B33F91200089BB3F90030C01A38
:1056800011F0F6F96E4911F047FA0146404611F063
:1056900039F91AF0010F0E9000F0CE83694B1968AA
:1056A00011F03AFA074694F81431002B57D0049BB6
:1056B000022B54D0089BDFF88481B3F90000049BCF
:1056C00038F91330C01A11F0D3F95E4B07465C4924
:1056D000186811F021FA0146384611F01DFA069AB1
:1056E000D4F818310746D31A574A1268934231DC6E
:1056F0004FF07E510A9811F0ADFB80B3534B5449E3
:105700001A68B1F90A00B8F900301B1A002BB8BFAB
:105710005B42934223DAB8F90230B1F90C105B1AFC
:10572000002BB8BF5B429A4219DD4A4BDFF8289143
:10573000D3F80080D9F80400414620F0004011F071
:1057400089FB60B1D9F80810404621F0004111F002
:105750009FFB20B1002084F814010CF06FF93E4B40
:1057600038463344D3F804A0DFF81091514611F0C5
:10577000C9F88046394B0D98F15811F0CDF94146E2
:1057800011F0CAF9049B0146022B46F8090006D124
:10579000334A344B10681B689847C9F80800099BC6
:1057A00053F8049F0993304B5968304B186811F037
:1057B000B3F90C9911F0B0F92D4BF15811F0ACF987
:1057C000414611F0A9F9494611F09EF8049B834621
:1057D000022B40F0008494F81C31012B02D0192BCD
:1057E00040F0F9834FF00103224940460E9311F037
:1057F0004FFB0E9B00B90346DBB2002B40D02BF0D1
:10580000004029F0004111F025FB00283BD037E093
:10581000BA3B0020582C002020250020202E0020FC
:105820009C220020FA26002078100020142E002050
:1058300080110020F6350020141100208C3100204A
:10584000CDCCCC3DFC2D0020242E0020282E002085
:10585000F02600202C2E002020410020D02D0020FA
:105860002431002020310020000000205C2C00208A
:10587000DC2D002000009642AC1000209422002075
:10588000099BC3F800B0049B022B6DD0A24AA34B26
:1058900051461B68B0589847A14AA24B01461B6865
:1058A000B0589847079B814693F83A30632B00F233
:1058B0009C839D4B1B88002B40F097839B4BF1589A
:1058C0009B4B186811F028F94FF07E51824611F079
:1058D000CBFA08B94FF07E5A964B5046196811F032
:1058E0001BF90146384611F017F9494611F00AF83C
:1058F000914B8146F15811F005F8904B196811F061
:10590000BFF98D4B074646F80390079B93F84890E4
:10591000B9F1000F1ED04FF07E510A9811F0AEFA87
:10592000C0B1874B27F00040196811F0B1FA88B177
:10593000844B28F00040196811F0AAFA50B10120F8
:10594000069BB9F1020F84F81401C4F8183101D193
:105950000CF074F87C4B0D98F15811F0DDF83946D5
:1059600011F0DAF8794B985194F828312BB9784B2B
:10597000F550099B1D60754BF550049B0133049352
:10598000089B02330893049B032B7FF41BAE714EDC
:105990003278072A05D10BF0C3FE0B9BC01A6E4B61
:1059A00058803378012B40F022830BF0B9FE6B490D
:1059B000D4F82C31684A0968C31A93805B1A0690A0
:1059C000D380C4F82C01664B664E1B6893F82F8079
:1059D000654B1B6813F4805F644B00F05583644A89
:1059E000B3F818901278F668D70758BF1A8B614B36
:1059F00058BFA4F83021DF88A9EB070B584611F0F7
:105A000037F882460146304611F02EFA002800F0A1
:105A1000F782D4F83831C4F83431574B1B68C4F8D6
:105A20003C31D4F84011D4F8480111F029F94FF075
:105A30007E51044611F018FA08B94FF07E54002147
:105A4000204611F01BFA00B900244C4DD5F8343132
:105A5000C5F848410793D5F83C3107981946089393
:105A600010F050FF464BC5F854011968384B0B90A5
:105A7000186810F049FF354B196810F045FF41498F
:105A80000C9011F049F8404B82461D6805F1004624
:105A9000314611F0DFF9002840F00A8329465046CC
:105AA00011F0E2F900B9AA46354B5968284B5868FD
:105AB00010F02AFF254B596810F026FF31490D9050
:105AC00011F02AF807460146304611F0E1F930B9E5
:105AD000394628462E4611F0C7F900B93E46284BF4
:105AE00099681B4B986810F00FFF26490E9011F033
:105AF00013F8264B81461D6805F10047394611F021
:105B0000A9F9002844D1294648464F4611F0ACF97E
:105B100000283DD12F463BE03C2E0020382E0020AF
:105B2000A02E00209C2E0020F63500202011002001
:105B3000F82D0020F42D0020981100205C2C00206E
:105B4000342E0020302E0020E82D0020AC22002032
:105B50009422002024250020FC220020082500207B
:105B600020250020481A00200C360020383600205E
:105B7000A4350020A42D00209023002078100020C0
:105B8000A02200206F12833A602C0020642C002099
:105B9000B8F1000F25D0924B1A7912B3914A1578BB
:105BA000FDB1187810F060FF8046284610F060FFC5
:105BB0000146404610F0B0FF8B4B0546188810F0A8
:105BC00053FF0146284611F05BF88849054611F05D
:105BD0004BF900B9854D4FF07E51284611F04EF932
:105BE00008B94FF07E55824B4FF000095B78002BCF
:105BF000804B14BF01204FF0FF3093F800B010F03D
:105C000037FF394610F088FF00237B4F0F900A932F
:105C10000993D945C0F266820A99099810F072FE7C
:105C2000764D4FF07E51C5F80401064611F030F96B
:105C3000002800F0988231464FF07E5011F020F895
:105C40000024074614AEA34500F384820CF042FC06
:105C500018B14FF07C53C5F84831DFF8A0A10025FA
:105C6000DAF8483109939AF8D8310A93644BDB7813
:105C70001093644BD3F80080404611F029F9814617
:105C8000614B1E6806F010031193604B06F48056BA
:105C90001C785F4B04F00104B3F906705D4B5A8B1E
:105CA00012930AF5AC730F9213935D45C0F0808296
:105CB00024B9594B594AA34500F3C2824F4BD3F83C
:105CC000DC21002A00F08E8493F81C31192B09D8AE
:105CD00001229A40524B1340002B40F0B782100330
:105CE00000F1F883484E4F4D336813F0200F30D049
:105CF00000200AF0D7FC4C4C8046208001200AF09E
:105D0000D1FC0746608008200CF0DEFB08B33B4B5B
:105D100095F90A1093F80232012B444B40F0E583C9
:105D2000484295F91620B3F90210B3F90030414307
:105D3000534332206FF0310291FBF0F193FBF2F20A
:105D400093FBF0F00A44A8EB020222800844384496
:105D500060800023364AEC18B4F90410B2F902004E
:105D6000B4F90640884203DB84422146A8BF0146BD
:105D70000C33602B22F8021FEDD12E4DAB89002B86
:105D800040F0C3831D4F97F81C31013B182B00F2E4
:105D9000F283DFE813F0E203F003F0035404F003AE
:105DA000F003F0034104F003F003F003F003F00309
:105DB0006004F003F003F003F0038404540471045E
:105DC000F003F0036004E2030123FFF7D0BB0023DC
:105DD0000B93FFF7D5BB4146484610F093FD1BE4FB
:105DE000FE350020441A0020321A0020713DAA3FDF
:105DF0002C25002004230020D01100207810002042
:105E000010360020C82600200C360020A4350020C3
:105E1000CC350020383600200823002058250020EB
:105E200032413003F82B0020542300208C31002015
:105E3000522300207A2C0020D4F8A890D4F8AC800B
:105E40004946404611F006F800287DD049464FF0FB
:105E50007E5010F057FD974B8146B3F90000B3F91F
:105E6000023080EAE07183EAE372A1EBE071A2EB19
:105E7000E37291426ADD0028D8BF404210F0F8FD7D
:105E80008D4910F049FE8D4B80461B78002B62D067
:105E90008B4B2946D3F800B0584610F0F9FF002884
:105EA00000F09780874B2946D3F800A0504610F0A9
:105EB000EFFF002800F08D804FF07E51484610F033
:105EC00021FD814910F028FE594610F0D9FE4FF00F
:105ED0007E5110F019FD41468146504610F012FDEA
:105EE000514610F0CDFE4FF07E51804610F0BCFFC1
:105EF00008B94FF07E582946404610F0BFFF00B960
:105F0000A8464946404610F007FE81466F4B0E9862
:105F1000196810F001FE4FF07E518046484610F09F
:105F2000A3FF08B94FF07E592946484610F0A6FF56
:105F300000B9A9464946404610F0EEFD01463846F4
:105F400010F0E2FCFFF7AEBB414680E7002BCCBF70
:105F50001846584292E75E4B5E49D3F800A050467F
:105F600010F078FF002830D051464FF07E5010F0EE
:105F7000C9FC594910F0D0FD41468346574810F0FE
:105F8000C1FC0146584610F0C7FD514610F0BCFC5C
:105F90004B4B196810F0C0FD80462946404610F072
:105FA00063FFB0B94FF07E51484610F0ABFC41465C
:105FB0008146454810F064FE0146484610F0ACFDAD
:105FC0004FF07E5110F0A0FC9FE73D4BD3F80080CE
:105FD000E3E7A9469AE74FF001034FF07E51D4F86A
:105FE00004010E9310F04AFF03E429467AE4072BDC
:105FF00003D10BF095FB0690E5E400230693E2E461
:1060000009EB070010F034FD0146304610F036FF72
:1060100000B3D4F8BC303046C4F83431D4F844313D
:10602000C4F83C3110F07AFFA4F83001484610F073
:106030001FFD0146304610F065FC0546384610F05D
:1060400017FD0146284610F05DFCC4F84801D4F85D
:106050004C11E8E4B4F830319B450ADBD4F8383110
:10606000C4F848A1C4F834311D4B1B68C4F83C3156
:10607000D7E4D4F8BC30C4F84851C4F83431D4F86B
:106080004431C4F83C31E2E7588B10F0F1FC014692
:10609000F06810F037FC124BC4F848011B68D4F8C4
:1060A0005011C4F83C31D4F8BC30C4F83431BAE4EF
:1060B000B246F9E48C310020CDCCCC3D082E002036
:1060C000042E00200C2E00200000C842002E0020CC
:1060D000102E0020AE47813F610BB63B00003443D9
:1060E000902300207968504610F016FDB96880466C
:1060F000304610F011FD0146404610F005FCF968ED
:1061000080460F9810F008FD0146404610F0FCFB59
:106110004FF07E518046284610F0BAFE20B140462E
:10612000294610F0F9FC80464146099810F092FE8D
:1061300068B941460A9810F097FE08B9CDF8288052
:1061400014AB43F82980103709F1010961E5CDF856
:106150002480F5E756F82400394610F0DDFC46F8B7
:10616000240001346FE50CF0B5F938B94FF07C51DB
:10617000204610F08DFE00283FF46FAD4FF07C51AB
:10618000304610F0C9FC05460146204610F062FE7C
:1061900050B929464FF07E5010F0B4FB2146054619
:1061A00010F062FE00B92546BB4BC3F8485154E5D8
:1061B000139A2B019958099810F0AEFC14AB53F8C0
:1061C000251010F0A1FB0B9910F0A6FC089910F017
:1061D0009BFB0A9B82463BB10899079810F094FB01
:1061E000514610F08FFB8246109B5046FBB110F0D9
:1061F0006FFE4845824606DB079810F069FE504561
:10620000A8BF504600E0484610F032FC119B824681
:1062100043B13CB136B90CF05DF918B90F9B9F4200
:10622000B8BFC2469D4B43F825A001353DE510F0AF
:106230004FFE8246089810F04BFE8245E4DBDBE718
:1062400052F8241043F82410013434E5944B1B8891
:10625000D90540F18C80934C206810F039FEADF8E0
:106260005000606810F034FEADF85200A06810F0E5
:106270002FFEADF854004FF47A724FF461618A48F2
:10628000B0F9023003F5E163534393FBF1F3A3F557
:10629000FA73ADF86830B0F9003003F5E1635A43A2
:1062A00092FBF1F27D4BA2F5FA7280491868ADF8C5
:1062B0006A2010F027FB10F00BFE7D4A129B11881C
:1062C0001B8BADF85600C91AADF858105188C91A81
:1062D000ADF85A109188C91AADF85C10D188C91A66
:1062E000ADF85E101189C91AADF860105189C91A4C
:1062F000ADF862109189D289C91AD31AADF8663007
:106300000023ADF8641019466A4A22F813100133CD
:10631000082BFAD14FF00C096427674B674C1B78A8
:10632000674DC3EBC3032344DFF8A481DFF884A1E6
:106330000993099BA3423DD100254FF00C09642726
:10634000604EDFF88C8109FB0583B6F9024093F9B2
:106350000A00444394FBF7F4E8B274800AF0A2F90F
:1063600001352044082D26F8020FECD1BAE4564935
:106370000C9810F0D1FB10F0ABFD5349ADF8500074
:106380000D9810F0C9FB10F0A3FD4F49ADF8520075
:106390000E9810F0C1FB10F09BFD00B2ADF8540058
:1063A000002E3FF468AF494B1B8B9F42BFF663AF93
:1063B00040425EE7A07928B11630C0B20CF084F8F4
:1063C000002867D094F800E094F9051009FB0E83CB
:1063D000DA889B8894F801C0D21A94F9043092B2FA
:1063E000534393FBF7F34FEA520BA3EB0B030891D4
:1063F000E1781BB207934FEA4C0681BB1CA90E44FF
:1064000036F8201C2980012309FB0EF158F80110F1
:1064100003FA0CFC1CEA010FB5F9006094F90210B4
:1064200008BF184601FB06F191FBF7F1079B18BF67
:106430004FF0FF30994209DB089B5A4392FBF7F279
:10644000A2EB0B031BB28B42A8BF0B463AF81E20EF
:1064500000FB03232AF81E300235073469E71CAB22
:106460001E44B5F9000036F9206CB04208DA014448
:10647000884203DC8E423046A8BF08462880C2E727
:10648000C1DD411AB14203DB8842A8BF0846064677
:106490002E80B8E72880DFE778100020082300204E
:1064A000F6350020481A00208C3100200080BB44C3
:1064B000CC35002054230020152B0020162B002063
:1064C0005A120020522300203333333F3836002045
:1064D000F82B00208F4A904830F8131022F8131040
:1064E0000133082BF8D1FFF7FDBBB3F90220B3F954
:1064F00000004A43322192FBF1F24244228095F996
:106500001620504390FBF1F021E4DFF808820024CC
:10651000C346824FDFF81C9238F9140010F0A8FA35
:1065200001462C2000FB049006F0EEFB11F0E4FA8B
:10653000B7F9043000B298424FEA440AB7F906208E
:1065400003DB82421346A8BF03460134082C2BF814
:106550000A3007F10C07DFD114E4AB7B002B54D0D9
:106560006C4BB3F90A0010F083FA0146002005F0E5
:10657000B1FE0123059333689A0603D497F81C31C2
:10658000052B16D1634CB4F9000010F071FA0146E6
:10659000059805F0AFFEB4F9020010F069FA059B0A
:1065A00001460133D8B205F0A5FE059B0233DBB2EC
:1065B00005933368DB0215D50024EE7B564FE5B218
:1065C0007319DBB2112B0DD8331937F9130010F002
:1065D0004FFA059B01461D44E8B2013405F08AFEDE
:1065E0000E2CECD14E4C94F8E021002A67D14D4B93
:1065F0001B78072B05D10BF093F8069BC01A4A4B6A
:10660000D88001232370FEF73BBA484B187810F06E
:106610000100A5D10021AAE73E4CB4F9060010F014
:1066200027FA0146002005F055FEB4F9080010F0E5
:106630001FFA0146012005F04DFE02239AE7354C72
:10664000B4F9080010F014FA0146002005F042FEEB
:10665000B4F90A00EBE70224DFF8B88038F9140037
:1066600010F006FAA31E01460134D8B205F042FE2E
:10667000082CF3D106237DE7264C049B34F9130044
:1066800010F0F6F9049B0146033BD8B205F032FE48
:10669000049B0133072B0493EFD104236AE7002402
:1066A000DFF8708038F9140010F0E2F90146E0B22A
:1066B000013405F01FFE082CF4D105945BE70CF0C3
:1066C00079F994E711F078F800283EF43FA94FF4E7
:1066D0008052174B1A800A23FEF71DB9B9F1020F39
:1066E0004FF4FA707DF4C4AC8345A8BF0020049B2E
:1066F000B8BFA0EB0B00584310F0BAF9B045B86032
:10670000BDF6C4AC57F8292002F1004247F8292011
:10671000FDF7B7BC54230020CC350020F82B002017
:106720007810002024250020FC220020A435002021
:10673000642300207C1200202DE9F04FA94B00F5C6
:106740009C4808F12008C3F80080A74B87B01C784C
:106750000746002C6AD0A54A1268904201D9013C34
:106760001C70A34C2368D90405D500200BF0ACFEA7
:1067700008B905F047FB9F4A537D9346002B00F074
:1067800080819D4A013B32F913009BF817301BB101
:10679000C0F53B60083000B2A0F57A70B0F57A7FA2
:1067A000A8BF4FF47A7020EAE07010F061F99349C5
:1067B00010F0B2F910F0B2FB914B18802368DFF8AB
:1067C0007CA213F4807F00F0D7818E4BDFF85092CB
:1067D0009F4205D999F8022012B9012289F80220B6
:1067E00099F80220002A00F0C7819AF8005099F821
:1067F000217005F001031B2000930BF065FE012FB3
:1068000008BF0025804EDFF83882019018BF05F0E0
:10681000020599F82020052A00F2AA81DFE812F08B
:106820006F01CF01DA01FA010702220209F09CFE92
:106830000646764DDFF8BC91DFF8F0A1A64246DCB3
:1068400042F201024FF47A71694BB7FBF1F91B6810
:10685000134001936E4B06D06E4A12781A706E4A3E
:1068600011786E4A11701B78009323B16B4B1E7820
:1068700086F0010300930F230024DFF8C8B1DFF88E
:1068800078A185F8243009F06FFE844249DB95F841
:106890002430634C0F2B0CBF01220022614B5A4D58
:1068A0001A7040F0D1801B200BF00EFE002840F043
:1068B000CB802B68E268A3609B1AC82B02D9012306
:1068C00084F82130584A13780133137049E7072CB4
:1068D000E1B25648D8BF14F80910DAF804309847E6
:1068E000032C1ADCC8B1524B33F8242003EB84018B
:1068F000831A4FF47A7058434B889B1A90FBF3F03D
:1069000040F2EE2300F57A709842B8BF184640F680
:10691000CA039842A8BF184680B225F81400013473
:106920008CE7009A6300D2B135F91400314A80B285
:10693000D18C81424FEA840103D8B2F828E0864521
:1069400020D23C4A515889450BD23AF80300019AAB
:10695000EAB92AF8030001340BF1060B93E700981B
:10696000E4E7E0B2029309F017FE032C029BEEDC91
:10697000012101FA04FE95F8241021EA0E0185F8A0
:106980002410E4E72B4E09F596727250DFE7264992
:1069900003EB040E91F800C00321BCFBF1F101EB05
:1069A0004101ACEB0101C9B2714405EB4101C8845E
:1069B00095F86E1029B9BCF1020FCAD9012185F8EA
:1069C0006E10BBF80010BBF802000844BBF80410BE
:1069D0000844194900B2C852032190FBF1F080B27B
:1069E000B7E700BFE4290020142B0020102B002063
:1069F0000C36002038360020CC350020AAF1823F2A
:106A0000F4350020404B4C00901B00202414002043
:106A1000A5350020B42900202004002021040020F6
:106A200010360020EE260020380F0020D829002044
:106A30006C2D00203C0F002094140020A435002071
:106A4000B83100204A1400200123914A1370914A62
:106A500013702B68A268E3609B1A62688E4D9342A4
:106A600084BF002384F82130002409F07DFD844296
:106A7000BFF628AFE0B209F08FFD25F8140001340D
:106A8000F3E7226812047FF599AE844AD2F88810A1
:106A9000791A0029FFF692AE8149C2F88880487CB5
:106AA000804931F810009BF8161080B290FBF1F08D
:106AB00092F88C10013101F00F0182F88C10114412
:106AC00081F88D0018468D32815C01300B4410280E
:106AD0001BB2F9D193FBF0F31BB2002B0ADB642B42
:106AE000A8BF64239BF8172032B918B20FF0C0FF7B
:106AF0006D495DE60023F5E7C3F16403F5E7009B0C
:106B00006BB30BF0F5FC012807D164203168B8F8AD
:106B1000062000FB0212C9F81020019B63B198F80F
:106B200004204AB10CF062FB032289F820204FF4C4
:106B30007A72C9F81C206CE6012F19D03268D9F896
:106B40001010914207D20CF051FB032289F820204B
:106B500040F6B832EDE7012289F8202059E6019B82
:106B60004FF4806043B30FF0FDF90022C9F8102004
:106B700015B128460FF0AAF90BF0BAFC06460BF047
:106B8000A9FC4A4D002800F099809AF80030DF07F0
:106B900040F19480BBF824000FF06AFF444B01469B
:106BA000D86810F06BF9002800F01E8101223B4BE1
:106BB00083F89D20012394E00FF0C4F9D5E7012F5D
:106BC00001D10522C8E798F80820012ABBD00CF0B3
:106BD0000DFB1EE6012F08BF0522009B08BF89F8A8
:106BE00020204BB10325BBF918102B4A118051808E
:106BF0009180B8F80210D1803268D9F8141091420F
:106C000002D3009B002B3FD147F23052C9F81C2021
:106C10000322A1E702200FF0B3F905F0F3F8316881
:106C2000D9F81C200A44C9F81820042294E7012F3F
:106C300011D13268D9F81810914299D21D4B1878A9
:106C400018B90BF041FC002892D11B490A8822F0A8
:106C500002020A80B5E73168D9F81C200A44C9F855
:106C6000182085E764203168B8F8062000FB02127E
:106C7000C9F8102000224FF4806089F8202089F89C
:106C800003200FF05FF9C4E5012F3FF4C2AD6FE7B9
:106C90002004002021040020CC35002024140020F2
:106CA000A00C0020B40C002014AE2341A011002041
:106CB000481A002000000020343600200022704BCB
:106CC00083F89D20002E7FF475AF00226D4B1A6073
:106CD0005A609A606C4B1B6893F83030002B7FF43D
:106CE00069AF2B709AF80030DD0723D52368D806EA
:106CF00020D5664A1278D1061CD4DA041AD40BF0D7
:106D0000E9FBB8B9624B5E4D1B78002B00F0878021
:106D1000604B9B78002E71D1002B00F082805E4B7F
:106D20001A685E4B1B689B1A002B7ADA05F06AF82A
:106D300085F89E6000221346BBF81A50BBF81C7001
:106D4000574931F912009B08A842C4BF63F07F0382
:106D5000DBB20132B842B8BF43F04003042AF0D19D
:106D6000474D95F89F209A4262D195F8A020F92AC4
:106D700002D8013285F8A020454F85F89F3097F85A
:106D80000080B8F1000F08D140460BF09DFB0028B1
:106D900050D085F8A18005F0C5F895F8A030142BE7
:106DA00040F09D803B7853B195F89F305F2B06D122
:106DB0009AF8003013F001065BD005F023F89AF83A
:106DC000003013F0010240F08A8095F89F30572B75
:106DD00074D1344807F022FF334B1B6858077ED527
:106DE0000A22324B1A807AE0002E7FF4E3AE244B65
:106DF00093F89D30002B7FF4DDAE66E73BB14FF496
:106E00007A71254A126801FB0323244A136095F81E
:106E10009E30002B8ED00FF03DF8002305E0002EB1
:106E2000F5D110200FF052F8012385F89E3081E74C
:106E300000229FE71E4B18609AF80030DB07ACD5A4
:106E40001C4B1B78002BA8D01B4BDB78002BA4D14C
:106E500095F8A1300133DBB2032B85F8A1309CD922
:106E60000C4B5B7813B104F0CDFF96E7002E94D164
:106E7000F9E70B200FF02AF885F8A0609FE700BF24
:106E800024140020A022002020250020ED26002030
:106E90000000002070110020901B0020B41C002076
:106EA000CC350020743C002028250020A81C0020A0
:106EB000B81C0020A53500201036002021684907A5
:106EC00040F1F2805A2B40F0EF8095F8A230002B71
:106ED00000F0DD80012385F8A22085F8A330236827
:106EE0005E0728D595F8A4309BB19AF80030D807F2
:106EF0000FD5994BB3F90620BBF81A309A4208DD3A
:106F000000200BF0E1FA20B9322385F8A400A5F89F
:106F1000A63011200BF0D8FA002800F00C8195F86B
:106F2000A8302BB995F8A23013B93223A5F8A630B2
:106F3000012385F8A8300023884E04AF049306F19E
:106F400050087B60314616F8010C0BF097FA30B10F
:106F500016F8021C232902D8384603F0F6FC043642
:106F6000B045EFD17E4B97E8030083E803007D4BEB
:106F70001F78002F00F0108101200BF0A5FA7A4F46
:106F80007A4E40B92368DA0540F10983784BDB7803
:106F9000002B00F004833B689B0740F10083358899
:106FA00015F0010540F0008301200EF0DBFF022008
:106FB0000BF08AFA002800F0F982002D00F0F6822A
:106FC00001200EF0BFFF33889D0702D402200EF08F
:106FD000C9FF3188012011F0030118BF01210AF017
:106FE00059FD3B6813F00A0F17D006200BF06CFA1E
:106FF000002800F0DF823388580602D440200EF0CB
:10700000B1FF07200BF060FA38B10A22594BB3F9EF
:10701000043093FBF2F3584A13800C200BF054FA1F
:10702000002800F0CB824FF480700EF09BFF534B92
:107030001B78082B01D00E2B02D140200EF082FFCE
:10704000236859050FD54E4B1B79002B40F0BB82AE
:107050009AF80030DA0740F1BC823C200EF0B8FB11
:10706000002840F0BB820122464B1A7004F0E4FE77
:107070003B685B0708D503200BF026FA002840F098
:10708000B38208200EF05EFF07B0BDE8F08F95F8E0
:10709000A43083F0010385F8A4301BB10C200EF05E
:1070A00015FF1CE70D20FAE75D2B00F0B2825B2B89
:1070B00000F0B5825E2B40F0B4820320AAE20022E9
:1070C000314B1A6095F89F30972B03D14FF4C8725B
:1070D0002E4B87E6A72B05D12D4A137843F00403E6
:1070E0001370FCE60022BB2B049213D10223ADF8EF
:1070F0001230284BBDF810105A890A445A81BDF845
:1071000012109A890A449A8108F026FA002385F819
:10711000A030E4E6B72B02D14FF6FE73E7E7BE2BB3
:1071200003D10223ADF81030E3E7BD2B7FF4D7AED7
:107130004FF6FE73F6E795F8A230002B3FF4FBAE56
:107140009AF8003013F0010302BF85F8A230012342
:1071500085F8A330EFE600BFCC3500207E18002074
:10716000F4240020C426002028250020F635002025
:10717000103600208C310020861000202C250020A5
:10718000361A0020C0100020B81C0020AA1C0020C5
:10719000ED260020F02600204FF00C09BB4E06F132
:1071A0005A08314616F8010C0BF068F9E8B131794C
:1071B000B37809FB0150B64A013B03EB4303134488
:1071C000D0F8B02096F803E093420ED0C0F8B0306B
:1071D000012303FA01F195F8DC3080F8ACE023EAF2
:1071E0000101C0F8B47085F8DC1006364645D8D1E8
:1071F000A84BDFF8B0821E68A74BA8F1AC051B684E
:107200000193A64B1B78029300230093D8F8043017
:10721000002B6BD01F78002F68D0D8F80820019978
:107220008A1A002A0DDB01F5FA720121C8F808203C
:10723000009A01FA02F295F8DC1021EA020285F8C0
:10724000DC20029A002A51D098F8002059780432A4
:10725000D2B2002940F05081914931F91210BBF8A7
:10726000182002F1C80081422ADD93F8029095F8B7
:10727000DC20009B1A41D10738D4B9F1000FCCBFF4
:107280000220012001F0BEFC7A1E162A41D8DFE858
:1072900012F035004E00580068007F008600A10003
:1072A000BC00D800E400F0004000680075008600D3
:1072B000A100BC009500B000CC000B011701250116
:1072C000C83A914203DA9978C1F10009CFE7012267
:1072D000009B02FA03F395F8DC2022EA030385F809
:1072E000DC30019B03F5FA73C8F80830009B08F105
:1072F0000C080133042B009388D13DE6317801203E
:107300004944FA29A8BFFA2121EAE17131700BF052
:1073100017F9D5F8E0000BF0A5F90122009B02FA5D
:1073200003F395F8DC20134385F8DC30DEE7B17811
:10733000022049446429A8BF642121EAE171B170A7
:10734000E5E731798944B9F1640FA8BF4FF06409CA
:1073500029EAE97986F804900BF006F949460320FA
:10736000D5E7B1790D2049446429A8BF642121EAF9
:10737000E171B1710BF0E4F80D2FCAD071790E20D4
:1073800049446429A8BF642121EAE1717171BEE713
:10739000F1790520494481F30801F171B7E7D5F887
:1073A000E0200F20D1784944C829A8BFC82121EA8C
:1073B000E171D1700BF0C4F80F2FAAD0D5F8E020FE
:1073C000122011784944C829A8BFC82121EAE171D7
:1073D00011709CE7D5F8E020102011794944C829A4
:1073E000A8BFC82121EAE17111710BF0A9F8102F93
:1073F0008FD0D5F8E020132051784944C829A8BF80
:10740000C82121EAE171517081E7D5F8E02011200F
:1074100051794944C829A8BFC82121EAE1715171B5
:107420000BF08EF8112F3FF474AFD5F8E020142044
:1074300091784944C829A8BFC82121EAE171917017
:1074400065E7D5F8E020092091794944C829A8BF0B
:10745000C82121EAE171917159E7D5F8E0200A20AD
:10746000D1794944C829A8BFC82121EAE171D17165
:107470004DE7D5F8E0200B20117A4944C829A8BF70
:10748000C82121EAE171117241E700BF1D190020F6
:1074900039A50108AC2D0020901B0020A535002047
:1074A000CC350020D0140020717815204944B1F566
:1074B000967FA8BF4FF4967121EAE171717026E7BB
:1074C000D5F8E020162092F83B104944FE29A8BFC9
:1074D000FE2121EAE17182F83B1018E7D5F8E0209F
:1074E000172092F83A1049446429A8BF642121EA80
:1074F000E17182F83A100AE701297FF40EAF514991
:1075000031F9121040F633029142A8BF11469A7821
:107510004FF49663B1F5617FB8BF4FF4617193FB8F
:10752000F2F3A1F561710C2F91FBF3F11ED0182F2E
:107530007FF4F3AEC9B2C8290B46A8BFC823D5F85B
:10754000E020D8B292F817E070453FF4E6AEA3EB26
:107550000E034FF0080E93FBFEF30133DBB2D07540
:10756000384603930AF0ECFF039B11E0364ACBB296
:1075700052789A423FF4D1AE184603930EF076FC4F
:10758000039B384619460AF0DBFF039B0133DBB24D
:10759000002B3FF4C2AE184601F034FBBDE60120DB
:1075A0000EF0D0FC012502E5002500E502200EF0DA
:1075B000C9FC0EE540200EF0C5FC22E54FF48070BA
:1075C0000EF0C0FC33E514200AF07EFF00287FF4A3
:1075D00044AD04F071F801F0C3FA44E501F0D0F8CD
:1075E0003C200EF0C1F83BE5348814F008047FF429
:1075F0004BAD08200EF0B6FC144B1A68144B1A6001
:10760000104BDA88134B1A80134B1C60134B1C6011
:107610003AE501200138C0B207F094FC5FE4022093
:10762000F8E7562B01D107F097FF3B78002B3FF48A
:1076300049AD95F89F306F2B7FF441AD04F072FC9B
:107640004DE400BFCC35002008160020A01000201B
:107650009C10002090100020941000208C1000201E
:107660002DE9F04F85B0804604F026F8C74B1B7813
:10767000002B40F06C83C64E3368009613F4806F85
:1076800000F06583C34BC44D1B78002B00F049818B
:10769000C24C2A68E368D31A7C2B40F2428124272B
:1076A000237CDFF830B30133DFF82C93E2602374DE
:1076B000ABF1300A384603F0EFFF5BF8040F0FF030
:1076C000D7F90190BAF810000FF0D2F9019B0146EA
:1076D00018460FF0D5FA49460FF01EFA0FF0F8FBE6
:1076E000013700B2FFB203F0C5FF272FE2D13020EF
:1076F00003F0D2FFB4F9140003F0BCFF03F0C4FFA1
:10770000237C980733D141F28833E2689A421BD92F
:107710006427DFF8C892102003F0BEFFD9F80000FC
:1077200090FBF7F000B203F0A5FF212003F0B4FFB7
:10773000D9F8003093FBF7F007FB10300028D8BFD2
:10774000404200B203F096FF142003F0A5FF944BD3
:10775000B3F904000A2390FBF3F003F08BFF1C2025
:1077600003F09AFF002003F085FF03F08DFF237CD8
:10777000590740F0B080022003F08EFF894BDFF8FC
:107780006092D8696423323090FBF3F000B203F0CA
:1077900071FF032003F080FF834B1B7813F0010F70
:1077A00000F073810AF0A4FE804B81490746D86837
:1077B0000FF0B2F90FF0B2FB80B22FB9009B1B683B
:1077C00013F0100F18BF002000B203F053FF99F818
:1077D0000430002B4DD0DFF80CA29AF800B0BBF1BA
:1077E000000F46D06427734B06201A88019307FBCD
:1077F00002B24FEA4B07B2FBF7F2278B3F01BFB251
:1078000047EA0227BFB2C2F30322174303F044FF43
:1078100038B203F02FFF228B019B013292B292FB10
:10782000FBF10BFB112B644A1F88537AA4F818B0A4
:10783000012B40F03081392003F02EFF38B203F0E5
:1078400019FF282003F028FF0A235C4F386890FBBB
:10785000F3F000B203F00EFF042003F01DFFB9F8AF
:107860000630002B00F03B8100F022FE00B203F056
:1078700001FF02A9524803F0D3FE132003F00CFFCE
:10788000BDF9080003F0F6FE1B2003F005FFBDF96B
:107890000A0003F0EFFE232003F0FEFE4E2003F06B
:1078A000E9FE02A9464803F0BBFE122003F0F4FEF5
:1078B000BDF9080003F0DEFE1A2003F0EDFEBDF96D
:1078C0000A0003F0D7FE222003F0E6FE452003F075
:1078D000D1FE03F0D9FE237C282B22D100231720D0
:1078E00023742C6803F0D8FE4EF660203C27B4FBCE
:1078F000F0F3B3FBF7F007FB1030000200B203F027
:10790000B9FE182003F0C8FE4FF47A70B4FBF0F40F
:10791000B4FBF7F007FB104000B203F0ABFE03F03E
:10792000B3FE284B1B78002B00F099801B4C264A95
:10793000E369A8EB030393427DD90022234B9A709D
:107940001A711C4A1288D1B2120A9977DA7719751E
:107950005A752968226A891A174AD07A4FF47A72BE
:10796000424391420AD32A682262194A1278013AA4
:10797000012A9FBF10229A7002221A710A200F4A10
:10798000C4F81C80116892682EE000BFC426002055
:107990000C360020781B0020901B002008150020CA
:1079A0008C31002034230020A4350020481A002008
:1079B000CDCC4C3E321A0020361A0020282300205D
:1079C00080969800821B00203F0D03008C0F002042
:1079D000F9350020E822002000007A44A0100020A1
:1079E000FE350020441A002091FBF0F192FBF0F2EA
:1079F000642083F82020121283F82120BA4A1977D4
:107A00001268091292FBF0F202F5FA7292B29A76BB
:107A1000120ADA766269597702F1300183F822108E
:107A200002F5EA4192FBF0F230310912783283F824
:107A3000231083F8242094F824A0BAF1000F00F05A
:107A4000A283E36A5BB194F82430002B71D040F636
:107A5000B732636BA8EB0303934200F29880A34B09
:107A6000D5F800801B78002B00F06C81A04F3B689C
:107A7000002B00F067819F4B1B78013B012B00F22C
:107A80006181DFF884929C4CB7E00523B9F80600C9
:107A9000B0FBF3F098E66E2315217B43527B93FBFA
:107AA000F1F322B19AF800209BB293FBF2F34FF06E
:107AB000640B9FB23A2003F0EFFDB7FBFBFA0FFA1D
:107AC0008AF003F0D7FD3B2003F0E6FD0BFB1A70B4
:107AD0000A2780B2053090FBF7F000B2AFE6B86835
:107AE00080F31000C2E63B7823B1C4F8288087F801
:107AF00000A0A6E7A36AA8EB0303B3F57A6FA0D3AF
:107B00000123D9F800003B7009F0C3FE0746D9F8FD
:107B1000000009F0BEFE7A0693D18E2891D194F828
:107B20002430002B8DD1754BE3622D2384F8303047
:107B300087E7012284F83830714B84F824201B68D1
:107B40009B781E3B93426F4B1CD91868022104306E
:107B500003F01CFD94F830206A4F013AD2B284F849
:107B6000302094F8381094F83930D2B94A1C0133D7
:107B700084F8382084F83930386809F090FEC4F869
:107B800034806CE70221186809F07DFEE2E794F882
:107B90003030002BDED1E36284F8243003F026FD80
:107BA000D8E7E06A013310F801EB84F839300EEBC6
:107BB000010284F83820E0627146DDE7386809F098
:107BC00068FE83B27E2B2A6807D1002384F83A30FE
:107BD00084F83B3089F801300FE099F8012062B950
:107BE00094F83A1061BB1B2B22D1386809F054FE7F
:107BF000002844D1012384F83B30386809F04CFE5A
:107C000001460028DAD13C4C94F83F30002B00F0BC
:107C10008B80637884F83F00302B40F08580A37818
:107C20005F09012F37D084F8400003F069FC7BE046
:107C30000D2B24D10122237084F83A20A187DCE7A0
:107C40007D2B03D1012384F83E30D6E794F83EE043
:107C5000BEF1000F04D080F02000C3B284F83E20B3
:107C60004A1CD2B2092A84F83A20635409D1A28F5F
:107C7000C2F1FF02934202D1012384F83F30012375
:107C8000A8E7082AB9D8A08F034403EB132303F015
:107C9000FF03A387B1E703F00F0013F0100337D001
:107CA00094F803E0237904F15402A4F84C306264A0
:107CB00083EA0E03724484F89430A4F84E10A26450
:107CC00084F84070631D002194F89420DFF83CE0B4
:107CD000676CA66CBE423DD1002948D173454BD19B
:107CE00084F8950020E000BFA0100020841B002035
:107CF000281A00208C1B0020081500208C0F002063
:107D0000701B00206C1B00200C00002010150020B0
:107D100094F8402042B194F89520013202F00F020D
:107D2000824227D084F84030B94FDFF8209394F88E
:107D30003B303BB12B68A3EB0803012B4AD900234E
:107D400084F83B30B34B1B78002B40F0178205B012
:107D5000BDE8F08F13F8011B07F1010C734582EAAF
:107D60000102C4F844C039704FF00101B0D384F867
:107D70009420B3E7E31CA6E71A7894F894309A426B
:107D80004FF0000284F8402003D0B4F94C100120D9
:107D90004BE7A14F636CDFF88892A048A36460644E
:107DA00009F58073394610387B60C7F800903A8136
:107DB0007A81FAF77DFB01304B4604D13A68511CB9
:107DC0003960022111703A683B607A600122904B61
:107DD0001A70A9E797F800A0BAF1000F60D08E4A98
:107DE0008F4913688B4294F8963038D1581C84F828
:107DF0009600B2F90A0003F00F0343F010030028C5
:107E0000B8BF43F020038DF8083053685B1A117A2D
:107E10008DF809304B4084F897300DF10A030025A6
:107E2000D2F804C094F897100DF10E00834228D2C6
:107E30001668ACEB060EBEF1000F1ADC0DB184F82B
:107E4000971094F897105A1C19700023824224D37B
:107E500002A9322003F068FB4FF0000A1AE0591C17
:107E600003F00F038DF8083084F896100DF1090324
:107E7000D5E7751C1560357803F8015B694001256D
:107E8000D4E70DB184F897108342DAD102A93220E9
:107E900003F04AFB87F800A051E702F8013BD5E761
:107EA00094F8983039F8130018B984F898004FF412
:107EB000036094F89830B0F5826F03F1010384F801
:107EC000983000F0E0805AD8B0F5007F00F095803F
:107ED0000ED8B0F5807F00F0BB80B0F5887F7FF4CE
:107EE00026AF504B1B685E077FF521AF61697CE0D0
:107EF000B0F5047F64D0B0F5806F7FF418AF94F8CC
:107F0000993042F210710133DBB2032B88BF012399
:107F100084F8993094F899305943434B1B88002BCF
:107F200040F0AF800131414B1B78D807404B48BF30
:107F300004311B88DA0748BF0A319E0748BF143155
:107F4000180648BF2831DA0548BF28315E0748BF08
:107F50006431180748BFC8319A0548BF01F5C87198
:107F60009E0648BF01F57A71D80648BF01F5FA614F
:107F70005A0648BF01F57A614FF4806035E0B0F5EC
:107F8000E26F7BD00ED8B0F5C06F69D0B0F5E06F6E
:107F90007FF4CDAE274A516B64234B43118A93FB88
:107FA000F1F122E0B0F5046F62D0B0F5116F00F08E
:107FB000B380B0F5E46F7FF4BAAE1E4AD16BEBE745
:107FC0001D4B1B79002B3FF4B2AE1C4B19780029D6
:107FD0003FF4ADAE1A4B1B4A5B7B63B1138893FB36
:107FE000F1F30A214FF40470594303F0B7FA002368
:107FF00084F83B309BE61388F3E70F4B5B79002B4B
:108000003FF495AE104B19680A2391FBF3F1ECE7AE
:10801000681B0020951B0020581A00205C150020CA
:10802000681A00202825002034360020A4350020BE
:10803000F6350020B8220020FE350020441A00202A
:10804000361A0020321A00202823002082A50108B9
:10805000564B1B685B077FF56AAE554B1968C4E742
:10806000544B5B79002B3FF462AE534B9968BCE7ED
:108070000A21524BB3F904305943B6E7504A916B89
:108080008AE702314FE7494B1B6813F0200A7FF45F
:108090004EAE009B1B681B0605D5514603F05EFAE9
:1080A00084F83BA043E6474B1B7B002B3FF43FAEDD
:1080B00094F89A30032B2DD8DFE803F002181F261E
:1080C000414A1268107892F803E09179090401EBB3
:1080D0000E21014401EB03610133DBB2042B08BF25
:1080E00000234FF4826084F89A307EE7364A1268A3
:1080F000507892F804E0D179E8E7334A1268907832
:1081000092F805E0117AE1E7304A1268507992F866
:1081100006E0F0E70021DDE7264B1B79002B3FF45A
:1081200006AE2B4B197800293FF401AE294B1A8873
:108130000A23534333E7306809F0ABFB264D8046F2
:108140002B783BB1013B2B70306809F0A5FB002870
:10815000F1D1FCE521460322601E11F07EFF0421CF
:10816000601E87F89E8003F048F90028ECD0601E5E
:1081700003F05EF92B7818442870E5E7174F184E86
:1081800007F19C04E0E7DFF86090D9F8000009F0FF
:1081900083FBC0B201287FF654AC0228114F3FF494
:1081A000A2AC03F013FA01233B704AE42825002017
:1081B000A0100020FE350020282300208C31002054
:1081C000B8220020361A002020250020AC2D0020E7
:1081D000441A0020321A0020A01B0020081500209D
:1081E0009C1B00200C0000206C1B0020024B1A88F6
:1081F0009B78028083707047A4A50108064A116825
:1082000049B1642350684343B3FBF1F303490B8046
:108210000023136053607047A81500202E1600201D
:1082200070472DE9F843304B06461B782BB92F4A8F
:10823000136053609360BDE8F8832D4B9F6898608E
:108240002C4B5B79012B09D001D3042B04D90022DC
:10825000264B1A605A609A60BDE8F88340F6E449FC
:108260004FF47A74244BDFF8A480DA79234B244D41
:1082700033F81200B8F9023080B209FB00F2C3EB08
:1082800012336343B8F9002093FBF2F3EB600EF076
:10829000EBFB01461B4804F037FD0EF03FFE80B2B9
:1082A00009FB00F9B8F90200B8F90030C0EB193940
:1082B00004FB09F494FBF3F4D5F80C80F01BAC60DC
:1082C00008FB00F00EF0D4FB0F490EF025FC6968A6
:1082D0000EF01AFB68600EF0FBFD044B286083E88B
:1082E00010019860BDE8F883441A0020282300207C
:1082F000A8150020FE350020A00C0020B40C0020A2
:10830000FC0F00200C1000202FE33E313C11002018
:108310002DE9F843224B234D1B79012B3BD1224BF6
:10832000224E9A78224B33F81240A4B220460EF027
:108330009BFB0146304604F0E7FC1E4B9F7893F808
:10834000009093F801800EF0E9FD44F6FB7209EB12
:10835000491983B209FB032309FB0424C8EB08383D
:10836000B3FBF8F3B4FBF8F4B3FBF7F3B4FBF7F4A7
:108370009BB2A4B226F8043C26F8024C2B806C80F9
:108380000D4B1B78022B04D10C4B6A881A802A886B
:108390005A80BDE8F88300232B806B80F0E700BF94
:1083A000FE350020321A0020A00C0020CC0F002047
:1083B000B40C00203811002024250020FC220020CD
:1083C000F8B524220021044611F061FE0022234664
:1083D0000521042510460A4FD65D0132042A9E70FD
:1083E000D9701D719871597103F10803F4D10123FB
:1083F0002380522384F8223064232384F8BD00BFF5
:1084000058A20108F7B5264E3368002B44D0254BFF
:108410001B78022B40D10024234D244F04F120006F
:10842000C0B20AF051F8C8B32B7883BBE25D72B3D7
:10843000306850B355218DF8001001218DF80220CD
:10844000AA228DF8011019468DF804308DF803200A
:108450001DF801205340082213F0800F02F1FF3273
:108460004FEA430318BF83F0310312F0FF02DBB27F
:10847000F2D101310429EBD18DF80330AA23052272
:1084800069468DF8043009F00DFA01232B70013490
:10849000032C05F10105C1D103B0F0BD2870F6E74A
:1084A000401000204710002044100020A7A501081C
:1084B00038B5194B187808B31849CC88FCB1204658
:1084C0000EF0D2FA164B054698680EF0D1FA014626
:1084D00028460EF017FA13490EF01EFB05462046FB
:1084E0000EF0C6FA014628460EF0CAFB0EF0F0FC6C
:1084F0006428A8BF642020EAE070C0B238BD0A4BEF
:108500004D781B880A7800FB15346423521B6343A3
:108510005043B3FBF0F0EBE7441A0020FE35002097
:10852000282300200000C842321A0020194B2DE9F0
:10853000F0411C6807460F2C984607DC0023164ABA
:108540009C4206DC0025144EA54208DD0020BDE853
:10855000F08152F823108F42F8D00133F0E756F83B
:108560002530681C7BB98000621B011F92003144DA
:108570003044013411F071FD46F82570C8F8004010
:108580000120BDE8F0811A7D3B7D9A42EBD3054680
:10859000DAE700BFC0150020C41500201128F8B587
:1085A0000FD00F280CD83422124B02FB003009B137
:1085B000C3684BB90022104D10492C68A24206DB5B
:1085C000F8BD0F4B1868F2E7BDE8F840AEE751F888
:1085D00022709300B84203EB010609D1A21A0433BA
:1085E000920019443046013C11F037FD2C60F8BD73
:1085F0000132E3E7DC000020C0150020C415002094
:10860000B41B002008B50C4B197801290CD00AD3F3
:1086100002290DD009F084F8084B00F5F42000F58C
:108620009070186008BD0021002009F033FAF1E7CE
:10863000002009F056F9EDE7AC1C0020B01C00202A
:10864000F8B506460D2009F03FFF10B10A200DF0E5
:108650003DFC294CE268002A4DD02369B3424AD838
:10866000264BA18A1878576838BB012018707B5CAC
:10867000002B34D01378224A013B126800FA03F32E
:10868000134201D109F0DAF901221E4B1A70FFF7EB
:10869000B9FFA38A43B9E3681B78053B012B03D8D4
:1086A00009F03EF8184B1860E368A28A5B689B5C8F
:1086B000FE2B0ED10023A382F8BD00251D707B5C2C
:1086C0006BB1284609F0BAF90E4B1D70FFF79AFFFF
:1086D000EAE7FF2B07D1BDE8F8400DF0DBBBE3680C
:1086E000A28A5B689B5C42F2107101FB036301325A
:1086F0002361A282F8BDF8BDA8150020AD35002089
:1087000074180020AC1C0020E824002010B504469A
:10871000204609F0BBF800B110BD0A2009F053F85B
:10872000F6E70023F0B51C46FF260949094D0A78F3
:108730005F57874204BF5E5502F1FF3203F10C031D
:1087400004BFD2B20124302BF2D104B10A70F0BDC3
:108750004C0B00205841002000230C2130B5074C61
:1087600001FB03425568A84203D00133042BF7D123
:1087700030BD0023C3621381536030BD58410020D7
:10878000F8B505460024094EA359A719AB4207D1F5
:108790002846FFF7E1FFCC220021384611F077FC94
:1087A000CC34B4F5197FEFD1F8BD00BFD40C002054
:1087B0002DE9F04F07464FF000090C2093B00293CB
:1087C0009DF870809DF874A02A4B0591039200FBE0
:1087D00009F2D118D256BA424ED009F10109B9F1C5
:1087E000040FF4D100207FE11F2FFBD1CDF800A0B2
:1087F0004346029A0399012039E00135072D67D1DC
:1088000000256CE00132072A40F08280002287E0D8
:10881000049B53B1711CC9B220B14FF00B0EC17152
:1088200080F806E01A2109F091F818F0010F00F025
:10883000BD800136F6B215B10C21EE71A9714A2145
:108840002846B1E04FF6DF72236D1A80DA6842F0F5
:108850002002DA6006E1226DD36843F08003D36022
:108860002FE143462846029A0399CDF800A003F071
:10887000D3FB2DE1584100200D89002DB2D11E2FD0
:10888000EFD0B1DC012FADD8994BFEB253F82740A1
:10889000002C00F01C81974BD4F854B02360029B4D
:1088A000DBF80420A36004F15A03636104F5AD739F
:1088B000A3614FF480732265E36023619BF8160087
:1088C0000CF082FCDBF80C20CAB18B491C208C46D2
:1088D00000FB051EDEF804309A428ED1EDB21C2159
:1088E00001FB05C5854B29695869014359610C2174
:1088F0002976711C69762263226D0432E264DBF80A
:108900000810002935D07C4800224FF01C0E054687
:108910000EFB020CDCF8043099427FF473AFD2B244
:108920001C2101FB0255754A2969506908435061B1
:108930000B202876701C687653699BF81900194340
:1089400051616F4A8009AA606A7B8DF81D008DF81D
:108950001C2000228DF81E2001226C6107A88DF8D2
:108960001F200CF04FFCDBF808206263226D0432FC
:10897000A26494F8580008F0C3FF054694F8590023
:1089800008F0BEFF08F002031AF0080F04933FF44A
:108990003FAF0136F6B210B10B22C67182711AF0E8
:1089A000100F14BF1A211E2108F0D0FFDBF80C2095
:1089B00012B1DBF808208AB99BF8182007A88DF8B7
:1089C0001C209BF81A309B098DF81D3000238DF870
:1089D0001E3001238DF81F300CF014FC01230026FB
:1089E00084F84430039B2662E362029BE661A66240
:1089F000666284F80580A36084F806A0204600F033
:108A0000EBFB18F0010F2DD0236B002B3FF41AAFB6
:108A100007A802F0AFFAE36C206B07934FF4805382
:108A2000109380230C93E36811960A9320230F93ED
:108A300063690B9608930D960E96099602F0C5FA97
:108A400007A9206B02F0A3FA226B216D136843F093
:108A5000010313608B8A9BB243F040038B825368FF
:108A60009BB22364049B002B2BD0636B002B3FF441
:108A7000F2AE07A802F07EFAA36C002507934FF42C
:108A80008053109380230C932369606B0A93102307
:108A9000119509930B950D950E950F9502F095FA8A
:108AA00007A9606B02F073FA636B1A6842F0020266
:108AB0001A60226D5D605D60938A9BB243F0800313
:108AC0009382226D93899BB243F400539381204695
:108AD00050B10C230B4A077103FB0929BDF8143070
:108AE000C9F80400A9F8083013B0BDE8F08F00BF42
:108AF000400B0020ACA5010814000020001002402B
:108B0000079000085841002038B1038813EA01009B
:108B100003D08B420CBF0120022070470023F0B528
:108B20001D460D490D4E8B75DAB2032A03D905B1E6
:108B30008A750020F0BD5F1C06EBC30436F83330A5
:108B400001321842D2B24FF0010502D08A75204698
:108B5000F0BD3B46E8E700BFA815002032410020E9
:108B60002DE9F74F0120FFF7D9FF0024214D224EB8
:108B700068B3022C2BD84FF0CC0909FB04F855F848
:108B8000087005EB080A17B10134E4B2F0E70323DB
:108B9000C27890F902000093184B019753F82230E5
:108BA00001213A46FFF704FE834640B14A46394662
:108BB0005046013411F06BFAE4B245F808B00021D8
:108BC000B27D0F4FD3B2032B04D901B1B37503B0FB
:108BD000BDE8F08F02F1010E07EBC20037F832203A
:108BE0000133D207DBB24FF0010101D5B375BFE706
:108BF0007246E7E7D40C0020A8150020F4A901086C
:108C0000324100204000402830B4A8BF402000235B
:108C100002251424064A9D5402339918984201F8FB
:108C2000014CF8D8FF21D1540F2030BC0DF04EB9C3
:108C3000D019002090F8493013B1002280F8492063
:108C40001846704737B50446056D90F85C106B46C2
:108C500006221830A847A8B101209DF800209DF8F1
:108C6000013043EA0223A3849DF802209DF80330DB
:108C700043EA0223E3849DF804209DF8053043EA8B
:108C80000223238503B030BD37B50446056A6B4621
:108C900006223B210830A847A8B101209DF80020FA
:108CA0009DF8013043EA022363829DF802209DF87B
:108CB000033043EA0223A3829DF804209DF8053087
:108CC00043EA0223E38203B030BD0346012283F866
:108CD000352053F8043C143803B118477047022379
:108CE00010B50168047B0A68A3401A420AD0002428
:108CF000054A40681470026822F001021204120C46
:108D000002604B6010BD00BFAC35002070B504465A
:108D1000192004F1180508F056FD636D0022152195
:108D20002846984710B9022008F00BFF94F8462017
:108D3000636D42F01802162128469847636D0022A1
:108D4000172128469847636D01223D212846984700
:108D5000636D2846BDE8704001223E21184713B5D7
:108D60000446C06908F056FE0723104A6946A06908
:108D700004F079F8E06908F052FE01209DF8012026
:108D80009DF8023043EA0223A3849DF803209DF856
:108D9000043043EA0223E3849DF805209DF8063061
:108DA00043EA0223238502B010BD00BFD4A5010809
:108DB00068200CF045BA10B5082204460F2118208F
:108DC0000CF03EFA0E22102118200CF039FA4FF464
:108DD0008053238210BD134B10B51B780446082224
:108DE0002D215320A3B10CF02BFA0A22312153205C
:108DF0000CF026FA0C222C2153200CF021FA9022A0
:108E0000382153200CF01CFA4FF48073238210BDDC
:108E10000CF016FA0A22312153200CF011FA0A2222
:108E20002C21EEE7FE26002068200CF059BA13B57D
:108E3000062204466B4601211C200CF051FA08B3AF
:108E400004219DF800309DF8012042EA032242F3FC
:108E50008D0292FBF1F29DF8023062829DF80320B0
:108E600042EA032242F38D0292FBF1F29DF80530B3
:108E7000A2829DF8042043EA022343F38D0393FB6F
:108E8000F1F3E38202B010BD13B5062204466B462F
:108E9000022118200CF024FAB8B19DF801309DF899
:108EA00000201B0203EB920363829DF803309DF8C0
:108EB00002201B0203EB9203A3829DF805309DF86C
:108EC00004201B0203EB9203E38202B010BD304B7F
:108ED0002DE9F3411B780546002B3BD000242646A4
:108EE0002746A04601346B46082232215320E4B2C3
:108EF0000CF0F6F918B9002002B0BDE8F0819DF839
:108F000001209DF80030202C03EB02231BB29DF8BA
:108F1000032098449DF8023003EB02231BB21F4448
:108F20009DF805209DF8043003EB02231BB21E447C
:108F30009DF8073003F07F0301D0002BD2D198FBBE
:108F4000F4F897FBF4F796FBF4F4A5F81280AF82DF
:108F5000EC82D1E76B460622322153200CF0C0F997
:108F60000028C8D09DF801209DF8003003EB0223B3
:108F70006B829DF803209DF8023003EB0223AB8245
:108F80009DF805209DF8043003EB0223EB82B3E744
:108F9000FE26002010B500222A2104461C200CF0D9
:108FA0004FF902220E211C200CF04AF903220F2156
:108FB0001C200CF045F912222B211C200CF040F94A
:108FC000152008F09DFC18B1202383710023C37184
:108FD000062108F0BBFC02222C211C200CF030F9E9
:108FE00001222D211C200CF02BF900222E211C2007
:108FF0000CF026F905222A211C200CF021F94FF44F
:109000008073238210BD022210B4047B0168A24049
:1090100043694A6041680A6822F001021204120C96
:109020000A60596A9A6A914203D0184610BC08F047
:10903000F9BB012210BC83F84420704710B5084BDF
:1090400007281B68C8BF14381844007E0C4608F077
:1090500057FC20B12146BDE8104008F0E5BC10BD2A
:10906000680C0020F7B5054690F84D00002874D034
:1090700008F046FC044618B1202383710023C37115
:109080000621204608F062FC354B6B61002C64D051
:10909000A388B3FA83F3C3F11F035A1C50D04FF0D7
:1090A0000F0E30481435C218D6792F4A216842F87D
:1090B0002350DAB202F0030502F0FC0202F1804212
:1090C00002F580329768AD000EFA05FE27EA0E071A
:1090D00001F140419760A1F584319768C1F3872180
:1090E000A9403943012707FA03F39160D9431F4A86
:1090F000536115680D40156055680D405560156841
:109100001D43156095680D409560D5682940D16074
:1091100091680B439360164B9A5DF02A10DDF022A4
:1091200030449A55C37D01A88DF8043003238DF88F
:10913000053000238DF807708DF806300CF062F8CA
:10914000A3880122B3FA83F3C3F11F0312FA03F3D6
:109150001FBF06490A6813430B6003B0F0BD00BF90
:10916000CB8C0008D4A50108F80A002000040140B7
:10917000380B0020026D70B515880446ADB2A90603
:1091800006D5036B23B9C36AA3B1908880B2984710
:109190002B0620D5636AA26A9A42236D17D0511C10
:1091A000A069A162825C9A802369994213D300234B
:1091B000A36270BDE169928840694E1CD2B2E6613B
:1091C0004254E169E268914228BFE361E0E7DA686E
:1091D00022F08002DA6070BD70B50446056D8668C5
:1091E000AB8986B023F400531B041B0CAB8183793D
:1091F000617913F0020F14BF4FF40052002213F0F4
:10920000040F14BF4FF48060002011F0010F14BF51
:10921000042300238907298A48BF43F0080389B241
:1092200021F4405111432982AA8922F4B05222F03C
:109230000C021204120C02431343AB81AA8A01A848
:1092400022F440721204120CAA8201F037FF294A5C
:10925000039B0499954218BF19461922AB894A43CA
:1092600013F4004F14BF7100B100B2FBF1F164269A
:10927000B1FBF6F3AA891801120406FB13132ED5CD
:10928000DA003232B2FBF6F202F0070242EA0003E1
:109290009BB22B81A379DB070BD5236D154A934233
:1092A00025D0A2F57442934203D101200121FFF79A
:1092B000C5FEA379226D13F0080F938A0BBF23F02C
:1092C00008039BB21B0443F0080308BF1B0C9382E6
:1092D00093899BB243F40053938106B070BD1B0188
:1092E0003233B3FBF6F303F00F030343D0E7002060
:1092F000DCE700BF00380140072838B5D8BF044676
:109300000B4BC8BFA0F114041B6805462344187E0C
:1093100008F0F6FA58B127220134C4718271122183
:1093200008F014FB2846BDE83840002186E638BD29
:10933000680C00202DE9F04300234FF00F0E0126AA
:109340000F8847FA03F2D20723D58C784FEAD30867
:1093500014F0100F18BF91F8039003F0070504F004
:109360000F024FEA850550F828C018BF42EA0902EB
:109370000EFA05F92CEA090CAA4042EA0C02282C44
:1093800040F828200AD1C26806FA03F422EA04024F
:10939000C2600133102BD4D1BDE8F083482CF8D142
:1093A000C46806FA03F22243F2E70348D0F8B0306B
:1093B0000BB1A83018477047140000200348D0F8BC
:1093C00094300BB18C301847704700BF1400002058
:1093D0000248836F0BB170301847704714000020AB
:1093E0000248C36D0BB15430184770471400002079
:1093F0000248036C0BB13830184770471400002046
:109400000248436A0BB11C30184770471400002013
:109410000248836803B11847704700BF140000205A
:109420001FB5074B074A0293074B08490193084BA6
:1094300008480093084B08F0E3FC05B05DF804FB16
:109440009BBF0108E5BF010892BF0108A5BF010845
:1094500086BF01086FC40108BFBF010838B50A4BB9
:109460000D4603EBC00494F8B820084853F82210C6
:1094700008F00FFC94F8BE302BB1691C0448BDE81D
:10948000384008F006BC38BDF4A501081ECD01081F
:1094900080CF01082DE9F04F00252F46AA465E4EE9
:1094A0008BB05E4B5E491A680023934223DB013583
:1094B000102D06F13406F4D1584991F84B30BBB168
:1094C0004FF47A73086E4A6EB0FBF3F35209896E5B
:1094D000544808F095FC0A2297FBF2F39AFBF2F14C
:1094E00002FB13775048009702FB11A208F088FC9A
:1094F0000BB0BDE8F08F51F82300864222D0013333
:10950000D3E74346079A0121484808F0C2FB4C467E
:109510003AE038B10DF0ACFA014645480DF0B0FB29
:109520000DF0D6FC044642462946424808F0B1FBFD
:109530004FF0000928E0584631E021463E4808F047
:109540005FFC5BE07368012D0793336BD6F80080F6
:109550000893B36AD6F82CB00993F069D9D138B121
:109560000DF086FA014632480DF08AFB0DF0B0FC92
:10957000324B81461B78012B90FBF3F4C1D9424654
:1095800001212C4808F085FBBBF1000FD3D041F23C
:1095900088314FF47A700BFB0411B1FBF0F0099B9A
:1095A0005B091DBF41F288324FF47A7103FB04223C
:1095B0001A4618BFB2FBF1F21849052D91F84B106D
:1095C0001CBF8244BF180029B7D04FF47A7E089997
:1095D000B1FBFEF104910A2192FBF1FE01FB1E2278
:1095E000039290FBF1F201FB120100920191CDF880
:1095F00008E05A462146124808F002FC012D7FF48B
:1096000056AF0E4B1B78012B7FF651AF4A46079998
:109610000C4808F0F5FB4AE7DC000020C0150020EC
:10962000C4150020DFC40108FFC4010898C4010864
:109630000024744989C40108DBC40108582C0020A7
:10964000ABC40108CFC40108374B2DE9F3411968B9
:109650004FF47A733548B1FBF3F108F0D1FB344B8A
:1096600034491A78344B098803EB8203334AD3F820
:1096700030311278324808F0C3FB324B3248196857
:10968000324B334FB1FBF3F108F003FB08F0A1FBC1
:10969000304B314A1C883149314808F0B1FB314A1E
:1096A000314BA4B2314DD31A2146B7F86C20304863
:1096B00008F0A6FB2E6D002E33D030460DF0D8F901
:1096C00001462C480DF0DCFA0DF002FC8046D5F87E
:1096D000EC0038B10DF0CCF9014626480DF0D0FA77
:1096E0000DF0F6FB0446E86938B10DF0C1F901460A
:1096F00020480DF0C5FA0DF0EBFBB7F86E104346AD
:1097000064290190A8BF6421009432461A4808F0E9
:1097100077FB1A4B1A48198802B0BDE8F04108F0EF
:109720006FBBB046D3E700BF901B00202DC50108DA
:10973000F9350020321A0020F4A50108441A00204F
:1097400047C50108100000206DC5010840420F0008
:10975000C0150020B83B0020005000200008000089
:109760007DC501080000020800F80108DC000020A7
:10977000A1C5010800247449DBC501083436002066
:1097800021C601082DE9F04F0746304C87B02378F9
:109790002F4A608852F8238003F0E8FC2D4BD0F864
:1097A00004A093F8703082689BB1D346924601269C
:1097B00007F040030593A379721E002B08BF012315
:1097C000934208DC244B08349C42E0D107B0BDE84A
:1097D000F08F9B46EBE7A38813441AF803501BF85D
:1097E0000330EA1AD2F1000949EB020993B9009655
:1097F00043461A4A4946384608F0C4FBC5B9059B9A
:1098000033B900964346154A4946384608F0D0FB1E
:109810000136D0E703F00F021B0940330292019397
:10982000009643460E4A4946384608F0ABFBE5E74A
:1098300005F00F032D09403502930195009643462C
:10984000074A4946384608F0B3FBE1E7ACA60108F1
:10985000F4A50108C015002024A701083CC6010892
:1098600050C601082DE9F04F89B007460CF090FB77
:10987000044628B94120FFF785FF09B0BDE8F08F05
:1098800002469149384610F045FC904D06460028A6
:1098900049D18F4808F0D2FC8E4CDFF86C82DFF89B
:1098A0006C9204F58C77A2882168B2FA82F201F1F9
:1098B0004041A379A1F58431890A413155F823301B
:1098C000C2F11F02404608F0E4F9E17911B14846BF
:1098D00008F0DFF9083408F07CFAA742E3D108F079
:1098E00078FA7D4808F0AAFC7C4CDFF82482DFF887
:1098F0002492DFF824A2237E01363246012140461D
:1099000055F8237008F0C5F9627E39463AB15046E1
:1099100008F076FA072E04F11C04ECD1ADE74846B6
:1099200008F06EFAF6E7384607AA6D490DF0B2FF67
:1099300005F1B80782460026B84617F836302246A9
:1099400055F8231050464FEAC60910F0E3FB30B13A
:1099500001360F2EF1D1634808F070FC8DE707AA9D
:109960005F490DF097FF04460DF038FF4D4495F820
:10997000BE200746EAB9002828DCC844B8F802002F
:1099800003F0F4FBFBB20193019AB8F80430277896
:109990001344029343680393002F00F092805249CE
:1099A000204610F07CFBD8B9039B029A98544F488C
:1099B000D2E7002805DD1346BB4209DA002A08BFBA
:1099C000012201214A4808F028FA56E70123F3E76B
:1099D00007AA434900200DF05DFF013F0446CCE794
:1099E000A7F14105EDB2072D04D9A7F16105EDB24C
:1099F000072D66D8601C0DF0F1FEC3B20F2B824616
:109A00005FD86C1C40EA0414E4B2204607F078FFEB
:109A1000002856D0002C49D04FF0000823094033CD
:109A20000493DFF8F89004F00F03059300272FE06C
:109A3000B9F8020003F09AFBB9F8043042683B44DD
:109A4000D15CA14223D1464504D101998F421ED059
:109A50000021D154059A0499264808F01AF95FFAB2
:109A600087FB5FFA88F3594618460093FFF7F6FC28
:109A7000464509D1204808F00CF900985946FFF7EF
:109A8000EDFC1E4808F005F91D4808F0D7FB01372A
:109A900099F80630002B08BF01239F42C8DB08F16C
:109AA0000108B8F10F0F09F10809BFD15FFA8AF276
:109AB00005F14101134808F0A3F9039B029A9C5455
:109AC000DBE608F0C1FBD8E666C60108F4A501088C
:109AD0006BC601083416002079C601081400002066
:109AE00005CE010897C601084BC60108A5C60108A6
:109AF0009FC60108ABC60108CFC60108D2C601083F
:109B000065CD0108DCC601086EC6010880CF0108DA
:109B10007EC601081DCD010890C60108ACA601084B
:109B20002DE9F84304460CF033FA054620B101282C
:109B30001ED123782A2B1BD1104808F07FFB00246C
:109B40004FF00D09DFF83C800D4F09FB04863846C5
:109B5000316808F09EF8291C18BF012130460134F5
:109B600008F02CF908F035F9B22CEED1BDE8F883F5
:109B70002046BDE8F84309F057BB00BFE8C601081E
:109B8000B9CF010840B201082DE9F84F0024804602
:109B900025464FF00D0ADFF85090DFF850B00AFB71
:109BA000049637684146384610F002FB78B13946D2
:109BB000584608F06EF80021304608F0FFF808F02B
:109BC00008F9304608F030F908F003F9013501349E
:109BD000B22CE4D125B9BDE8F84F024808F02EBBFD
:109BE000BDE8F88FFBC6010840B20108B9CF0108F3
:109BF0002DE9F04F0D468DB0C249044604F028FA15
:109C00000646002840F02882BF49204604F020FA8A
:109C10000646002840F02282BC49204604F018FA8B
:109C20000646002840F01C822046B94904F010FA8C
:109C30000028064612BF0824264601240DB144F030
:109C40001004B44DB44FBD42C0F00C820123B34D9B
:109C500085F8703005F08AFC00F090FEB04930467F
:109C600004F0F6F908B144F0200414F0090F00F0F4
:109C7000DB810020FFF7D4FB04F01803182B04D17C
:109C8000A74808F02FF808F0A4F895F89031A54AF5
:109C9000002B0CBF01210021A34B204618BF134607
:109CA000A24A08F085F92046FFF76CFDDFF8E48250
:109CB0009F4B98F800601B789E4FA6EB0309D9F1E3
:109CC000000646EB090607EB83033146D3F83C3127
:109CD000994A204608F056F998F80030314607EBCB
:109CE0008307D7F83C31944A204608F061F90021F7
:109CF000D5F8A4014FF001060DF0A2F800B9064610
:109D000006F001018D4A204608F052F98C4A20469F
:109D100002F180018B4E07F06DF98B4A8B4920468A
:109D200006F0F6FD96F902104FF00009B1FA81F144
:109D3000874A4909204608F03BF9324685492046C2
:109D400004F0A4F9DFF850B2D5F8A472D5F8A882CF
:109D5000814B53F82960002E40F08B81B14668EAB0
:109D60000703DFF838B203937B4B53F82960002ECA
:109D700040F0A081D5F8AC32DFF824920393039A27
:109D8000D5F8B432DFF81CA25340DB43059301271A
:109D9000059A07FA06F31A42039A14BFB8464FF021
:109DA0000008134004934FF00C036C4A414603FB38
:109DB0000623D3F808B014BF4A4652465B462046F5
:109DC00008F0E0F8049A5B46002A14BF52464A465F
:109DD000414620463E4408F0EBF8132ED7D100232D
:109DE0005F4EDFF8C4E1DFF8C4C19A5D13F80E10CE
:109DF0000CA8104400F8181C13F80C000DF13008E2
:109E0000804408F80C1C2FB1A2EB0008D8F1000721
:109E100047EB08070133082BE7D1002609AB514A6D
:109E2000394620468DF8206008F0ACF806AB4D4A64
:109E30003946204608F0BCF84B4A4C49204608F009
:109E4000C9F84B4A4B49204606F044FF4A4A4B4961
:109E5000204606F0ABFE464A4649204606F0EEFD97
:109E6000474A204602F1500108F028F9454A2046A9
:109E700002F15A0107F0FCF9434A4449204607F031
:109E800023F84FF00108DFF828A1DFF828B17300AC
:109E900003931AF816201BF816309A4240F03181CD
:109EA00018F80A7018F80B10781A47424741022A2E
:109EB000DFF8809040F0278119211BF808204B44DF
:109EC0004A4393F8243302F2EE2201920093304A7F
:109ED00033463946204608F055F8192218F80A305A
:109EE0003946534303F2EE230193730013F80A300B
:109EF000274A994499F8243320460093334608F0C2
:109F000057F859E01FC7010856D401080DC10108D0
:109F100026C7010850E20108FCE50108C015002031
:109F20002AC701085017002008C7010833C70108D5
:109F30002C250020F4A501083BC7010844C70108EF
:109F400064170020862B0020F82B00208C2C00208A
:109F500053C70108EC2C0020A0A701081CA8010889
:109F60006437002077C70108324100208841002073
:109F70002434002070360020A4340020F036002065
:109F80007C1800201C1900206C2D00205C2D002066
:109F90007EC701082F25002060C701086CC7010893
:109FA0000AC7010814C70108ECAB010838360020C5
:109FB0007C2D0020E92A00200136122E08F102082B
:109FC0007FF465AF2146002007F06CFF210740F1C8
:109FD000B2802146002095F88C6104F025F82146D6
:109FE000012004F021F82146022004F01DF830463B
:109FF00004F0A8FF594803F041FC2146002095F8E1
:10A000008D6103F0FDFF2146012003F0F9FF214699
:10A01000022003F0F5FF30460BF028FF4F4803F015
:10A020000DFC4F4807F05EFEA20704D5214695F8C7
:10A030008C0103F0F9FF630704D5214695F88D01E3
:10A0400003F0DEFF474C484B9C427FD3002385F84A
:10A0500070300DB0BDE8F08F0124EFE50224EDE58E
:10A060000424EBE56A886968A8680DF0DFFB143505
:10A07000E9E53378DBB14FF0010A68EA07030AFA31
:10A0800009FA13EA0A0F14BF0121002133465A4688
:10A09000204607F077FF67EA080313EA0A0F5A46DB
:10A0A000334614BF01210021204607F081FF09F14A
:10A0B00001094DE633780BB34FF0010A0AFA09FAA9
:10A0C00018EA0A0F0BD067EA080313EA0A0F5A4688
:10A0D000334614BF01210021204607F053FF17EA41
:10A0E0000A0F0BD0039B5A4613EA0A0F18BF01212F
:10A0F000334608BF0021204607F05AFF09F1010945
:10A1000032E60027D3E64B4493F8243339460093D4
:10A11000164A3346204607F035FF154B72009B5C0C
:10A120003946994499F82433104A0093204633461F
:10A1300007F03EFF40E7214695F88C0103F074FFDD
:10A14000214695F88D0103F05BFF6DE76288A168F9
:10A1500060680DF06BFB143475E700BF0BDD010880
:10A160009BC7010850E20108FCE501088EC7010801
:10A170007C2D002038B504462568084629460CF099
:10A18000C1FB61680CF0C8FC29460CF0BDFB2060E7
:10A1900038BD0846704770472DE9F04F0022002572
:10A1A000624B634EB3F80AC087B034684FEA0C2A9A
:10A1B00005901889B4EB0A0A65EB020BA0FB0A456F
:10A1C00000FB0B55B3F80480E00940EA45604FEA14
:10A1D00008440719D8888E464FEAE511A0FB0A45C6
:10A1E00000FB0B5541EB0208CDE90278B3F8028081
:10A1F000200A40EA05604FEAC83410EB04084FEA31
:10A20000252141EB02099A89B446A2FB0A0102FB0F
:10A210000B11C20D42EA412212F5FA604FEAE153F6
:10A2200043F10001B0F5FA6FCDE9000171F10001D1
:10A230005DDADDE902670524A2FB040104FB0311DA
:10A2400000FB03F402FB0144A0FB020121444D107A
:10A250004FEA3004361B4FEA900467EB050744EAE7
:10A2600081748D104FF0FF313248B8EB040869EB70
:10A270000509DDE90045844275EB0101CDE902677E
:10A2800022DA40F6AC50002112184B4102FB03F1D8
:10A29000A2FB022303EB4103D900D000101A41EACC
:10A2A000527163EB0101341847EB0105CDE902451A
:10A2B0000B24A2FB040104FB031149104FEA3000F8
:10A2C000B8EB000869EB01090AFB0BF3DDE90001BB
:10A2D000AAFB0AAB0BEB430B4FEADA7242EA4B02E2
:10A2E000801A4FEAEB7361EB0301CDE90001DCF862
:10A2F0000410A1FB082301FB0933540D44EAC324D5
:10A300005D15DDE90223A21A65EB03031D46D30B9D
:10A31000059A43EA454302B11360BEF1000F02D033
:10A32000009BCEF8003007B0BDE8F08F90270020EA
:10A33000141A002024FAFFFF2DE9F74F6A4CDFF8CA
:10A34000ACE123880091DEF80810B4F90480C3EB77
:10A35000211252435B00C3EBE103B4F9021005463E
:10A360005943131308FB03F84FEAA83808EBE1211F
:10A3700001EB8102B1F5FA3802F180024FEAE1798E
:10A380004FEA222349F1FF39B4F90820A8FB08ABB2
:10A39000019308FB09F3A16102FB09F10BEB430BED
:10A3A000D31708FB0311A2FB08230B441F0316035A
:10A3B00047EA1257B4F90A2002FB0BF1D3170AFB44
:10A3C0000313A2FB0A011944020A42EA016292192C
:10A3D0004FEA2123E6887B410032A2FB060143F5C8
:10A3E000004306FB03114A10CB1752EA03016FD05A
:10A3F000B4F91060B4F90E0006FB0BF1F7170AFB75
:10A400000711A6FB0AAB00FB09F68B44C11708FB3A
:10A410000161A0FB08898944DEF80C104FEA484628
:10A42000C1F5801E1AEB060A76464FEA494747EA0D
:10A43000D8374BEB070BF7170026F90741EA5E0107
:10A440004FEACE7040F6354EB4F90C8016EB0A0692
:10A450004FEAC80747EB0B07861B61EB0707A6FB14
:10A460000E010EFB07110CF079FDB4F916204E1306
:10A4700002FB06FE470B47EAC147D31707FB03EE73
:10A48000A2FB07235643734407FB0366A2FB072383
:10A490003344560E46EAC3163218B4F914604FEA34
:10A4A000636747EB01037143F71700FB0717A6FB30
:10A4B00000013944C60C46EA413692194FEAE14799
:10A4C000B4F912607B41100A40EA036032011218AD
:10A4D0000DB1120A2A60009B13B11A46019B13604A
:10A4E00003B0BDE8F08F00BFA4270020141A00209D
:10A4F00070474FF40063038270474FF40063038298
:10A500007047037F13B1012B04D070474FF4806371
:10A51000038270474FF40063FAE737B50C46056DC8
:10A5200001AB02221B211830A84760B14FF48C7296
:10A53000BDF804305BBA9BB203F54E53103393FB66
:10A54000F2F32333238003B030BD38B5054600BF96
:10A55000064C206807F05EFA2946054802F0B1FC77
:10A56000206807F05CFA00BF38BD00BFBC0F0020B8
:10A57000003800400122482177200AF061BE012204
:10A58000582177200AF05CBE3122F42176200AF0AF
:10A5900057BE07B5032201AB002177200AF0A0FEC9
:10A5A0009DF805309DF804001B0243EA00439DF826
:10A5B0000600184303B05DF804FB08B5FFF7E9FF98
:10A5C000014B586008BD00BF141A002008B5FFF702
:10A5D000E0FF014B186008BD141A002007B50622E1
:10A5E0006B46F72176200AF07BFE9DF801309DF83E
:10A5F00000101B0143EA01339DF80210094A43EAA7
:10A600001113D3609DF804309DF803101B0143EA39
:10A6100001339DF8051043EA1113936003B05DF810
:10A6200004FB00BF141A002070B5044604F118059D
:10A63000FEF718FD636D80226B2128469847642041
:10A6400007F0C1F8636D03226B2128469847636DBC
:10A6500094F848201921284698470F2007F0B3F8AE
:10A66000636D94F846201A2128469847636D182296
:10A670001B2128469847636D18221C2128469847BD
:10A68000636D0222372128469847636D2846BDE84E
:10A69000704001223821184738B5044604F11805E6
:10A6A000FEF7E0FC636D80226B212846984764200A
:10A6B00007F089F8636D07226821284698476420CF
:10A6C00007F081F8636D00226B21284698476420CB
:10A6D00007F079F80122636D6B21284698470F2017
:10A6E00007F071F894F847301B21022B8CBF1A2217
:10A6F0001822636D284698470F2007F064F8636DB1
:10A7000018221C21284698470F2007F05CF8636D3B
:10A7100094F846201A21284698470F2007F053F84E
:10A72000636D94F84820192128469847642007F063
:10A730004AF8636D10223721284698470F2007F00A
:10A7400042F8636D2846012238219847BDE8384019
:10A750000F2007F038B810B504468021806902F058
:10A7600063FB012007F024F82046FFF795FF102235
:10A770006A2104F1180002F0D8FB642007F023F8E6
:10A78000A069022102F050FBBDE81040012007F053
:10A790000FB82DE9F74F054610461F4688460CF0C6
:10A7A00063F94C49044640460CF0B6F90146204690
:10A7B0000CF0B2F980460DF0D9F9044640460DF090
:10A7C00055F93946834638460CF09EF80146204636
:10A7D0000CF056FA9DF830600746012E4FF0000449
:10A7E0004BD008D3022E5FD02346A3462646A04670
:10A7F000A146A2461DE059464FF07E500CF082F86B
:10A800004FF07C5181460CF087F94FF07E51824623
:10A8100038460CF079F84FF04041064658460CF0A7
:10A820007BF9394683464FF07E500CF06BF8D046EA
:10A8300003463146504601930CF022FA3146286017
:10A8400048460CF01DFA3146686040460CF018FA94
:10A850003146A86058460CF013FA019BE860314677
:10A8600018460CF00DFAAC6128616C612C62EC6149
:10A87000AC626C6203B0BDE8F08F4FF040415846C7
:10A880000CF04AF94FF07E51814638460CF03CF806
:10A89000394606464FF07E500CF034F84FF07E58A3
:10A8A0000346CB46C246C4E74FF07E5100F1004854
:10A8B0000CF02AF84FF04041064658460CF02CF9AF
:10A8C000394683464FF07E500CF01CF8BA460346DA
:10A8D000A146AEE727D4D236002307B50093034B39
:10A8E000FFF757FF03B05DF804FB00BFF304353FEB
:10A8F00070B50D460CF0B8F8044628460CF0B4F8D4
:10A90000014620460CF0BCF90DF0ECF801460BF0C6
:10A91000FBFF4FF080440546014620460DF02CFA1F
:10A920004FF07C51064628460CF0F6F801462046CA
:10A930000DF022FA4FF07E51044630460BF0E2FF54
:10A94000014620460CF09CF970BD01234A0901F034
:10A950001F0103FA01F150F822300B4340F8223076
:10A96000704701234A0901F01F0103FA01F150F871
:10A970002230194214BF0120002070474FF47A6240
:10A980000221294BF0B51A80284A64201170002159
:10A99000517040F219421A820122254B6E27DA705B
:10A9A00058715981D981234B4D241A46502603F101
:10A9B000240510705770917054719471D6710C32D7
:10A9C000AA42F6D164266E2500244D2050211E7027
:10A9D0005D709C7058719871D9710C339342F6D1A7
:10A9E0003220154BC82283F83A003C2083F83B20E4
:10A9F0001870D97046205A219A712D2219715870F9
:10AA0000DA7111201E2212215A75DA759870597167
:10AA10000A4B1B78012B95BF2C220122084B094BB6
:10AA200094BF1A719A70F0BD78230020B8310020CD
:10AA3000BA3B002040110020AA320020E40A002086
:10AA400064110020D43A0020094A0A4913781844B6
:10AA5000C0B210F0800F18BF803810701078134605
:10AA60000A78904202BF00220A701A70704700BF35
:10AA7000E93A0020E83A002010B50A4B0A4A1B7850
:10AA800042609C18094A0460127893429DBFD31A11
:10AA90000B600023C3F1800392BF4B600B604A60E0
:10AAA00010BD00BFE93A0020EA3A0020E83A002051
:10AAB0001FB502A86946FFF7DFFF044B00981B682B
:10AAC0001844019B184405B05DF804FBE43A0020EB
:10AAD000054B1878054B1B78984236BFC3F18003AD
:10AAE000C01AC018704700BFE83A0020E93A0020B9
:10AAF00037B5104C2078C0B105238DF80030002305
:10AB00008DF8013000BF0C4D286806F083FF02234A
:10AB10006A4601A9094802F0A6F9286806F07FFFF5
:10AB200000BF9DF8050000F00100207080F00100DA
:10AB300003B030BDC00F0020BC0F00200038004023
:10AB400070B50646044C2568FFF7D2FF18B9236894
:10AB50005B1BB342F8D970BD901B00202DE9F04F6C
:10AB600087B0019300238246029103920093039AD7
:10AB700093420CDB019B002B40F08880FFF7B8FF6D
:10AB8000002840F08380019807B0BDE8F08F029A5A
:10AB9000009952F82320013311440091E7E7022283
:10ABA0008DF814201A0C8DF8152006201A0A8DF83D
:10ABB00016208DF81730FFF7C3FF0620FFF7C5FCFE
:10ABC0000123334A137000BF4FF00008D1462746D7
:10ABD000304B186806F01EFF042305AA00212E48FA
:10ABE00002F041F9029D039B984515DA2B684FEA64
:10ABF000880B002B44D09F4233D83B465AF80B2099
:10AC00000021254802F02FF95AF80B303B444AF84E
:10AC10000B302B68DF1B2F601E4B186806F0FFFE01
:10AC200000BF1E4B361B1B681C441C4B1C60019B49
:10AC3000A3B19EB1194B1B68DCB23219B2F5807F0B
:10AC4000174A88BFC4F58074D26898BF34469342CF
:10AC5000A5D30023134A1370134A1370009B981B4B
:10AC600092E7D9F8002000210B4802F0FCF82A688E
:10AC7000D9F80030BF1A1344C9F8003000232B6004
:10AC800008F10108043509F10409ACE7009ED0E79A
:10AC9000C00F0020BC0F002000380040E43A002024
:10ACA00038040020E83A0020E93A002030B50B4C87
:10ACB0000B4D22782B7885B09A420CD002A96846B9
:10ACC000FFF7DAFE0123022202A96846FFF746FFDA
:10ACD00000232B70237005B030BD00BFE93A00207F
:10ACE000E83A002030B50E4D0E4C2A78237885B016
:10ACF0009A4212D002A96846FFF7BEFE0023022244
:10AD000002A96846FFF72AFFFFF79EFE28782378FE
:10AD1000C31A5842584105B030BD0120FBE700BFBF
:10AD2000E93A0020E83A002008B545F20820FFF78C
:10AD300007FF0620FFF709FC0122064BC7201A7007
:10AD4000FFF703FC0023044A1370044A1370044AFB
:10AD5000136008BDC00F0020E83A0020E93A002047
:10AD6000E43A0020032373B58DF80430030C8DF80A
:10AD700005308DF80700030A06200E4614468DF8AC
:10AD80000630FFF7DDFEC0B100BF0D4D286806F0AC
:10AD900041FE042300210DEB03020A4802F063F890
:10ADA000234600223146074802F05DF8286806F085
:10ADB00036FE00BF204602B070BD0446FAE700BF71
:10ADC000BC0F002000380040084BDA68D10709D4D6
:10ADD000DA68520708D4DB6813F0100F14BF0320A1
:10ADE0000420704701207047022070470020024075
:10ADF0002DE9F0410E46054607464FF6FF7443180D
:10AE00009F4211D1DFF83880BD4212D1E1B2D8F8AB
:10AE1000000006F044FDD8F80000210A06F03FFDCE
:10AE2000B01CC0B2BDE8F08117F8012BA41AA4B27F
:10AE3000E6E715F8011BD8F8000006F030FDE3E75F
:10AE4000241A002007B58DF80610090A8DF807109E
:10AE50000421062360F05F008DF805000DEB010072
:10AE60008DF80430FFF7C4FF03B05DF804FBA0F1D8
:10AE70007D03012B70B504460D460B4E11D87D2184
:10AE8000706806F00CFD84F02001706806F007FD84
:10AE900035B12888204400EB102000F0FF00288006
:10AEA00070BD0146F1E700BF241A00205E2810B5EE
:10AEB0000146094C09D15D21A06806F0F0FC3E2155
:10AEC000A068BDE8104006F0EABC5D29A068F8D192
:10AED00006F0E5FC3D21F3E7241A0020F0B50C460E
:10AEE000054689B01422002120460FF0D0F804A9AD
:10AEF0002A6800230D461D4EC2F3855040FA03F721
:10AF0000FF0748BF9F5D03F1010344BF0F7001318C
:10AF1000062BF3D1002315480B70C2F30321014423
:10AF20008979C2F305368DF818100D300DF119012D
:10AF300046FA03F7FF0748BF1F5C03F1010344BF54
:10AF40000F700131062BF3D100230B70C2F3834342
:10AF5000029306AB0193009502F00F030449C2F37C
:10AF6000031220460AF0D8FB09B0F0BD88A90108F9
:10AF7000A2CB01080023036043608360C3600361C8
:10AF800043618361C36103624362836270478B687C
:10AF900010B50C6A026823430C6922F4FF42234374
:10AFA0004C6922F0700223438C692343CC6923430C
:10AFB0004C6A23438C6A234313430360CB6843608A
:10AFC0000B6883604B68C36010BD036823F0010306
:10AFD0001B041B0C03600023036043608360C36099
:10AFE000284B984204D1284A536843F00F0326E0C7
:10AFF000264B984204D1244A536843F0F0031EE0E4
:10B00000234B984204D1204A536843F4706316E0FE
:10B01000204B984204D11C4A536843F470430EE01D
:10B020001D4B984204D1184A536843F4702306E03C
:10B030001A4B984205D1144A536843F47003536085
:10B040007047174B984204D10F4A536843F070631E
:10B05000F5E7144B984201D1134AC5E7134B9842C8
:10B0600001D1114AC8E7124B984201D10E4ACBE7F1
:10B07000104B984201D10C4ACEE70F4B9842DFD1DA
:10B08000094AD1E708000240000002401C000240CB
:10B090003000024044000240580002406C00024070
:10B0A0008000024008040240000402401C040240E8
:10B0B000300402404404024058040240214A10B5C2
:10B0C000536803F00C03042B25D0082B26D01E4B0D
:10B0D000036053681D49C3F303130B44DC7C03680E
:10B0E000E34043605468C4F302240C44E47C23FA34
:10B0F00004F484605468C4F3C2240C44E47CE34048
:10B10000C3605268C2F38132114491F82320B3FB2B
:10B11000F2F3036110BD0E4B1B68D9E75368516809
:10B12000C3F38343C90303F1020302D409494B4328
:10B13000CEE7516811F4003F0549096818BF490876
:10B14000F5E700BF0010024000127A0088A901084C
:10B15000D800002000093D0010B50446FFF734FE7A
:10B16000012806D10CB9052010BDFFF72DFE013CCA
:10B17000F6E7002C08BF052010BD0B88F0B54E88FF
:10B18000B1F804E00F89CC88002B3CD1038C23F06C
:10B1900001031B041B0C0384018B824B89B221F039
:10B1A000F301058C4EEA010141EA07119842ADB264
:10B1B00089B212D003F5006398420ED0B0F1804FEF
:10B1C0000BD0A3F59833984207D003F580639842DB
:10B1D00003D003F58063984212D125F0020546EAB8
:10B1E000050343F0010301830384038B23F00C0365
:10B1F0001B041B0C0383038B9BB21C430483F0BD15
:10B2000025F00A05EBE7042B44D1038C4FEA0E2E00
:10B2100023F010031B041B0C0384038B4EEA073737
:10B2200023F440731B051B0D1F435E4B018C98429A
:10B2300089B2BFB212D003F5006398420ED0B0F1CC
:10B24000804F0BD0A3F59833984207D003F5806365
:10B25000984203D003F58063984214D121F0200175
:10B2600041F0100343EA06139BB207830384038B68
:10B2700023F440631B041B0C0383038B9BB243EA40
:10B280000424A4B2BAE721F0A00146EA010343F086
:10B290001003EAE7082B038C3FD123F480731B04CF
:10B2A0001B0C0384818B3F4B89B221F0F301028C8C
:10B2B0004EEA010141EA0711984292B289B212D0D6
:10B2C00003F5006398420ED0B0F1804F0BD0A3F588
:10B2D0009833984207D003F58063984203D003F572
:10B2E0008063984213D122F4007343F4807343EADD
:10B2F00006239BB281830384838B23F00C031B04FE
:10B300001B0C8383838B9BB21C438483F0BD22F48C
:10B310002063334343F48073ECE740F6FF4223F4A9
:10B3200080531B041B0C0384818B038C0A4039035C
:10B3300041EA0E2111431B4A9BB290421FFA81FE43
:10B3400012D002F5006290420ED0B0F1804F0BD0C7
:10B35000A2F59832904207D002F58062904203D065
:10B3600002F58062904215D123F4005343F48053D8
:10B3700043EA06339BB2A0F81CE00384838B23F4DA
:10B3800040631B041B0C8383838B9BB243EA04241E
:10B39000A4B2BAE723F400735B045B0C334343F4B9
:10B3A0008053E8E7002C01400F4B1A6842F001027D
:10B3B0001A6059680D4A0A405A601A6822F084726D
:10B3C00022F480321A601A6822F480221A605A68C5
:10B3D00022F4FE025A604FF41F029A604FF000629E
:10B3E000034B9A60704700BF001002400000FFF856
:10B3F00000ED00E080F30888704702464FF6FF73C7
:10B4000030B58C1E151AAC420BD8014411F8012C32
:10B41000B2EB132F0AD1005DDBB2C31A5842584178
:10B4200030BD12F8015B5B1B9BB2EBE7002030BD27
:10B4300013B5304B4278197B02F00F0409B904B1FF
:10B440001C73197B8C4203D3611AC8B202283ED9FF
:10B4500000204CE0902A13D106238DF80430264BAF
:10B4600064F06F04194491F8273004218DF80630F8
:10B4700002238DF805408DF807300DEB010034E014
:10B48000A02AE5D11C4A114491F82720022A19D09C
:10B49000032A09D0012ADBD10A21184BB3F9443021
:10B4A000594301F5C87108E00A21DA895143DA7F6E
:10B4B0001AB193F8203091FBF3F189B22046FFF7DF
:10B4C000C1FC14E0186B0BF029FD81B2F6E702F025
:10B4D000F002802ABED10423022164F07F048DF89B
:10B4E00004308DF805400DEB0300FFF781FC02B03E
:10B4F00010BD00BF241A002088A90108CC3B002001
:10B500004FF6F672074BDA8703F144025A630122C1
:10B51000998703F1450183F84400996383F8442136
:10B52000704700BF241A0020002373B502AD25F830
:10B53000023D0C462946FFF79AFCA61D14F8010BA4
:10B540002946FFF794FCB442F8D19DF8060000218B
:10B55000C043C0B2FFF78BFC02B070BD07B50B0A49
:10B560008DF800008DF802108DF80330000A0B0CE6
:10B57000090E8DF801008DF80510102069468DF830
:10B580000430FFF7D1FF03B05DF804FB73B50E4C38
:10B590000646D4F848010D46FDF7DEF8E37D227E2D
:10B5A000003318BF01230AB143F00803019396F951
:10B5B000000000954FF4964300220821FDF7F8F8AB
:10B5C000C4F8480102B070BD241A002010B5064C22
:10B5D000D4F8480106F060F900B910BDD4F848016C
:10B5E00006F057F9F4E700BF241A002008B50B4B0A
:10B5F000D3F84C2192781E3A012A08D9D3F8480191
:10B6000001210430FFF7C2FFBDE80840DEE7012159
:10B61000D3F8480106F037F9F6E700BF241A0020F6
:10B620000028114AB8BF404290FBF2F330B50F4CEE
:10B6300004FB03053C2068430D4D90FBF2F26D7E48
:10B6400075B903EB830303EB830302EB83030B80E6
:10B650004FF47A7304FB020292FBF3F24A8030BD8E
:10B66000C3EB0313F1E700BF80969800806967FF82
:10B67000241A002010B50446C0B2FFF717FCC4F32B
:10B680000720BDE8104011E4024B5E21986806F0E7
:10B6900006B900BF241A002038B50546054C5E21C6
:10B6A000A06806F0FCF82946A068BDE8384006F01E
:10B6B000F6B800BF241A002073B56F4CD4F850615F
:10B6C00076B1304609F0B8F950B194F8543133BB33
:10B6D000D4F858311BB3A360012384F854311EE021
:10B6E00094F85C0109F0C0F994F85431054683429E
:10B6F00015D0002800F09D808EB1E37D96F9020000
:10B70000B3FA83F35B09019302230022009304211F
:10B710004FF41653FDF74CF8A0600028DCD194F8E4
:10B720005D0109F0A1F994F85E31054683421DD010
:10B73000002800F08580D4F84C31BBB1227E93F90B
:10B740000200002A0CBF002208220323019200936A
:10B7500000224FF496430821FDF72AF8C4F8480167
:10B7600020B1FFF743FF012384F85E3194F85F01B5
:10B7700009F07AF994F860310546834222D0002816
:10B7800067D0D4F86421EAB1237E92F90200002B3D
:10B7900014BF08230023E27D2021002A08BF43F0C4
:10B7A000010301930323002200934FF46143FCF74C
:10B7B000FFFF606030B1012384F8683184F86031A4
:10B7C000D4F86C3194F8700109F04EF994F87131A5
:10B7D000054683422BD0002844D04FF47A72274B81
:10B7E000C3F8B822D4F874310BB31A8802F4825229
:10B7F000B2F5825F1BD093F90200E37D0022002B9B
:10B8000014BF09230823019303234FF480510093AD
:10B810004FF4E133FCF7CCFFC4F8780138B10023D2
:10B8200001222060237384F8712184F87C3102B0F6
:10B8300070BDA068FCF790FFA56084F854516EE7D6
:10B84000D4F84801FCF788FFC4F8485184F85E51E9
:10B850008CE76068FCF780FF656084F8685184F8C5
:10B860006051AFE7D4F87801FCF776FFC4F878515F
:10B8700084F87151DBE700BF241A0020D8000020B3
:10B88000426A806A131A58425841704741717047A2
:10B8900043799B070AD5436A8269D154436A016997
:10B8A0000133B3FBF1F201FB12334362704743797A
:10B8B00013F0020308D00369426A806A013B101A40
:10B8C0001840C0B2181A704718467047437913F0F1
:10B8D00001031FBFC369026AC0689B1A1ABF00F147
:10B8E000FF3018401846704710B54379014613F0F1
:10B8F00001030ED0FFF7EAFF60B10B6A4A69CC681A
:10B90000D05C0133B3FBF4F204FB1233C0B20B6220
:10B9100010BD184610BD90F8433230B53BB9012434
:10B9200090F8411290F84232DAB2914200D830BD1C
:10B93000B0F84A5204FA03F22A43A0F84A2201332B
:10B94000F2E7836B19685A79012393400A8C9BB202
:10B9500092B222EA03020A840A8C92B213430B8445
:10B96000704710F80A3C0133DBB20A2B00F80A3C9E
:10B9700007D9002310F8131C024A22F8113000F8EE
:10B980000A3C7047BC29002070B51424454B1A7836
:10B990000132B2FBF4F004FB102298681A705A6C62
:10B9A0008142DC680A4404D293F84C0008B102F5E5
:10B9B00080323D480678B2FBF6F2944223D293F8E7
:10B9C0004C501DB14FF4803595FBF6F5101B451B0F
:10B9D0001D61DA6040F68C2200209960196983F8B5
:10B9E0004C00914241D9187993F94920904230D1C5
:10B9F000021F082A2DD893F84A20182A0BD80132A2
:10BA000083F84A2009E04FF4803090FBF6F0001BE9
:10BA100010441861DDE783F8480093F9482090420C
:10BA20000FD193F84B1061B10021204C204D914271
:10BA300011DB00241E490B2A13DD1E490A7801324E
:10BA40000A70012283F84B20002283F849001A7102
:10BA500070BD0022D4E754F8046F25F8116001315D
:10BA6000E5E721F812400132E5E793F84B20C2B137
:10BA700040F2DA52A1F2EF20904207D81A790B2A4D
:10BA800004D803EB820041610132E0E7002283F831
:10BA90004B20114613460848C2180433302B11615D
:10BAA000FAD170BDB81B00201C040020C81B002068
:10BAB000BC290020B5290020BC1B002010B514248F
:10BAC000094B1A780132B2FBF4F004FB10221A7011
:10BAD0005A6C01320A445A644FF6FF72914204BF15
:10BAE000012283F84C2010BDB81B0020704770471E
:10BAF00038B5A0F517746379A579DB0744D594F8B8
:10BB000040321BB3A06B0268938DC3F34E03938442
:10BB100094F85132012B07D094F8453223B1B4F890
:10BB20004C320133A4F84C32E94301F0010109F031
:10BB3000A6FC012384F84332002384F8413284F8C0
:10BB4000423284F84032A4F84A3238BD94F8433285
:10BB50002046012B04BF94F8413284F84232FFF7AB
:10BB6000DAFE94F843324BB90123E94384F84332B7
:10BB70001940A06BBDE8384009F081BC002305F0F6
:10BB8000010184F84332F4E738BD10B583790446E7
:10BB9000DB07006B4CBF2A214A2105F0D7FE0123A9
:10BBA00084F8443284F840320023204684F841323D
:10BBB000BDE81040C5E6084B10B41A681346B3FB45
:10BBC000F1F4B4F5803F03D3012BFAD95B08F6E713
:10BBD000A1B210BC05F0FCBC100000208160806B9D
:10BBE000E9E78379406BDB0744BFB1FA81F149098A
:10BBF00009B105F014BF05F00DBF10B5A0F515741F
:10BC000063799A0714D594F84522002A59D1A36A7A
:10BC1000616A994221D194F844324BB9A3791B0748
:10BC200006D5606B062105F091FE2046FFF7ADFFBB
:10BC30006379D90740F1998094F84032002B40F0A5
:10BC4000948094F841320133DBB2092B84F84132FD
:10BC50004DD12046BDE810405DE6591CA069A162A7
:10BC6000C35C2069DBB25B0043F40073A4F8483284
:10BC70000A2381424FF0010184F8463294F844329D
:10BC800028BFA26284F84512002BD1D0A3791807EF
:10BC9000CED5A06B02684079138C81409BB223EA19
:10BCA00001031384138C206B9BB21384062105F0CF
:10BCB0004DFE0023122184F84432606B05F046FEED
:10BCC000B6E794F946327BB1B4F8481220464B08E7
:10BCD000A4F8483201F00101FFF783FF94F84632DF
:10BCE000013B84F84632A3E784F84532A0E70A2BEB
:10BCF0003BD194F843322BB9B4F84A3243F00103F4
:10BD0000A4F84A32B4F84A02820501D4C3071AD40F
:10BD1000B4F84E320133A4F84E320122002384F8E5
:10BD2000402294F8432284F84132012A1DD1A1799E
:10BD3000A06B84F8433201F0010109F0A0FB20461A
:10BD4000BDE81040FDE5E36AC0F347000BB198473A
:10BD5000E3E7E3696269D054E369E1680133B3FB67
:10BD6000F1F201FB1233E361D7E710BD182370B580
:10BD70000E465843074A14181558A16830460AF071
:10BD8000CBFEE1680AF0C0FD0BF0B6FE80B2288061
:10BD900070BD00BF802500202DE9F04718255026F2
:10BDA0004FF028084FF00009144C154F05FB0045D3
:10BDB000A54201D1BDE8F087237CCBB1D4F804A023
:10BDC000504605F03DFCEFF3128386F31288BAF873
:10BDD000242008FB007092B201324267BAF81420A6
:10BDE000DBB292B242F00102AAF8142083F3118868
:10BDF00054F8183BA3F80090DAE700BF8025002034
:10BE0000B81B002008B50A4A1378D9070FD523F0CC
:10BE100001031370074B9B780BB100F0BFFE0020AD
:10BE200005F00CFEBDE8084004200AF04FB808BD3C
:10BE3000A4350020D43A002038B5334B1B78D907FD
:10BE400005D5BDE838400121002005F023BE1B20A8
:10BE500006F03AFB2D4C00283CD004200AF090F864
:10BE600006F046FB00283AD008200AF089F8284B53
:10BE70001B781A0738D410200AF082F8254B1B884B
:10BE8000642B36D920200AF07BF8234B234D1B6806
:10BE900013F0040F02D0B5F8F02042B9B5F8F22043
:10BEA0000AB19B0703D41E4BB3F8A83033B340202C
:10BEB0000AF066F8238803B1022385F8F43005F010
:10BEC0002FFCD5F8F830C01A00281CDBBDE838403C
:10BED000FCF798BB238823F004032380C0E7238862
:10BEE00023F008032380C2E7238823F01003238074
:10BEF000C4E7238823F020032380C6E7238823F0A8
:10BF000040032380D6E738BDA43500203436002016
:10BF1000ED2600202E16002028250020B81B00202A
:10BF2000CC3B002070B5314C23783BB1304D2B78A1
:10BF300023B9304802F072FE01232B70FFF77CFF1B
:10BF40002D4B1A8802BB2D4A137813F001014BD1F7
:10BF500043F0030313700A22294BB3F9043093FB17
:10BF6000F2F3284A1380284B284A1868A3784FF424
:10BF70007A7404FB03030520C2F8FC30C2F80011F8
:10BF8000BDE8704009F0A2BF194B1B781BB1204BD4
:10BF9000B3F8A83043BB92FAA2F3002AB3FA83F3B2
:10BFA00008BF4FF0FF33194A0133D2F800118B421A
:10BFB0001AD0C2F80031DBB29B00402BA8BF40234F
:10BFC000002214260A20052512495418565404321A
:10BFD0006070A5709A4202EB010404F8010CF4D3DE
:10BFE000FF230F208B54CBE770BD00BF70110020E2
:10BFF00078110020743C002034360020A435002045
:10C000008C31002086100020901B0020B81B0020DF
:10C01000CC3B0020D01900202DE9F04F4FF41874CC
:10C0200089B098469DF84830814E039300F10A0389
:10C03000334493F8D0B593F8C435059144430021B7
:10C04000054658460292019303F0B0FB0021079089
:10C05000019803F0ABFB8146584605F051FC069071
:10C06000019805F04DFC039B06F5827713F0080359
:10C07000049307EB040A069A079B00F09B80B9F132
:10C08000000F03D1002009B0BDE8F08F3319C3F8C9
:10C090003C91C3F83801C3F8340105F10B03DBB25E
:10C0A00010B10B22C37182714FF418794FF0000B5D
:10C0B0004FF4807209FB05695E4BC9F81021C9F87D
:10C0C0000431029BC9F81421C9F80C319DF80C30D9
:10C0D000029989F80A31059BD9F83C01C9F8303139
:10C0E00004F140033B44C9F8183104F5A0733B4404
:10C0F000C9F81C3189F80981C9F824B1C9F820B1FF
:10C10000C9F82CB1C9F828B189F85453A9F850B32B
:10C11000A9F852B389F848B389F849B3FFF74BFD42
:10C12000039BD9F83C0103F0010109F0A8F9424A48
:10C1300004F51773C9F86023404A04F5157418F024
:10C14000020F3B44C9F858232744C9F85CB362D0B6
:10C15000D9F8400100285ED0D9F83C11026809687E
:10C160008A4258D00122029989F855230193FFF79A
:10C1700022FD3A465946D9F8400105F07DFA019B67
:10C180005A461946D9F83C0105F076FA049B63B982
:10C190004FF4187303FB05651221D5F8380105F03B
:10C1A000D5FB01215046FFF71CFD5046FFF7EDFC83
:10C1B000504668E718F0010E12D0BBF1000F3FF4B3
:10C1C00061AF002B3FF45EAF3119C1F83C3105F18E
:10C1D0000B03C1F83421DBB212B10C21D371917180
:10C1E00018F0020F3FF460AF019B002B3FF44AAF01
:10C1F0004FF4187303FB0563C3F83801BEF1000F59
:10C2000006D1B9F1000F3FF43DAFC3F83C9144E7CC
:10C21000C3F8409141E74FF41870002200FB05601D
:10C22000194680F855233A46D0F83C01ACE700BFE8
:10C23000B81B0020B4A90108F1BA0008FBBB000834
:10C240001FB50123ADF808300023ADF80C30ADF870
:10C250000A30094BADF8041093F8E83501A9012B19
:10C2600008BF0323ADF8062008BFADF80C30FEF779
:10C2700084FF05B05DF804FBB81B002038B510F84A
:10C280000E2C044650F8043C52B9012220F80C1C34
:10C2900000F80E2C597918680222BDE83840CFE723
:10C2A000002530F80C2C20F80A1C891A89B220F8D5
:10C2B000081C074A10F80F0C22F8101004F80E5C46
:10C2C0002A4659791868FFF7BBFF04F8065C38BDA9
:10C2D000BC2900201823064A10B503FB0020D0F823
:10C2E000EC4524B108460BF007FC80B2208010BD5D
:10C2F000B81B0020072800D8ECE77047084608F074
:10C3000099BE0FB407B504AB53F8042B04490020C1
:10C31000019301F0A2F803B05DF804EB04B070479C
:10C32000FDC200082DE9F74F3A4C0025D4F80080F3
:10C3300004F10C01464608F1300746F8040B04F1FD
:10C34000180B04F1240A04F13009685801910AF02D
:10C35000BFFD46F8040B55F80B000AF0B9FDB060BC
:10C3600055F80A000AF0B4FD2B4B7061EB185868C1
:10C370000BF0C2FB09EB05035B6B043527F8020BDE
:10C380000C2DBB800199E0D10025244F08F128062F
:10C3900057F825000AF09CFD0135042D26F8020B04
:10C3A000F6D10025B4F8743094F87C70A8F83C30CD
:10C3B000B4F87630DFF87090A8F83E30B4F87830F2
:10C3C00008F14406A8F84030B4F87A30A8F84230B2
:10C3D000BD4216DB124B5B88A8F86430D4F8A43059
:10C3E000A8F86630D4F8C430C8F868300D4B1B8804
:10C3F000A8F86C30B4F8D630A8F85E3003B0BDE8C9
:10C40000F08F59F825000AF063FD013526F8020B7C
:10C41000DEE700BF8822002020410020481A0020CB
:10C42000321A0020F43500200823002010B50446FD
:10C430007F2C04D8E0B2BDE8104008F0FBBD64F0EA
:10C440007F00C0B208F0F6FDE409F1E70EB477B55D
:10C45000064607AC482054F8045B08F0EBFD2020AA
:10C4600008F0E8FD304608F07BFD3A2008F0E2FDD8
:10C4700023462A4609490020019400F0EEFF0446B5
:10C480000A2008F0D7FD064A033413681B1B13600B
:10C4900003B0BDE8704003B0704700BFFDC20008A4
:10C4A000D03A00200E4BB3F8DC200132A3F8DC2098
:10C4B000D3F8E0200132C3F8E020B3F8E4200132E1
:10C4C00092B2202A03BF0022A3F8E420B3F8E620AA
:10C4D000A3F8E42004BF0132A3F8E620704700BFB0
:10C4E0008822002038B5244B054693F8E8300C46E6
:10C4F000093B012B3ED8452008F09CFD284608F05A
:10C5000099FD0E2D0DD003D83DB10D2D0ED038BDA7
:10C510001E2D06D0FF2D28D038BD2068BDE838403C
:10C5200084E72068FFF782FF6068F7E76378207888
:10C53000A3B180F0800008F07DFDA468E0B208F0AF
:10C5400079FDC4F3072008F075FDC4F3074008F037
:10C5500071FD200EBDE8384008F06CBD08F06AFDA2
:10C560006068BDE8384008F01CBE044808F0F8FCDC
:10C570000020EFE738BD00BF882200201CCC010856
:10C580002DE9F04F634C8BB0B4F8E4300546624FB0
:10C59000002B40F0C7803B78012B04D17B78202B07
:10C5A00001D101F061FF2846FFF7BCFE2568492054
:10C5B0002E4608F03FFDD4F8E000FFF737FF56F8AD
:10C5C000040BFFF733FF304609F00AF905F11000BC
:10C5D00009F006F910264FF0010905F11C08D4F8FE
:10C5E000EC2009FA06F3134203D0D8F8000008F053
:10C5F000D8FD0136132E08F10408F0D1032105F10E
:10C60000280008F0D3FDB4F80031B5F92E00C01AA7
:10C61000FFF70CFFD4F8EC30D80408D5B4F80601C5
:10C62000B5F86430C01AC0F30D00FFF7FFFED4F870
:10C63000EC30990403D5B5F86600FFF7F7FED4F89F
:10C64000EC301A0502D5A86E08F0ABFDD4F8EC303A
:10C650001B0403D5B5F86C00FFF7E8FE032105F1D4
:10C66000300008F0A3FDD4F8EC30DE0204D503213D
:10C6700005F1360008F09AFDD4F8EC30980204D5A4
:10C68000042105F13C0008F091FD0126B5F94400B4
:10C690000AF0EEF9D4F808110AF034F90AF03EFC79
:10C6A000FFF7C4FE94F87C9005F14608B14527DCFD
:10C6B000D4F8EC30990505D5B5F95E00A0F2DC5050
:10C6C00008F06FFD22686260A2601449144B521A90
:10C6D000121153430322013393FBF2F202EB4202A5
:10C6E0009B1A702202FB03132360012384F85C323F
:10C6F000BB78012B01D1FEF7F5FA0BB0BDE8F08F46
:10C7000038F9020BB5F944300136C01A08F049FD7A
:10C71000CCE700BF88220020D43A002094230020D8
:10C72000B76DDBB6D4F86032D4F864229A4207D0F1
:10C730000AA941F8203D0020C4F86432FFF7D2FE78
:10C740000422B94988180DF079FC60B1D4F8683238
:10C750000AA90393D4F86C321E2041F8203DC4F896
:10C760006832FFF7BFFE3978B4F8E43078780B44CC
:10C77000013BB3FBF0F200FB12339942B8D901F050
:10C7800073FE2846FFF7CEFD5020D4F80090D4F871
:10C79000048008F04FFCA268236810681B68626878
:10C7A0000344106809F10405A3EB400008F0F9FC0C
:10C7B000002308F1040050F8231055F82320521AE2
:10C7C00002A941F823200133032BF4D100250846A8
:10C7D00009F006F809F1100008F1100151F82520C0
:10C7E00050F825309B1A02AA42F825300135032D56
:10C7F000F4D1104608F046FC1026012209F11C0B6A
:10C8000008F11C0AD4F8EC3002FA06F1194208D0FB
:10C81000DBF80000DAF800300192C01A08F0C1FC21
:10C82000019A0136132E0BF1040B0AF1040AE9D127
:10C83000002309F1280008F1280131F9026B30F9D1
:10C84000022B921B02AE46F823200133042BF4D1B5
:10C85000002602AB53F82530B600F6B22BB103F137
:10C8600008020F2A61D846F0010615F1FF35F0D213
:10C870000025304608F0DEFBAA460DF1080B06F055
:10C880000303022B63D0032B75D0012B07D1BAF120
:10C89000000F52D19A46DBF800502D01EDB20BF19A
:10C8A000040B06AB5B454FEA9606E8D1BAF1000FE0
:10C8B00002D0284608F0BEFBD4F8EC3013F48055C3
:10C8C00006D00125B9F86420B8F86410521A029213
:10C8D0009A040AD50AAA02EB8501B8F86600B9F8ED
:10C8E00066200135121A41F8202C1E050AD50AAA25
:10C8F00002EB8500D8F86810D9F868200135521A83
:10C9000040F8202C18044AD50AAB03EB8502B8F88E
:10C910006C10B9F86C3001355B1A42F8203C012DDF
:10C9200068D1029808F03DFC3BE08033FF2B94BFB8
:10C9300046F0020646F0030697E7DBF800004FF0EA
:10C94000000A00F00F00284308F074FBA7E7BAF1D3
:10C95000000F04D19BF8000008F06CFB9FE7DBF8A8
:10C960000000C0F30310284308F064FBDBF800501C
:10C970002D01EDB293E7BAF1000F04D19BF801004D
:10C9800008F058FBE6E7DBF80000C0F3033028436B
:10C9900008F050FBDBF80000C0F30710E4E7002DBF
:10C9A000BDD10321302001F0BBFDD4F8EC30D90219
:10C9B00003D50321362001F0B3FDD4F8EC309A0200
:10C9C00003D504213C2001F0ABFD94F87C104420F9
:10C9D00001F0A6FDD4F8EC309B0506D5B9F95E0050
:10C9E000B8F95E30C01A08F0DCFB63682268A36007
:10C9F00062606AE600206B1E02AA52F82320400003
:10CA0000C0B20AB140F0010013F1FF33F4D208F0D4
:10CA100011FB002602AB53F8260008B108F0C1FB59
:10CA20000136AE42F6DBBCE7F02400202DE9F74FDB
:10CA3000A3EB020B16460E9B0D9A002914BF062588
:10CA400004259B1A01934F4B0446D3F8782289465C
:10CA50000132984629D1D3F87422954240F28F8052
:10CA6000DFF834A15AF8220009F092FA0B3008F0EE
:10CA700013FA074618B1012003B0BDE8F08FD8F8CB
:10CA8000741241485AF82120032994BF214649468F
:10CA9000FFF737FC3D4988F87C720A68101AD8F80D
:10CAA000782208600132C8F87822DFF8E090D8F8E0
:10CAB00078420C9B9C421BDB13D1012008F0ECF95F
:10CAC00078B932490A200A68013A0A6008F0B2FAD5
:10CAD000D8F874220132C8F874224FF0FF32C8F837
:10CAE0007822D8F87402854294BF00200120C3E761
:10CAF0000D9B53B1019B04FB03F20D9B995C01223A
:10CB00008A40D8F8EC100A4228D004FB0BF4D8F87D
:10CB10007422371942BB305909F03AFA00F1050A7C
:10CB2000504608F0B9F90028A5D1D9F8000098F8C6
:10CB30007C22A0EB0A00C9F80000C2B12C2008F04A
:10CB400079FAD8F87422B2B9305908F009FA97F98D
:10CB500004104B1C02D00E48FFF7D3FBD8F8782204
:10CB60000132C8F87822A2E74FF0030AD8E7012281
:10CB700088F87C22E5E7174439790648ECE700207D
:10CB80007AE700BF8822002027CC0108D03A002095
:10CB900036CC010881CF0108DCA9010810B50C4C86
:10CBA00094F8E8200B2A0BD8012340F603019340A8
:10CBB00019400CD113F4C06F02D0FF20FFF792FC94
:10CBC000044B1B68C4F878320B2384F8E83010BD9E
:10CBD00088220020901B00202D2343702E23C37039
:10CBE0002F2343717047074B984209BF064A4FF005
:10CBF000FF30538B013301BF9BB25383508B80B204
:10CC0000704700BF00380040740C002070B501244C
:10CC1000B0FBF4F58D4202D21CB91C7070BD4C43C0
:10CC2000F6E7B0FBF4F6092E0BDD002A14BF37251A
:10CC30005725354404FB160003F8015BB4FBF1F4FF
:10CC4000EAE73025F5E703685A1C0260197070475F
:10CC5000002B2DE9F04106460F46144614BF4FF055
:10CC600030084FF02008069B13F8012B3AB92546EF
:10CC7000002D0FDC24EAE47404E0013CF4E7002C0E
:10CC8000FBDC0024069D641B281915F8011B31B933
:10CC9000BDE8F08141463046B847013DE8E73046FF
:10CCA000B847F1E770B50446A56808462B1D013565
:10CCB00044F82310E168A56009F026FE6668E0608C
:10CCC000B54204BF0023A360A368043354F82310C3
:10CCD00009F018FE0546E0602068864207DB304612
:10CCE00009F0C6FE0146284609F0CAFF70BD0130B2
:10CCF000206009F0BDFE0146284609F0C1FF4FF053
:10CD00007E5109F001FE70BDF8B50E46044601687B
:10CD1000304609F001FF616A09F0F6FD61680546D9
:10CD2000304609F0F9FEA16A09F0EEFDE168074618
:10CD3000284609F0F1FE0146384609F0E3FDA168F6
:10CD40006062304609F0E8FE21690646284609F08F
:10CD5000E3FE0146304609F0D5FDA0622846F8BD45
:10CD60002DE9F0410E46044601684769C569304621
:10CD700009F0D2FE61688046384609F0CDFE0146D2
:10CD8000404609F0C1FDA1698046A06809F0C4FED3
:10CD90000146404609F0B8FDE1688046284609F0A2
:10CDA000BBFE0146404609F0ADFD216A8046206980
:10CDB00009F0B2FE0146404609F0A4FDA761666194
:10CDC0002562E061BDE8F08100232A220360427001
:10CDD0002B22C270012243604271C3717047024B23
:10CDE000186804F05CBD00BFA83300202DE9F041B5
:10CDF00001270B4DDFF82C802C686A6914400CB9B0
:10CE0000BDE8F081B4FA84F3C3F11F0358F823009E
:10CE100007FA03F60368984724EA06046E61EEE712
:10CE200000040140F80A002041F4807191FAA1F257
:10CE30000029B2FA82F208BF4FF0FF320388013AAC
:10CE400023F040031B041B0C038003889BB223F0D8
:10CE5000380343EAC2039BB2038003889BB243F0CA
:10CE6000400303807047F8B584894FF6FF764FF48E
:10CE70007A740BB90120F8BD92B115780132078997
:10CE8000BF070FD54FF47A74ADB285810589ED07E0
:10CE900012D58589ADB209B10D700131013BE8E7CA
:10CEA000FF25ECE7013CA4B2B442E8D1FFF79BFEBA
:10CEB000003018BF0120F8BD013CA4B2B442E5D156
:10CEC000F4E708B540F2E9330289920708D540F249
:10CED000E93389B281810289D20709D5808905E0C9
:10CEE000013B9BB2002BEFD1FFF77DFEC0B208BD26
:10CEF000013B9BB2002BEED1F6E7F8B504460F4696
:10CF000016461D46406804F085FD47F08001206804
:10CF1000FFF7D7FF3346002229462068FFF7A3FF1B
:10CF2000606804F07CFD0120F8BD70B504460E4633
:10CF30001546406804F06EFD31462068FFF7C1FFDA
:10CF400029462068FFF7BDFF606804F068FD0120F6
:10CF500070BD2DE9F74F254C254E264F54F8033C64
:10CF60000093002B3AD02422A1464FF0000814F978
:10CF700007BC002102FB0B6528460DF088F817F866
:10CF80000B3007EB0B0292F802A0019319F8010F86
:10CF9000019B984203D1184604F0B2FCA86099F8AE
:10CFA0000300504503D1504604F0AAFCE86008F1A4
:10CFB0000108B8F1030FE9D1242101FB0BF172182C
:10CFC000906858B1D06848B1009BE01F536007EBF0
:10CFD0000B03705019799B7911745374064B1434F8
:10CFE0009C42BBD103B0BDE8F08F00BF3BAA010853
:10CFF000703B00204825002063AA010810B5427A42
:10D00000044632B1036800F10A01406898470023E2
:10D01000637210BD2DE9F341056906460F46002DE8
:10D020003BD1D0F80080C8F3090373B300234FF459
:10D030000050D6F800800193FEF78EF8042821D125
:10D040002A4C4FF40050236943F001032361BBB223
:10D05000A8F80030FEF780F804283CD108F102035C
:10D060000193019B3F0C1F804FF40050FEF774F8B2
:10D070002369042823F001034FEAC3434FEAD34353
:10D0800023612FD06FF0010507E04FF43020FEF749
:10D0900063F8042805D04FF0FF35284602B0BDE8FC
:10D0A000F081124C4FF43020236943F002032361D6
:10D0B000C4F81480236943F040032361FEF74CF861
:10D0C0002369042823F002034FEAC3434FEAD34302
:10D0D0002361ABD0DFE7236923F00103DB04DB0C22
:10D0E0002361CFE7336804333360D6E70020024082
:10D0F000F8B504460D4600278E18B54201D12069C7
:10D10000F8BDE368591CE16015F8012B234404299C
:10D110001A72F2D1A1682046FFF77CFFE760206118
:10D12000EBE770B50D46064644880021C4F30B04B6
:10D13000224628460CF0ABFF33690A4A934209D3D2
:10D14000094A934206D222462846BDE87040194655
:10D150000AF06CBB23B121462846BDE87040184751
:10D1600070BD00BFFCE5010896E60108064B0749C3
:10D170008B4202D30023184670471A88C2F30B0271
:10D180009042F8D01433F3E750E20108FCE50108BF
:10D19000024A136823EA00001060704768180020F4
:10D1A0002DE9F84302780346202A00F10100F9D066
:10D1B000092AF7D02D2A4BD10346444D1C460026A0
:10D1C000DFF80C81234614F8012BA2F13007F9B2E5
:10D1D000092943D92E2A09D127463D4CA0463B4672
:10D1E00017F8010B3038C2B2092A44D91A7802F074
:10D1F000DF02452A63D15A782D2A4CD10127023308
:10D2000000240A20013B13F8012F303AD1B209293A
:10D2100047D9B4F59A7F28BF4FF49A744FF07E50E7
:10D22000A046DFF8B090B8F1070F3DD8DFF8A08036
:10D2300004F00704002C3DD1002F42D001463046B7
:10D2400009F01EFD0146284609F066FCBDE8F8839A
:10D250002B2A08BF03464FF07E55AFE741463046C4
:10D2600009F05AFC0646384609F002FC314609F03E
:10D270004BFB0646A6E709F0FBFB214609F000FD43
:10D280000146304609F040FB41460646204609F07B
:10D2900043FC0446A3E72B2A14BF013302330027C3
:10D2A000AEE700FB0424AEE7494609F035FCA8F1DF
:10D2B0000808B8E7414609F02FFC013CBAE74FF0F7
:10D2C0007E500146304609F027FCBBE7000080BFD6
:10D2D0000000204120BCBE4C002330B50C4687B076
:10D2E0000021054600930193029309F0D1FD2949DD
:10D2F00000283DD0284609F007FB274909F00CFC1F
:10D3000009F0E6FD054680EAE07003A9A0EBE570B0
:10D3100008F018FA002DACBF20232D2303A88DF8A8
:10D32000003008F035FE012826D130238DF8013079
:10D330008DF802308DF8033003A968460CF0CDFE5D
:10D34000684608F025FE0338C5B22A4669462046DD
:10D350000CF019FF00231149635520460CF0BDFE67
:10D360000DEB050120460CF0B8FE204607B030BD9D
:10D37000284609F0C7FAC0E7022805D130238DF806
:10D3800001308DF80230D7E7032804BF30238DF831
:10D390000130D1E76F12033A00007A4465CD0108ED
:10D3A00070B50646B6FBF2F40846154614B12046A1
:10D3B000FFF7F6FF05FB1464024B1B5D00F8013B11
:10D3C00070BD00BF55CC0108026810B51146531C52
:10D3D000036011F8024BD31C01605178036093780D
:10D3E0001B0443EA0123111D0160D078234343EA63
:10D3F000006010BD03685A1C02601A4612F8021B36
:10D400000260587841EA0020704738B50446154656
:10D4100000680AF00BFA22682A44226038BD0368CB
:10D420005A1C0260197003685A1C02600A0A1A70BA
:10D4300003685A1C02600A0C1A700368090E5A1C11
:10D4400002601970704703685A1C02601970036803
:10D45000090A5A1C0260197070472DE9F04F824684
:10D460008B4615461C46002789B00DF11408297813
:10D47000002930D0252904D050460135D84701373E
:10D48000F5E76A784FF00009302A12BF0023012324
:10D49000AA780293A2F1300314BFAE1CEE1C092B34
:10D4A0000CD8A2F13003D9B2092918D9A2F161032D
:10D4B000052B1AD8A2F157030A2B10DD6C2A74D160
:10D4C0003278751C642A00F0AB8022D8252A66D0F9
:10D4D00012D8002ACBD1384609B0BDE8F08F0A2215
:10D4E00002FB093916F8012BDBE7A2F14103052BFA
:10D4F000E4D8A2F13703DFE7582A18D0632AB6D15F
:10D500002E4621785046D847251D01372C463546F2
:10D51000ADE7732A37D006D86E2AA8D12E462368E5
:10D5200004341F60F3E7752A65D0782A9FD14346FB
:10D530001021A2F15800424204F104064241206841
:10D5400007E02D2340428DF814300DF11503002221
:10D550000A21FFF75BFB3446CDF80080029B4A4668
:10D5600059465046FFF774FB074480E72D2340429D
:10D570008DF814300DF1150300220A21FFF746FB48
:10D580003546039CE8E72E4623684A4600935946F1
:10D5900000235046FFF75CFB251D0744B6E72E46E7
:10D5A00025215046D8470137B1E7642A31D00AD83F
:10D5B000252AF5D002D8002A8DD0A8E7582A0CD009
:10D5C000632A9ED0A3E7732ADED002D86E2AA6D0A3
:10D5D0009DE7752A14D0782A99D1A2F158014A42C0
:10D5E00004F104054A412068434610212C46FFF708
:10D5F0000DFB3546B0E7261D434600220A219EE773
:10D60000231D0393002243460A212068FFF7FEFAF8
:10D61000B6E72068231D00280393A7DB4346ABE74A
:10D620002068261D00288CDB434690E70FB437B5F1
:10D630000B4906AB0B4853F8042B096800680193AB
:10D64000FFF70BFF0446084D286804F01FF9002877
:10D65000FAD0204603B0BDE8304004B0704700BFA8
:10D66000D80A0020DC0A0020A833002010B541F2BF
:10D6700021040A44914200D110BD11F8013B80EA17
:10D680000320082310F4004F4FEA400018BF604009
:10D69000013B80B2F6D1EDE7F8B51A4D2B789F2B00
:10D6A0002ED16B78BE2B2BD105221749A81C0CF06C
:10D6B00031FD28BB072229464FF6FF70FFF7D6FF42
:10D6C000124FEC1D22884AB1A618BE4218D2052A74
:10D6D00016D92146FFF7CAFF3446F3E72146022256
:10D6E000FFF7C4FF0222A118FFF7C0FF0634084B62
:10D6F000641B1C8041F60F53C31A58425841F8BDB1
:10D700000020F8BD00F8010881BF010800000208F0
:10D710002C16002080EAE073A3EBE0738B4206DB5B
:10D72000002801DD401A704702D0084470470020ED
:10D73000704770B5044609F0CBFB203040284DD827
:10D74000274D284E2946204609F0A2FB002830D15B
:10D75000254D244E2946204609F07CFB00282ED179
:10D760002249204609F094FB00282ED021461C486F
:10D7700009F0C8F804462146204609F0CDF90546CF
:10D780001B4909F0C9F91B4909F0BEF8294609F0FF
:10D79000C3F9194909F0B6F829460646204609F0AA
:10D7A000BBF90146304609F0B7F9214609F0ACF85B
:10D7B00070BD2046314609F0A5F80446C2E7204670
:10D7C000314609F0A1F80446C4E70C49204609F0A7
:10D7D00041FB0028CFD021460348C9E7002070BD97
:10D7E000DB0F4940DB0FC940DB0F49C0DB0FC93FEE
:10D7F00092E741B99730083C15A82A3EDB0FC9BF14
:10D8000070B5044610460E4609F02EF9054630461E
:10D8100009F02EF90146284609F07EF9014606482E
:10D8200009F02EFA0AF068F93C28A8BF3C2001282C
:10D83000B8BF0120606070BD0024744938B504464B
:10D840000B4D204604F0CBF930B10A4B0A48597809
:10D85000BDE8384004F0D4BA204609F0BFFF0228E2
:10D8600004D8C0B208F002FB2C46EAE738BD00BF7E
:10D870000BDD0108081600207ACC010870B50446BB
:10D880000A4E0B4D204604F0AAF930B1074B094867
:10D890001978BDE8704004F0B3BA204609F09EFF45
:10D8A000022802D830702C46ECE770BD0816002024
:10D8B0000BDD01087ECC01082DE9F743074604F093
:10D8C0008EF9044620B104F0BFFC03B0BDE8F0833C
:10D8D000384601AA2E4909F0DDFF2E4FDFF8CC8033
:10D8E000DFF8CC9070B9022CEDD1A6F57A73B3F5C0
:10D8F0007A7F2DD94FF4FA624FF47A71264804F0FA
:10D900008CFAE2E744B1012C1ED001AA2049002084
:10D91000013409F0BFFFE5E709F060FF051E0DDBEC
:10D920003B789D4204DA29464846FFF77FFEECE744
:10D93000FF2D03D14046FFF779FEE6E73978174817
:10D940000139FFF773FEC0E709F048FF0646DCE740
:10D95000FF2D0AD104460F4B114F1D78AC4210DB4E
:10D960003146104804F04CFAAFE7304609F07CF835
:10D970000B4B324643F8250029460B4804F040FA89
:10D98000A3E7304609F070F847F824000134E5E7D2
:10D9900005CE01080423002045D10108B1CC0108BF
:10D9A00058250020E7CC0108DACC01089CCC0108FE
:10D9B00089CC01082DE9F0470546204FDFF8848027
:10D9C000DFF87C90DFF894A0284608F0E1FA0646DC
:10D9D00050B91B4B1B4A1B781B48013B52F82310C4
:10D9E000BDE8F04704F00CBA0246394628460CF070
:10D9F00091FB40B1002458F82410A1B91348BDE8A8
:10DA0000F04704F01BBC124804F06CF9114C124DA5
:10DA100054F8041F19B1284604F03BF9F8E7BDE8B3
:10DA2000F04704F0D6B9324628460CF073FB0134B7
:10DA30000028E0D189F800405546C5E766C60108D0
:10DA40002C25002034A70108F6CC0108FBC60108EC
:10DA500000CD010830A701081DCD01080BDD01082C
:10DA60002DE9F74F824608F093FA474D04462F6898
:10DA7000E8B9464804F00DF90125454EDFF8348138
:10DA800005FA04F33B4206D00C2303FB0463404633
:10DA9000996804F0FEF80134132CF1D117B93D4810
:10DAA00004F020F903B0BDE8F04F04F092B902464B
:10DAB000394950460CF02EFBDFF8D490064668B981
:10DAC000364804F00FF9364D09EB060399682846ED
:10DAD0000C3604F0DEF8FC2EF6D1E3E79AF80030BD
:10DAE0004FF000082D2B0CBF4FF0010B4FF0000B37
:10DAF0004FF00C0304BF0AF1010A04F1FF3403FBE9
:10DB00000892966850462246314601930CF002FB7B
:10DB1000019B70BBBBF1000F19D0B8F1130F0BD1F3
:10DB2000204B2B60204804F0DDF831461C4803B040
:10DB3000BDE8F04F04F064B9B8F1140F01D16B687F
:10DB4000EFE7012303FA08F31F432F60EAE7B8F178
:10DB5000130F03D1C5F800B01448E4E7B8F1140F6F
:10DB60001DBF012303FA08F39F436F6018BF2F60A6
:10DB7000F2E708F10108B8F1150FC0D10C4803B065
:10DB8000BDE8F04F04F05ABB741800200BCD01081B
:10DB90001CA8010815CD010866C6010800CD0108C2
:10DBA0001DCD0108FFFF070021CD01082ACD010886
:10DBB000FBC601081CCD010870B5134C054613487F
:10DBC00004F090F8206AFFF719FA606AFAF79EFDF0
:10DBD0000F4B1820197800231E4628348B420BDB8C
:10DBE00040F2DC5003F0E4FD0A4B0B4A15B10B4840
:10DBF0000B490860DA6070BD00FB03F2125902B1F4
:10DC000016800133EAE700BF5825002032CD010815
:10DC10000423002000ED00E00400FA05EFBEADDEB5
:10DC2000F04F002010B50C4C206AFFF7E7F90023F5
:10DC3000D4F8702184F8E830C4F8683184F86C3185
:10DC400044F823200133082BFAD10020FFF7B4FF5A
:10DC50000023236210BD00BF5825002008B501F045
:10DC600085FC01F085F9BDE808400020A4E708B56F
:10DC700001F07EF9BDE8084000209DE701209BE708
:10DC80002DE9FF41074608F083F908284AD100250D
:10DC900001AE7C5D09F0AAFD2044437803F0030344
:10DCA000022B08BF203CAC550135082DF1D10025D1
:10DCB000DFF87C808DF80C507C5D09F097FD2044E6
:10DCC0004378404603F00303022B08BF203C745501
:10DCD000E4B221460CF010FA28B101352146701942
:10DCE0000CF00AFA20B104F0AFFA04B0BDE8F081FC
:10DCF000082DE1D10D49304602F0F0FB00230B4C1A
:10DD00000B481A5D04A90A44195C0133082B02F878
:10DD10000C1CF6D1002301A906488DF80C3004F044
:10DD20006FF8E2E70028E9D0DDE700BF38360020D1
:10DD3000ECAB010877C701082DE9F84F054608F05C
:10DD400027F9364F0446D7F80090B0B9344803F0AD
:10DD5000C9FF0126334D344F55F8241049B106FA56
:10DD600004F313EA090F02D0384603F092FF01349E
:10DD7000F2E7BDE8F84F04F02CB802462B492846DC
:10DD80000CF0C8F978B92A4803F0ACFF294C2A4DA9
:10DD900054F8041F0029ECD00B78002BF8D028464B
:10DDA00003F077FFF4E72B7800262D2B0CBF4FF004
:10DDB000010A4FF0000ADFF86CB004BF013504F12E
:10DDC000FF345BF82680B8F1000F04D11B48BDE892
:10DDD000F84F04F033BA2246414628460CF09AF92F
:10DDE000D0B90120B040020601D51548EFE7830500
:10DDF000FBD4BAF1000F0AD0FFF7CAF9114803F0BB
:10DE000071FF4146BDE8F84F0B4803F0F9BF40EA07
:10DE1000090038600C48F2E70136D2E768180020A4
:10DE20003ECD0108A0A7010848CD010866C601083B
:10DE300000CD01089CA701081DCD0108FBC6010803
:10DE40004CCD010821CD01082ACD010870B5054649
:10DE500008F09EF8044690B1112200210F480CF002
:10DE600016F922460E4928460CF07BF938B1102CE1
:10DE70002246294628BF102208480CF084F9BDE844
:10DE80007040084B012013F8042F002A044A06BFF3
:10DE9000012113460021044A04F08AB80C16002020
:10DEA00008C701080816002033C7010808B50D4847
:10DEB00004F0C4F90C4B186AFFF7A0F8FCF734FF24
:10DEC000FCF716FE48B1132008F000F803F081FFBC
:10DED000BDE80840054804F0B1B9642003F073FCC4
:10DEE000EEE700BF58CD01085825002061CD01089C
:10DEF0002DE9FF410A480488856846888788D0F85C
:10DF00000C80FCF7D5FD8DE88001029033462A464F
:10DF10002146044803F074FF04B0BDE8F08100BF5F
:10DF20003804002067CD0108F0B585B0054603F040
:10DF300056FE002838D104462B78002B3CD1062C05
:10DF400042D1BDF904309AB2072A3DD840F2DC54E0
:10DF5000BDF90610A1F2EE2292B2A24234D8BDF968
:10DF60000820A2F2EE2080B2A0422DD8BDF90A000E
:10DF7000814229DC824227DB914225DCBDF90C502D
:10DF800005F16404A4B2C82C1ED8BDF90E40112CB2
:10DF90001ADC0C27194E07FB03639980DA8018817D
:10DFA0009D72DC7205B0F0BD00220120134905B05E
:10DFB000BDE8F04002F0ACBC2D2B03D0A3F1300241
:10DFC000092A16D8052C04DD05B0BDE8F04004F0A0
:10DFD0003BB9284609F002FC04AB661C03EB440481
:10DFE00024F80C0C15F8013F303B092BFAD93446C4
:10DFF000A2E7202BE8D101352646F8E7F82B0020D0
:10E00000022810B50C460CD807F030FF0548FFF782
:10E0100015FC03F0DEFE2146BDE81040082003F0A9
:10E0200041BF10BD0BDD0108022810B50C460CD80D
:10E0300000F088FF0548FFF721FC03F0CAFE2146E7
:10E04000BDE81040042003F02DBF10BD0BDD01081A
:10E0500070B5044608460E4607F09AFF3146024660
:10E0600020460CF057F808B1002070BD09F0BEFB47
:10E070000546304607F08CFF235C1D446A78120782
:10E0800001D4002BF0D10130204470BD2DE9F04FB8
:10E09000824691460E46154600278FB0337896F992
:10E0A0000280089373780993F3780A9396F9043001
:10E0B0000B9396F905300C93B3790D93B8F1000FDB
:10E0C00004D10FB0BDE8F04F03F083BEB9F1000FEB
:10E0D0004CD02B78089C6A789C4295F90210E8781D
:10E0E00095F904E095F905C095F806B03CD1099C76
:10E0F000944239D1884537D10A9C844234D10B9C53
:10E10000744531D10C9C64452ED10D9C5C4514BFE7
:10E11000002401240390029101920093CDF818B0DD
:10E12000CDF814C0CDF810E03B46114A21465046C8
:10E1300003F028FF0D9BCDF8088006930C9B0C4A3A
:10E1400005930B9B214604930A9B50460393099B1E
:10E1500007360193089B073500933B46013703F0D0
:10E1600027FF102F9AD1ACE70024D3E74C46E1E714
:10E17000C2CD01082DE9F0478AB0054607F008FF37
:10E18000024630B995490120FFF780FF0AB0BDE88B
:10E19000F0870522924928460BF0BCFF044660B97F
:10E1A000702201468D480BF072FF204622468D4BAF
:10E1B000C2500C306028FBD1E8E704228A49284687
:10E1C0000BF0A8FF0446002841D1284603F00FFDBC
:10E1D00006460028DAD007F0DBFE0746DFF830827B
:10E1E00058F824501DB9814804F028F8CEE73A4683
:10E1F000294630460BF08EFF01340028F0D1774BD2
:10E200000246194603F170069A719A705A7003F823
:10E21000072BB342F8D1764B13F8347003EBC404E8
:10E22000B84205DB2946734803F0EAFD724886E0F0
:10E230006368C0EBC0021344D3F800E08E1841F8C5
:10E2400002E09A880130B2809B79B371E8E7072237
:10E250006A4928460BF05EFF0446002875D120214C
:10E2600028460BF049FF064607F092FE054680BBA4
:10E27000634803F00EFD2C46624D214628460134CA
:10E2800003F007FD0E2CF8D103F0A3FD0024DFF806
:10E290008491544FDFF880810C262146484603F0D4
:10E2A000F8FC002506FB0476DFF870A10123326834
:10E2B000AB40134214BF414651465348013503F069
:10E2C000E8FC0E2DF2D1013403F083FD082CE3D1DC
:10E2D0005CE7304601AA4D4909F0DCFA4B4E02AD2D
:10E2E00000283DD0022C15D1029A072A2AD803997A
:10E2F0000D2927D80378722B17D06E2B22D10C232F
:10E3000053430122374802FA01F1C25822EA0102BE
:10E31000C25013E009F062FA01AA45F82400314620
:10E32000002009F0B7FA0134DAE70C230120534347
:10E330002C4C00FA01F1E0580843E0502F48FFF759
:10E3400019FF23E703F080FFF8E7284601AA2F49C9
:10E3500009F0A0FA00242D4E02AD78B1082C02D1AC
:10E3600003F072FF12E709F039FA01AA45F8240018
:10E370003146002009F08EFA0134EEE7082CEFD187
:10E38000029B0F2BECD8DDF80CC0BCF1070FE7D8CF
:10E39000049F0D2FE4D8059E06F16402C82ADFD839
:10E3A000069DFF2DDCD807986428D9D808996429E0
:10E3B000D6D88842D4DA099C032CD1D8DFF81CE0E7
:10E3C000C3EBC3020EEB02030EF802C05F709E7037
:10E3D000DD70187159719C7128E700BF862B0020F1
:10E3E000DFCD0108F82B0020E5CD0108FBC60108B0
:10E3F0005CAA0108EACD01080BDD0108F4CD010893
:10E400001FCD0108FCCD010801CE010805CE010891
:10E4100034A7010881CF0108DFCE0108BEC1010881
:10E4200010B50E22002104460BF031FE0A23238092
:10E4300000236381A381A380E380238110BD03783F
:10E440008B4286BF024B33F811000020704700BF9B
:10E45000CC260020034B187E10B1002201201A7632
:10E46000704700BFCC2600207FB5284E284932884F
:10E47000284CB2F5805F284B284A096826D31B78C0
:10E48000C4F8191092F8202094F82110E37794F83A
:10E4900022306177A27784F82030532006F0CAFD3D
:10E4A000D4F81900FDF7C2FF607FFDF7BFFFA37F1F
:10E4B00001A80193E37F029394F82030039306F0C0
:10E4C000E1FD00230120338004B070BD1B7892F879
:10E4D0002020019194F821108DF80A3004F11905DB
:10E4E00094F822308DF808108DF80920294608226A
:10E4F00001A88DF80B300BF0A1FD0028E4D001AB92
:10E5000003CBC4F81900C4F81D10C6E7642300202B
:10E51000F4240020CC260020A53500201036002051
:10E520002DE9F041884600240C4B93E8E0000544B7
:10E5300006440744444501DBBDE8F08137F9142067
:10E5400036F9143035F914001344022293FBF2F328
:10E55000C01A06F026FE0134ECE700BF8822002036
:10E560002DE9F04F102285B00021B3480BF08FFD4C
:10E5700000263D23B14C232084F84D30E66103F0A2
:10E5800022F904AB03F80B6D0122752104F1180088
:10E59000FAF74AFC04F11805002841D0A84B0122E3
:10E5A0002365A84B314663654323284684F85C30D5
:10E5B0000DF10603FAF738FC9DF8063003F07E03F0
:10E5C0008DF80630002840F0FD809DF8053003F0FE
:10E5D0007E03682B8DF8053040F019810622022356
:10E5E000114684F84B30266D02AB9748B0479DF832
:10E5F0000D309DF80B209B00520002F0020203F048
:10E60000040313439DF8092002F00102134300F0B4
:10E61000EF80012B40F0E080002384F84C3039E09B
:10E620008A4BE069A36110B92C2003F069F9884E88
:10E63000E06196F8232082B910B11C23C271837166
:10E64000132103F083F9E06903F0E9F90221A069DD
:10E65000FEF7EAFB012386F82330E06903F0DAF9DC
:10E66000F521A069FEF72DFC0123002202A9A06973
:10E67000FEF7F9FBE06903F0D2F99DF80830712B41
:10E6800000F0918000F28780122B00F09780702BB1
:10E6900000F03D82002384F84A3094F84B30022B7E
:10E6A00040F039826B4A22606B4A62606B4AE260DA
:10E6B0006B4A2262012284F84A20073B052B88BF5F
:10E6C0000023684E684F326897F8039042F00102C9
:10E6D000326088BFFB71B9F1000F03D0B9F1070FA9
:10E6E00040F0F280FB79B878002B00F0E78003233C
:10E6F000DFF890A184F84730431E84F8483008F0D2
:10E70000B7F9514608F008FA08F008FCDFF828814C
:10E710002368C8F8000084F84690484898473B783A
:10E720000BB184F84A304FF000094FF0010BCA4694
:10E730004E4C06F0BDFE442200212046D8F8007061
:10E740000BF0A5FC95E80300494D04F1080304F122
:10E75000200E83E8030095E80F008EE80F0035F8DF
:10E76000053C3B4DA4F81B3095F8278084F81A909F
:10E77000B8F10C0F00F2E481DFE818F0B000E2011C
:10E78000B000DC00EB000001DC00120112011201FC
:10E79000120112011201AC2B00F0BB81AF2B0FD084
:10E7A000732B7FF477AF062384F84B30432384F830
:10E7B0005C30304B2365304B63656BE70823F3E730
:10E7C0000923F1E7682B7FF400AF012384F84B3075
:10E7D0001D2384F85C305DE7022B01D101231CE787
:10E7E00003F00303032BF9D0032003F0AAF951E748
:10E7F0000DF10703266D01220C211348B0479DF847
:10E80000073013F00F03EFD0042BE7D104E7702B90
:10E8100004BF042384F84B303CE7184A84F84A309C
:10E8200022600D4A04236260154AA2600B4AE2602E
:10E830000B4A226241E700BF20410020CC3B002070
:10E84000298E0008B18D0008E43B0020003800400C
:10E85000CC26002029A60008458C0008358C00082D
:10E8600090C1793D28250020BA3B0020B822002025
:10E870001C3C0020FBCE00082BCF00080D8D0008AB
:10E880001BA500080000FC41B84A2260B84A62603B
:10E89000B84A063BDBB2E260B74A032B226296BF5E
:10E8A000B64A0723D35C012284F84A20002B00F0EB
:10E8B000408102E7B24A2260B24AE8E70223DFF869
:10E8C00014A384F8473017E70023DFF80CA384F87B
:10E8D0004730012010E74FF0000847E704AB03F88A
:10E8E00008AD01220021532006F0FAFC10B39DF878
:10E8F0000830E52B1ED1A44B85F832A02360A34B32
:10E9000063600423A3763368A14843F002033360B5
:10E910004FF480732382236898474FF47A732363FC
:10E92000AB8E002B4CD195F82630002B00F00C81DB
:10E93000A37609E1E37E022B0BD1964B2360964B25
:10E940006360237F002B0CBF6F236E23237601238C
:10E95000D8E704AB03F8089D01220D211C2006F026
:10E96000BFFC58B19DF808302A2B01D01A2B05D1D5
:10E970008A4B23608A4B63600223C3E704AB03F82E
:10E98000089D01220021182006F0AAFC40B19DF844
:10E990000830FB2B04D1834B2360834B6360D6E7A5
:10E9A000E37E042B40F0C980804B23607A4BF5E76F
:10E9B0000BFA03F313F4587F00F0C2807C4BF4E7AA
:10E9C0000027DFF81882A88E08F04EF8226B014667
:10E9D00008EB07002C37FBF77FFF842FF3D1A2E76A
:10E9E0000A2002F0F0FE0DF107030122A02177209A
:10E9F00006F076FC0446002852D0002701221E2192
:10EA0000772006F01DFC4FF42F6002F0D1FEB846CF
:10EA1000DFF8CC91A7F1600102AB0222C9B27720E6
:10EA20008DF808808DF8098006F05AFC9DF80820C2
:10EA30009DF8093043EA022327F809300237102FE6
:10EA4000E8D100231946B5F8D22002F00F0702F4EE
:10EA50007F42A5F8D22021F001002844B0F8C4007C
:10EA6000002818BF002411F0010F1ABFC0B24340A4
:10EA700083EA1023082013F4004F18BF83F4C05317
:10EA800001384FEA4303F6D101311029E3D13A436B
:10EA9000A5F8D22024B9C3F303339F4200F0A2802B
:10EAA00095F8D44074BB142002F08DFE414B012236
:10EAB000D021762006F014FC95F8D530582B01D0E3
:10EAC000012037E03C4B18228821762006F008FC14
:10EAD0003122F421762006F0B3FB0123374A85F872
:10EAE000D430374B9A60374A1C805A6045F6D812AA
:10EAF0005A80354ADA60354A1A61354A5A6101E06E
:10EB0000012BDDD0336843F004033360D8E70523DD
:10EB10004AE6072348E6012B3FF47FAE042B3FF47F
:10EB2000B3AE092B05D801229A4012F4587F7FF426
:10EB3000C1AE002005B0BDE8F08F092B7FF638AFDD
:10EB4000B8F1010F3FF6C7AE95F8BC30042BD7D80B
:10EB500001A252F823F000BFE1E90008C1EA000871
:10EB6000E1E90008E1E90008A1EA000899A6000827
:10EB7000458C0008358C000890C1793DC7AB010871
:10EB800057A700085F8D0008D78D0008CF8E0008BA
:10EB9000B822002003A50008898C0008958F000882
:10EBA0002F8E0008B78D0008898E0008F3A4000896
:10EBB000FBA40008A1270020A4270020F1A400083E
:10EBC0003423002097A1000889A50008DDA50008CE
:10EBD00039A300080000FA4200007A44042700200C
:10EBE0009027002042F21072064B1A805A80064A83
:10EBF0005A60064A9A60064ADA60064A1A61064A6C
:10EC00007CE700BF342300207FA50008CDA50008C5
:10EC100075A50008BBA5000899A10008064B1A6855
:10EC20004FF47A73B3FBF2F3C3EB431203EB8203AB
:10EC3000DB000380704700BF2041002002392DE92E
:10EC4000F843426804460368806806290DD8DFE867
:10EC500001F0040873767B7E810022605B42636072
:10EC600003E05B425242236062603C4B1B78002B06
:10EC700060D1206807F0FCFE8046606807F0F8FE6F
:10EC80000746A06807F0F4FE354D0646D5F8F410A7
:10EC9000404607F041FFD5F800118146384607F09D
:10ECA0003BFF0146484607F02FFED5F80C11814680
:10ECB000304607F031FF0146484607F025FE08F0D0
:10ECC0001BFFD5F8F8102060404607F025FFD5F867
:10ECD00004118146384607F01FFF0146484607F0F9
:10ECE00013FED5F810118146304607F015FF014696
:10ECF000484607F009FE08F0FFFED5F8FC106060FA
:10ED0000404607F009FFD5F808118046384607F05D
:10ED100003FF0146404607F0F7FDD5F814110746FA
:10ED2000304607F0F9FE0146384607F0EDFD08F0E1
:10ED3000E3FEA060BDE8F883524222608FE75B42A9
:10ED400023604042A06090E722606360F9E752428E
:10ED50006260F6E7524222605B42F6E71D04002043
:10ED6000CC26002003680A7A591C01601A7070478B
:10ED700038B50546064C206800B938BD4368EB1A23
:10ED8000002BFADB8368236003689847F3E700BF32
:10ED9000602A002000231A4630B5084C0372191966
:10EDA0008D79AD0742BF097981540132D02B03D050
:10EDB000072A03F11003F2DD30BD00BF90BE010849
:10EDC000002210B5064C04EB02118B7913F00103FD
:10EDD00002D00B79037010BD01320E2AF3D1F9E78E
:10EDE00090BE010814220123427015220370837122
:10EDF000C27103712122837011234271C370704765
:10EE000038B54D680446284607F0C2F82946024640
:10EE10002046FEF7FAFA23685A1C22603B221A7039
:10EE200038BD08B50B4B1820197800231D460A4C35
:10EE30008B4207DB40F2DC5002F0BAFC074A084B79
:10EE4000DA60FEE700FB03F2125902B115800133CC
:10EE5000EEE700BF04230020802500200400FA050F
:10EE600000ED00E030B500220C25074905FB02F457
:10EE70006318645C844201D1184630BD0132242AF3
:10EE8000F4D1002030BD00BF24AF01082DE9F84FB8
:10EE900000248046914625464E01DFF834A006F155
:10EEA0002007214650465FFA84FBFBF75AFD50B11C
:10EEB000AE4207D8AF4205D95846FFF7D3FF014607
:10EEC0004046C84701350134242CEAD1BDE8F88F0B
:10EED000CC0C002080B50121022002F0DBFD144B98
:10EEE0001B7803F00503052B12D1124B0024186880
:10EEF00007F0EEFF104B114F1D7806B2AC4210DB4D
:10EF00000F4B1B780BB103F055FD322002F05BFC78
:10EF10000021012002F0BEFD0021084602F0BAFDEA
:10EF2000FEE7304607F0A4FD47F824000134E5E78A
:10EF3000E50A0020C8260020042300200823002022
:10EF400058120020022828BF0220064B064A1870DB
:10EF50004A2303FB0023054A0130C0B21360F9F7CE
:10EF600051BE00BF08160020AA3200202025002034
:10EF70002DE9F04F8DB001F055FB0326DFF84C91E1
:10EF80004D4FA7EB0907182200210DEB02000BF0F3
:10EF90007EF84A4B4A4ACDF8189007975A6002F11A
:10EFA00088325A6001228DF82C203422DA60454BD9
:10EFB00004A918689A889B790490ADF8142006A8D3
:10EFC00007228DF81630FEF793F8072204A94FF6B2
:10EFD000FF70FEF74BFB4FF0000A80463A4CDFF81B
:10EFE000F0B05C4536D300250CAC24F82C5D022231
:10EFF000214606A8FEF77CF8022221464046FEF78D
:10F0000035FB40BAC0430222ADF8080002A906A8A9
:10F01000FEF76EF8099860B108ABC0F1040229460A
:10F0200018440BF034F8089906A8FDF7F3FF09958A
:10F030000A909DF82C300A9A23B120490B6943F0BD
:10F0400080030B61013E2DD0002A9CD1FEF724FBEA
:10F0500050B32CE0658806A8C5F30B05AA1DADF8D2
:10F06000082022888DF80DA0C2F30B01120BADF819
:10F070000A108DF80C2002A90622FEF739F80622A4
:10F0800002A94046FEF7F2FA804661682A4606A8C1
:10F09000FEF72EF8616840462A46FEF7E7FA143478
:10F0A00080469EE7002AD1D0052002F04AFD01F0FB
:10F0B000A1FA0DB0BDE8F08F000002080020024068
:10F0C00023016745CCAB010850E2010800F80108B4
:10F0D000FCE501082DE9F843344B354D5A899989EF
:10F0E000914228BF0022198A28BF5A81DA899142A9
:10F0F00024BF0022DA81DA78002A50D0072A4ED0C5
:10F1000001222A709A7000222A4CDA71D9799A78F1
:10F11000002946D0102A38BF1022274C9A709878C0
:10F1200007F0A6FC214607F0F7FC814695F8008021
:10F13000224C404607F09CFC494607F0EDFCA678BF
:10F140000146022E97BF1E4B1B4F03EB86039F68A1
:10F15000384607F09DFE80B14946384607F090FDDD
:10F1600007F0B6FE1028A8BF10200128B8BF012064
:10F17000C0B2404528BF4046287023796BB1013E9C
:10F18000032E0AD839464FF07E5007F079FD08F07B
:10F19000B3FC2388984238BF2080BDE8F883094C2F
:10F1A000B4E7032A38BF03229A70B8E7BA3B0020BD
:10F1B000582C00206F12833A6F12033878230020F6
:10F1C000CCAB01086F1203392DE9F84301F02AFA9C
:10F1D000AC4CAD4FDFF84883BC422DD2AB4D00E0C4
:10F1E00015462E88002E00F0AA81AA19424580F00B
:10F1F000A681052E40F2A38123886988C3F30B03FF
:10F200009942EDD16B799B07EAD16168204695F868
:10F210000490FDF786FF2388B9EB133F0AD163887A
:10F22000B21FC3F30B039A42A8BF1A46A91D606818
:10F2300008F0FCFA1434CFE7954B5A78022A84BFC1
:10F2400000225A705A78022A05D80C20914900FBF6
:10F25000021291490A601A78904E022A84BF002255
:10F260001A701878022806D84A228D4B02FB00300B
:10F27000306001F033FA8B4A1178A1F11703022BA9
:10F2800012D9894BC80013F8314024B11C186468A6
:10F290000CB91724147003445B782BB1834B13F81B
:10F2A00031300BB918231370814B9A78042A40F03F
:10F2B000DD809A8AB2F57A7F02D24FF47A729A820E
:10F2C0007C4C7D4A23681A4012B943F00103236045
:10F2D0002368DD0702D57948FDF75AFF23685804F3
:10F2E00002D57748FDF754FF2368190702D5754802
:10F2F000FDF74EFF23689A0103D546F20900FDF79A
:10F3000047FF23689B040FD56F48FDF741FF4FF47B
:10F310000040FDF73DFF6D4B40205A79012A04BFA4
:10F3200000225A71FDF734FF336800259A8CD98C7E
:10F33000674F914224BF00229A84FFF7CBFE2C46F0
:10F34000B9464FF0FF08EA5B530803F077339008A3
:10F3500000F03330D31A1B1AD00800F011301B1AFA
:10F3600003EB231303F00F3393FBF8F012F00101CA
:10F37000C0EB002018BF0134A3EB000318BFE4B2B8
:10F38000012B0DDD022B40F0DF8011B112F42F7F35
:10F3900006D109EB050005F04FFB002800F0D480F2
:10F3A0000835202DCFD1013C022C00F2CD80494BF5
:10F3B0001B78012B05D8484BDA78022A04BF0122BA
:10F3C000DA7003F0D1F83022002144480AF05FFEE1
:10F3D000002003F03FF8424B80F0010034681870C1
:10F3E000404B414A1C60414B0024197864234B4335
:10F3F000C83353609460D460146154619461D461E3
:10F4000082F8204082F8214039493A4A3A4D0A6050
:10F410003A4E32F8042C286B3280002840F082806B
:10F42000374D384B28881E8807F022FB364907F0F5
:10F4300073FB364C6060688807F01AFB324907F0AE
:10F440006BFB6B79324A23722B7920606372314BEC
:10F4500030461A6007F00CFB01462F4807F010FCFD
:10F460002E4B1860BDE8F84301F0C4B8002A7FF4C1
:10F4700027AF1A88B2F5F07F84BF4FF4F0721A807C
:10F480001EE700BF50E20108FCE5010807F801088B
:10F490000816002040110020AC2D0020202500205F
:10F4A000AA3200202C25002010AC01085CAA01081B
:10F4B000782300206818002009600002086000021C
:10F4C000092000020160000209400002FE35002010
:10F4D00032410020E40A0020F0260020D014002051
:10F4E000000000200415002010360020B831002054
:10F4F000F8330020F4260020B82200200027002046
:10F50000FA270020B810002017B7D1387431002036
:10F510003661023DA0310020C0C9FB48BC1000206C
:10F52000000002080A4F308807F09EFA2A6B014655
:10F5300038192C34FBF7D0F9842CF4D170E76168CA
:10F540002046FDF7EEFD75E60248F8F739FF2EE795
:10F55000042700203241002008B5FFF709FDFFF71E
:10F5600033FEBDE808400120F9F74CBB38B50E4C1E
:10F570000E4DAC4211D30025FBF700FA0C4C0D4B9D
:10F580000D482570186001F0A9F80C4B0C4A657005
:10F590001A60BDE8384005F0FDBA61682046FDF705
:10F5A000C0FD1434E5E700BF50E20108FCE50108A6
:10F5B0000816002020250020AA320020AC2D0020B3
:10F5C0004011002070B50C2948D8DFE801F007474A
:10F5D00047474847474784474747BE00038C15883D
:10F5E00023F001031B041B0C0384038C8488018B10
:10F5F00023F0020321F073010904090C2943568802
:10F6000015891B0435431B0C2B43674DA4B2A8423C
:10F610009BB20FD005F50065A8420BD005F54065FB
:10F62000A84207D005F58065A84203D005F580659E
:10F63000A8420ED1558923F008032B43958823F067
:10F6400004032B43D689958924F4407435432C4315
:10F65000A4B2D288848001838286038470BD038C27
:10F66000148823F010031B041B0C0384038C85886F
:10F67000018B23F0200321F4E6410904090C41EA3F
:10F680000421568814891B0434431B0C43EA0413D9
:10F69000454CADB2A04289B29BB203D004F50064E0
:10F6A000A04213D1548923F0800343EA04134FF698
:10F6B000BF741C409388D68944EA0313948925F4C7
:10F6C0004065344345EA84059BB2ADB2D28885805B
:10F6D00001830287C1E7038C148823F480731B0421
:10F6E0001B0C0384038C8588818B23F4007321F029
:10F6F00073010904090C2143568814891B043443FF
:10F700001B0C43EA0423284CADB2A0429BB203D0A9
:10F7100004F50064A04213D1548923F4006343EA42
:10F7200004234FF6FF341C409388D68944EA032310
:10F73000948925F44055344345EA04159BB2ADB293
:10F74000D28885808183828787E7038C158823F49C
:10F7500080531B041B0C0384038C8488818B23F44B
:10F76000005321F4E6410904090C41EA05215688B9
:10F7700015891B0435431B0C43EA05330A4DA4B21B
:10F78000A84289B29BB203D005F50065A84205D115
:10F79000958924F4804444EA8514A4B2D2888480F4
:10F7A0008183A0F8402058E7002C014030B598B183
:10F7B0000A4B00221C461D79854207D19D792942BA
:10F7C00002D004EB021030BD0029FAD001320E2A1B
:10F7D00003F11003EFD1002030BD00BF90BE01083F
:10F7E0000149024801F090BE801C00200008004042
:10F7F0000149024801F088BE581C00200004004066
:10F8000002494FF0804001F07FBE00BF301C002055
:10F810000149024801F078BE081C0020002C01407C
:10F82000FFF7F6BFF0B5002541F221072B4624492A
:10F830000A78961EECB2B44219DB0244941E013AD7
:10F840000C440A446478527802EB042292B2934248
:10F850000CD100244FF4AF6791F82450194E0130B9
:10F86000E3B29D4217D80122174B1A70F0BD044431
:10F870000C44647883EA0423082413F4004F04F151
:10F88000FF344FEA430318BF7B4014F0FF049BB2E0
:10F89000F3D10135CEE700EB4303DAB28B18013226
:10F8A0000A4493F801E0537803EB0E239BB27B43A9
:10F8B0001B1303F5487326F814300134D0E700BF5A
:10F8C0000C280020CC260020E426002007298FBF2A
:10F8D0000020034B03EB8101886A80B2704700BFB0
:10F8E0000C2800202DE9F041174D95F8482012B959
:10F8F0000020BDE8F081002285F8482095F84920D5
:10F90000A82AF5D195F85C40002CF1D10F4F104E8C
:10F9100005F14908283508EB0403D8781B7903EB77
:10F92000002007F0A1F8394607F0F6F8314606F056
:10F93000E9FF07F0F3FA45F814000234102CEAD17D
:10F940000120BDE8F08100BF0C2800200000203E0F
:10F950000080BB43034B03EB4101B1F85E00C008DC
:10F96000704700BF0C2800201F4BF0B593F87E2095
:10F9700019460AB90020F0BD002093F87F40B3F883
:10F98000806003EB440595F8857095F8862083F830
:10F990007E0042EA07229642ECD193F88330012B95
:10F9A00002D0812B14D0F0BD1846102C88BF102334
:10F9B0004FF0000288BF81F87F300C4B91F87F40F8
:10F9C000A3F12705D1B28C4203F1020302D8F0BDA6
:10F9D0000320EAE713F8026C13F8011C41EA062140
:10F9E00025F812100132EDE70C28002091280020A4
:10F9F00003788B420CD9074B890093F8A7200B445E
:10FA0000D3F8A80002B1400800F5777080B27047C3
:10FA1000002070470C280020054B03EB8101D1F832
:10FA2000D80000EB8000C00800F55C7080B2704721
:10FA30000C2800205E4B10B593F82001002800F040
:10FA4000B680002293F8234193F8240183F8202103
:10FA500093F8222104F0070142EA012200F03F015D
:10FA6000490141EAD401C3F8D82093F82521C3F80D
:10FA7000DC1093F82611920093F8274142EA901285
:10FA800001F0010042EA8022C3F8E02093F8280147
:10FA900004F00F02D20142EA510200F07F01C3F8E4
:10FAA000E420090193F8292141EA141193F82A412D
:10FAB0005200C3F8E81042EAD01204F0030193F8B0
:10FAC0002B0142EA4122C3F8EC2093F82C2100F0EC
:10FAD0001F018901D20041EA940142EA501293F8D1
:10FAE0002E4193F82F01C3F8F42093F82D21C3F889
:10FAF000F01004F0070142EA012200F03F01490141
:10FB000041EAD401C3F8F82093F83021C3F8FC107F
:10FB100093F83111920093F8324142EA901201F0C9
:10FB2000010042EA8022C3F8002193F8330104F077
:10FB30000F02D20142EA510200F07F01090141EABD
:10FB40001411C3F80811C3F8042193F8342193F871
:10FB50003541520004F0030142EAD01242EA412248
:10FB6000C3F80C2193F8372193F83601D20042EA0A
:10FB7000501200F01F01C3F8142193F838218901B5
:10FB800041EA9401D407C3F810114CBF40F214713C
:10FB9000AD21C3F8181191074CBF40F21471AD218B
:10FBA00012F0080F14BF03200120C3F81C1110BD70
:10FBB0000C28002008B5084B03EB8101D1F83C016B
:10FBC00006F052FF054906F0A7FF054906F09CFE26
:10FBD00007F0A4F980B208BD0C28002001F11F3FF6
:10FBE00000405C446B4B30B593F87C210AB900208F
:10FBF00030BD002283F87C2193F87F21162AF6D1AC
:10FC0000082112F0800F4FEA420218BF82F0D5029D
:10FC10000139D2B2F5D193F87E015F4D02388142AD
:10FC2000C0F2A78093F896119142E0D1182293F880
:10FC3000814193F8820183F87E2193F8802104F0BA
:10FC4000070142EA012200F03F014901C3F83C21CB
:10FC500041EAD40193F88321C3F8401193F8841149
:10FC6000920093F8854142EA901201F0010042EAC5
:10FC70008022C3F8442193F8860104F00F02D201D8
:10FC800042EA510200F07F01C3F84821090193F8CC
:10FC9000872141EA141193F888415200C3F84C11AE
:10FCA00042EAD01204F0030193F8890142EA4122AA
:10FCB000C3F8502193F88A2100F01F018901D20076
:10FCC00041EA940142EA501293F88C4193F88D0175
:10FCD000C3F8582193F88B21C3F8541104F007019D
:10FCE00042EA012200F03F014901C3F85C2141EAE8
:10FCF000D40193F88E21C3F8601193F88F1192000C
:10FD000093F8904142EA901201F0010042EA802209
:10FD1000C3F8642193F8910104F00F02D20142EA82
:10FD2000510200F07F01090141EA1411C3F86C117E
:10FD3000C3F8682193F8922193F89341520004F09C
:10FD4000030142EAD01242EA412293F89401C3F837
:10FD5000702193F8952100F01F018901D20042EA39
:10FD6000501241EA9401C3F87411C3F878210120BC
:10FD700030BD6C18E4786240082412F0800F4FEA1E
:10FD8000420218BF82F0D502013CD2B2F5D1013156
:10FD900045E700BF0C2800208929002070B5304EAF
:10FDA000054633782F4C3BB1D4F8A43183429EBF33
:10FDB0000023337084F8A8312B4B1B6813F0010229
:10FDC0001CD094F8A92194F8AA3193420CD00123B5
:10FDD000002184F8A831254B84F8AA211970D4F8A1
:10FDE000AC312B44C4F8A43194F8C83173BBD4F8B7
:10FDF000D801854234BF0020012070BD13F40053A8
:10FE000008D013461A4A32F8131009BB01330C2BE1
:10FE1000F9D1E9E784F8C831D4F8D4319847C30759
:10FE2000E2D5012300F00200002814BF1A46002288
:10FE300084F8C8310D4B5A700CBF01230023337076
:10FE4000D4F8AC312B44C4F8A431CDE7012070BD07
:10FE50000123002284F8A831044B1A70F0E700BF98
:10FE6000A53500200C2800200C360020200400209E
:10FE7000BC29002000207047002070470023032B7E
:10FE8000CCBF012200220CBF05211E2100F8132047
:10FE900000EB43020133122B5170F0D1704710B5C3
:10FEA00000234FF47A744FF4FA61C452C218043339
:10FEB000102B5180F9D110BD024B03EB4101B1F879
:10FEC000B00170470C280020024B03EB4101B1F850
:10FED000B00170470C280020044B93F8DC0118B1E6
:10FEE0000022012083F8DC21704700BF0C2800208D
:10FEF000024B03EB4101B1F8DE0170470C280020F2
:10FF0000024B03EB8101B1F8040270470C2800207A
:10FF1000034610B500F16004064A0C3303CA43F8E7
:10FF20000C0C106843F8081C43F8040CA342F3D1EE
:10FF300010BD00BFE0AB010840F2DC530380322368
:10FF400043800123042283730023C2731A4630B511
:10FF5000084C838119198D792D0741BF0D798118BE
:10FF60000D710132D02B03D0072A03F11003F1DD0C
:10FF700030BD00BF90BE010870B5054601F0D0FB52
:10FF8000324CD4F83C32C4F83C02C31AB3F5FA5FE1
:10FF900082BF002384F8403284F8413294F8403222
:10FFA00033B9A12D1ED1012284F841221B222270D7
:10FFB00094F841222AB1E218EDB20133557084F869
:10FFC000403294F840522378AB420AD194F842323E
:10FFD000052B0ED0062B0FD0002384F8413284F875
:10FFE000403270BDA22DE3D1012284F841222322A8
:10FFF000DDE70020FFF716FCA3781E2BECD10020D4
:020000040801F1
:100000000246013DC3B2AB4207DB25446B789A42FE
:10001000E2D10320FFF706FCDEE7082123445B78EA
:10002000DBB282EA030616F0010F4FEA530301F137
:10003000FF310CBFDBB283F08C0311F0FF01C2F380
:100040004702EED101301A46DCE700BF0C28002041
:1000500010B5044601F064FB41F288310D4BD3F832
:100060004422C3F84402821A8A4284BF002283F8E1
:10007000482293F84822142A03EB02010CBF012204
:10008000013281F8494014BF83F8482283F84820A0
:1000900010BD00BF0C28002010B5044601F040FB45
:1000A000254BD3F84C22C3F84C02821AB2F57A6F72
:1000B00084BF002283F8502293F850224AB9A82C1A
:1000C00038D183F87E20A3F88020991881F88240E7
:1000D00006E0022A02D183F87F40F6E7242AF4D909
:1000E00093F87F1001320231D2B249008A4283F87C
:1000F000502216DA082241F22101B3F88000E4B25E
:1001000080EA042010F4004F02F1FF324FEA400071
:1001100018BF484012F0FF0280B2F3D1A3F880006C
:1001200010BD01318A4201BF002283F85022012212
:1001300083F87E2010BD00BF0C280020F8B5434C8A
:1001400094F85802002859D0002384F8583294F8C3
:10015000593294F85A5205EB032501F0E1FA3C4B71
:10016000ADB2B0FBF3F0D4F86C32002B47D1A4F859
:100170007052C4F86C020322D4F8743294F87352AB
:100180001E7894F8720294F87872511E631893F8EE
:1001900059322B4103F00F03B34212D20B2B10D86C
:1001A00008B183420DD0214491F859E2A11891F889
:1001B00059120EEA070E04EB830301EB0E21C3F87C
:1001C000A8100232112AE0D194F87932ABB194F838
:1001D0007A3293B194F85B321B060ED501F0A0FA87
:1001E000D4F854321B4964301BB15A68121A002AE1
:1001F00028DB194AD36004320A600120F8BD984216
:10020000B9D0C31A012BB2D194F87222002AAED011
:10021000B4F8703294F8A71092002244EB1A49B156
:100220006FF01301DB0293FBF1F303F50063C2F8F7
:10023000A8309CE76FF013019B0293FBF1F303F5E9
:100240008063F4E703F108019B68CDE70C280020E8
:1002500020A10700602A00202004002010B50446D9
:1002600001F05EFA41F288310E4BD3F87C22C3F8DC
:100270007C02821A8A4284BF002283F8802293F88B
:1002800080220F2A0DD8511CC9B21A441029E4B299
:1002900082F8594214BF0022012283F8801283F8A9
:1002A000582210BD0C28002010B5044601F038FA81
:1002B00040F6AC51104BD3F88422821A8A42C4BF54
:1002C000002283F8882293F888228AB90F2C11D152
:1002D000C3F88402511CC9B21A44192982F8214179
:1002E00014BF0022012283F8881283F8202101E044
:1002F000182AEFD910BD00BF0C28002010B5044605
:1003000001F00EFA124BD3F88C2202F57A72904269
:1003100084BF002283F8902293F8901219B9C3F891
:100320008C02052204E00229FBD993F87E210232D7
:100330008A420CDD481CC0B28242CCBF002201229E
:10034000194483F8900281F87D4183F87C2110BD27
:100350000C28002010B5044601F0E2F9284AD2F832
:100360009432C31AB3F5FA7F134628D9002283F8D2
:10037000982283F8992293F89822C3F8940292B9AC
:10038000E1B2042901D0202921D183F89B1283F8FE
:100390009C120221002083F89D124FF6FF7183F812
:1003A0009A02A3F89E12991881F8A04293F89C1221
:1003B00001398A4220D1012283F8C02210BD92F86F
:1003C00099120029D7D0013982F8991210BD93F8FB
:1003D0009B1271B9552C0CD101211F2083F89A1260
:1003E00083F89B4283F89C02A3F89E2283F89D1217
:1003F000D9E78C42D7D010BD013283F89822FAE7B2
:100400000C28002010B5074C94F87A2242B104F26F
:10041000C121D4F8D80201F045FA002384F87A32D9
:1004200010BD00BF0C280020F8B52A4E96F8C03247
:1004300034460BB90020F8BD002596F89A3286F8AC
:10044000C052012B96F89C1232D1314491F89F3260
:1004500091F89E22B6F89E0202EB032296F89D3296
:1004600092B203F11C05EDB2E61896F8A17296F867
:10047000A012023301EB0721DBB20144AB4288B288
:10048000F2D18242D6D1002294F89D52124905EB56
:100490004203DBB2234493F8A10293F8A03203EBAA
:1004A000002341F8223001320E2AF0D10120F8BD9C
:1004B00006F52870FAF7A1FF0028BBD096F89B320A
:1004C000202BE0D006F52870FAF7B2FF86F89902E3
:1004D000B0E700BF0C280020102A00202DE9F041D1
:1004E00005460F460446094E06F10808217809B969
:1004F000BDE8F081054809F0FFFD20B140453EBF51
:10050000801B631B3B540134F0E700BFECAB0108D8
:1005100010B500212C22044609F0B9FD01236372B5
:1005200023751E23A37540F2DC53238340F24C4312
:10053000638340F26C73A3830223A377132384F8AD
:100540002030062384F8223040F24653A38440F240
:100550007533E38440F64303214623850148BDE813
:100560001040BBE707CE0108094A92F8DC325BB9BC
:10057000084B92F8CC1193F822300433DBB28B4253
:1005800028BF0B4682F8DC3292F8DC02704700BFCD
:100590000C28002038360020124B03EB400393F860
:1005A000DD222AB1022A12D00F4B33F81000704717
:1005B000022809D90328F7D10C4B1B6813F4805F7C
:1005C0000B4B02D1D88C7047094B188B704793F8AE
:1005D000DE0200EB800000EB800000F2EE2080B233
:1005E000704700BF0C280020CC3500200C360020BE
:1005F0003836002008B501F093F80222064B83F844
:100600000823C3F80403054B1A68054B9A600122BE
:1006100083F8212008BD00BF0C280020901B00207B
:100620001036002008B501F07BF80222074B00F5D8
:10063000B71083F80823064A00F55870C3F804037E
:10064000936803F2DC53936008BD00BF0C280020C0
:100650001036002070B50024114D2146702205F29D
:100660000A3085F8094309F012FD214605F27A3473
:10067000A4F17000631893F902207AB11E680A1879
:100680000E509E889B790731937195F80933702934
:1006900003F10103968085F80933EBD170BD00BFEB
:1006A0000C2800200C230B4A03FB002393F8F7339C
:1006B0001146FF2B07D092F8CC219A4203D9064A63
:1006C00032F9130070470C2303FB0010B0F9F40358
:1006D000704700BF0C280020CC35002038B5134AE5
:1006E000134C054694F84C3410685843114B18606D
:1006F00006F0BAF9104906F00FFAC4F8500428467B
:1007000002F06EF8284601F0ADFF688D06F0B0F9F2
:100710000A4906F001FAC4F85404A88D06F0A8F9B5
:10072000064906F0F9F9C4F8580438BD2041002004
:100730000C28002008250020BD3786356F12833A2B
:100740002DE9F04F85B0044601F049FA064620B184
:1007500001F07AFD05B0BDE8F08F204603AA5E499E
:1007600007F098F834460546B0464FF0FF37DFF8FB
:100770009491DFF894A1DFF894B1BDB90C26394605
:100780005648FCF753FF564B78B206FB05F2D118DA
:10079000D256824200F086800135042DF5D1B8F1A1
:1007A000000F33D14F48FCF741FFD3E7012E0ED0A5
:1007B000022E11D01EB9284607F010F8074603AAEA
:1007C0004549002007F066F801360546D5E728467A
:1007D00007F004F88046F2E74946284609F0E8FCAD
:1007E00020B94149284609F0E3FC08B144F001046E
:1007F0005146284609F0DCFC28B95946284609F03C
:10080000D7FC0028DBD044F00204D8E7002C08BF56
:1008100003240022E4B20192009443461146F7F704
:10082000C7FF054608B93148BDE741463048FCF7E7
:10083000FDFE3048FCF7FAFE2F4B1C682046F7F708
:1008400065FF2846F7F762FF0021084601F022F90C
:100850000021012001F01EF9204601F01DF870B1C1
:100860000121002001F016F9204601F012F801469E
:10087000284601F014F80021084601F00BF928463B
:1008800001F00AF80028E7D00121002001F002F968
:10089000284600F0FEFF0146204601F000F8002146
:1008A0000846D7E74D68002D3FF479AF1348FCF7B1
:1008B000BDFE54B169798C4207D022461048FCF73E
:1008C000B5FEE1B2284600F0DEFFEB6A002BB0D0A7
:1008D0000023EB62ADE700BF05CE010816CE01088C
:1008E000584100201FCE0108FEC7010837CE01087D
:1008F0004ECE010891CE01087C25002063CE010870
:1009000073CE010810CE010813CE010823CB0108D5
:100910002DE9F04F8046894616460D4614464FF0A5
:10092000000ADFF810B189B0002E6FD06A686368E2
:100930009A4269D1AF68A368FB1A5F425F4194F99C
:100940000B305A46049394F90A3039460393B4F9AC
:10095000083040460293B4F906300193B4F90430EC
:100960000093534601F00EFB95F90B305A46049361
:1009700095F90A3039460393B5F908304046029399
:10098000B5F906300C340193B5F904300C350093F9
:1009900053460AF1010A01F00BFBBAF1080FC3D16B
:1009A00000242546DFF890A096B300270123325992
:1009B00003FA07FB59F8043053403BEA030314BF22
:1009C0000123002312EA0B0F079306D000972B4652
:1009D00052460799404601F0D5FA59F804301BEA0F
:1009E000030F06D000972B4652460799404601F068
:1009F000DFFA01370E2FD9D10135082D04F10C048F
:100A0000D2D109B0BDE8F08F002798E73746ABE7B1
:100A10003746012359F80420BB40134206D0009703
:100A20002B4652460121404601F0C2FA01370E2FF3
:100A3000EFD1E1E7B4CE0108CCCE01082DE9F04FAB
:100A40000546884614460027DFF8E0A085B0062357
:100A500000267B430393039B334408EB030292F885
:100A6000C0B0002C5ED0234493F8C0305246ABEBAC
:100A70000300D0F1000949EB0009019300963B46C1
:100A80004946284601F07EFA8DE840083B4652462A
:100A900049462846013601F08BFA062EDBD1013794
:100AA000062FD4D10026DFF884B008F1E40A1AF842
:100AB000019B002C38D0A31993F8E4305A46A9EBD7
:100AC00003014F424F4101930096062339462846C1
:100AD00001F058FA8DE840020623144A39462846A8
:100AE000013601F065FA0B2EE1D198F8F0606CB197
:100AF00094F8F0302846F21A0193002354425441EE
:100B000000930A4A0723214601F03CFA002301968C
:100B10000093064A07232146284601F049FA05B00A
:100B2000BDE8F08FA146AFE72746D3E7E1CE010845
:100B30007FB5054601F053F8044630B1002218494C
:100B40000120FFF77BFF04B070BD28466A461549B7
:100B500006F0A0FE134E01AD78B1032C02D101F0D6
:100B600073FBF0E706F03AFE6A4645F8240031468A
:100B7000002006F08FFE0134EEE7032CEFD101AC2C
:100B800070CC32462946E0B203F084FF0028E6D05C
:100B900033462A462146044801F032F9D3E700BF24
:100BA0002434002005CE0108E1CE01082DE9FF47DD
:100BB000814690460E4615460027DFF864A0B8F13E
:100BC000000F2AD02B8832889A4224D174886A88F0
:100BD000A21A54425441EA7821460292AA78484621
:100BE0000192009352463B4601F0CCF9F37852460D
:100BF0000293B3782146019336F8043B48460093AC
:100C00003B46013701F0D4F9102F05F10405D6D188
:100C100004B0BDE8F0870024DDE74446E6E700BF06
:100C2000F5CE01082DE9F041064600F0D8FF044654
:100C300028B1BDE8F041002222490120B6E7304644
:100C400006F0CCFD0F2805462EDC304600F0CFFF25
:100C50000646DFF87C801C4F2035304606F0BEFD8E
:100C600038F81430984226DC012C11D0022C13D015
:100C700027F8250030462C2109F03EFA064678B1C7
:100C8000012301360134B3B1032CE6D1BDE8F08174
:100C900007EB85039870EDE707EB8503D870E9E76C
:100CA000A21E53425341EDE72146BDE8F0410F2219
:100CB000064801F0B2B8002347F82530BDE8F041FE
:100CC00001F0C2BAA4340020243400209FC60108D9
:100CD00004AC01082DE9F04F07468A461646002469
:100CE0008FB0DFF860800DF124095AF824304946AE
:100CF00002A80293FAF7F2F816B356F82430029DD0
:100D00000393EB1A5D420DF1100B5D41594603A8A8
:100D1000FAF7E4F8CDF800B02346424629463846B3
:100D200001F030F92346CDF8009042462946384676
:100D3000013401F03DF9202CD7D10FB0BDE8F08F80
:100D40003546EFE707CF01082DE9F04F87B005469C
:100D500000F045FF044638B1002255490120FFF755
:100D6000B9FF07B0BDE8F08F284606F037FD1F2811
:100D7000074600F39780284600F039FFA046064654
:100D8000A246A1462546A346494B009443F8274076
:100D90000193484BE1B2E05C00230DF10C0CB64628
:100DA00016F8012B1AB190420FD00A2B09D106AECA
:100DB00033440026904203F80C6C08D001F044FA4A
:100DC000CFE703F80C200133E9E70246EFE70139EA
:100DD0000EF10106032932D8DFE801F04E1F025B55
:100DE0004FF0010EDFF8DCC00DF10B0010F8011F11
:100DF00049B30023304AD25C8A4203D00133072B27
:100E0000F8D15346002212F80CA08A453DD10EFAC3
:100E100002F248EA02089A46E8E74FF0010C0DF1A9
:100E20000B0111F8012F72B10023244813F800E0E0
:100E3000964526D10CFA03F349EA0309F1E703A822
:100E400006F0CCFC83460134052CA2D1009B05F0B2
:100E50000F0545EA834545EA895949EA0A2A4FEAD6
:100E60000B134AEA0838019ADBB248EA030342F856
:100E7000273003F08FFE74E703A806F0AFFC0546A9
:100E8000E1E70133062BD0D1CBE70132062ABAD1F4
:100E9000C1E703A806F0A2FC03460F28C8BF002341
:100EA0000093D0E71F222146054800F0B6FF58E71F
:100EB000243400200AAC01088EA9010888A9010881
:100EC0009FC6010895A901082DE9F34781460F4601
:100ED000904602260024DFF860A0B8F1000F28D069
:100EE00037F8242038F824309A4238F806201ED1EA
:100EF000BD5BA91A4D424D410192009352462346D3
:100F00002946484601F03EF8BB5B5246019337F84C
:100F100024302946009348462346013401F048F81E
:100F2000042C06F10406D8D102B0BDE8F0870025F4
:100F3000E2E74546E8E700BF11CF0108F8B50546EE
:100F400000F04DFE064628B1BDE8F84000222649D3
:100F50000120B9E72549284609F0A1F868B94FF4FE
:100F60007A714FF4FA62204B19805A809980DA80A6
:100F700019815A819981DA81F8BD284606F02EFC44
:100F80000328044628D8284600F031FE064658B10A
:100F900006F024FC01270546304600F028FE30B953
:100FA000BDE8F84001F050B905460746F4E706F001
:100FB00015FC002FF4D040F2DC53A5F2EE229A4249
:100FC000EED8A0F2EE229A42EAD8074B23F824503A
:100FD00003EB84035880F8BD3146BDE8F840032296
:100FE000034800F01ABF00BF6C2D0020DFCD0108C0
:100FF0009BD501082DE9F04F0E461546002797B006
:1010000008900992D6F800800021404605F018FFAC
:101010000446002869D173680493B3680593F368A4
:101020000693099B002B3DD0D5F800B0EB685946DC
:101030004046D5F804A0D5F80890079305F000FFC6
:1010400080B15146049805F0FBFE58B14946059819
:1010500005F0F6FE30B10799069805F0F1FE041C84
:1010600018BF012413A95846FCF736F910A9834686
:101070005046FCF731F90DA982464846FCF72CF999
:101080000AA981460798FCF727F9CDF80890039044
:10109000CDF804A0CDF800B03B46154A214608988B
:1010A00000F070FF13A94046FCF716F910A904469A
:1010B0000498FCF711F90DA980460598FCF70CF986
:1010C0000AA981460698FCF707F93B4603908DE88C
:1010D0001003074A00210898013700F069FF082F24
:1010E00006F1100605F110058CD117B0BDE8F08FA0
:1010F00022CF01082DE9F84F07460026534D384608
:1011000000F06DFD804628B10022BDE8F84F4F4940
:1011100001206FE705224E49384608F0FBFF38B939
:1011200000224A4BC25010308028FBD1BDE8F88F16
:1011300004224849384608F0EDFF04463846002CA2
:101140003FD100F054FD814600287CD004F020FF00
:10115000DFF818A15FFA80FB5AF82480B8F1000F7D
:1011600004D13D48BDE8F84F01F068B85A46414601
:10117000484608F0CFFF013407460028ECD1374B32
:101180002E6003EBC404D4F810E02E612E622E63AF
:101190002E642E652E662E67BEF1000F03D094F8E4
:1011A0000CC0674505DB41462D4800F029FE2D4F58
:1011B000A5E73B01EC1873440FCB013784E80F001F
:1011C000EFE706F00BFB0728054635D8384600F058
:1011D0000EFD064628B3FBF7E3FF01241B4A2B0153
:1011E000D050304600F003FD064630B1FBF7D8FF83
:1011F000164B013403EB05135860304600F0F7FC42
:10120000064630B1FBF7CCFF104B013403EB05135E
:101210009860304600F0EBFC28B9BDE8F84F01F0CB
:1012200013B80446DDE7FBF7BBFF084B032C03EBC9
:101230000515E860F1D167E74146BDE8F84F0722A0
:10124000094800F0EABDBDE8F88F00BF6417002030
:10125000DFCD0108E5CD0108FBC6010804AC01089B
:10126000EACD01080BDD01089FC6010834A701087B
:101270002DE9F04F814690460C4615460026192769
:10128000DFF8B0A087B0B8F1000F51D023782A78EA
:1012900093422B794AD160786978884246D1A07808
:1012A000A978884242D1E078E97888423ED1217914
:1012B00099423BD161796879081A414241410593CD
:1012C000EB7848460493AB788B467B4303F5617318
:1012D00003936B7801927B4303F5617302936B79FF
:1012E00052460093334600F04DFE23795246059353
:1012F000E37859460493A37848467B4303F561732A
:101300000393637806357B4303F561730293237877
:101310000634019314F8013C00933346013600F083
:1013200047FE0F2EAFD107B0BDE8F08F0021C6E712
:10133000C346DAE736CF0108F7B5074600F04FFCA1
:10134000044630B1002236490120FFF791FF03B077
:10135000F0BD384606F042FA0E28054659DC06264E
:101360004643781C8DF8074000F041FC2C4C0746A2
:1013700050B106F033FA032806D8A31958719DF826
:10138000073001338DF80730384600F030FC07464F
:1013900058B106F023FA0D2807D806236B43E05412
:1013A0009DF8073001338DF80730711C0DF10702ED
:1013B0002144384600F027FC00F019FC074660B1D4
:1013C00006F00CFA182808D8062303FB0543D8704A
:1013D0009DF8073001338DF80730384600F007FCE0
:1013E00060B106F0FBF90D2808D8062303FB05457C
:1013F0009DF80730287101338DF807309DF80730CC
:10140000062BA4D00023A219A351938000F01CFF47
:101410009DE70E222146034800F0FFFC97E700BF3E
:101420001C1900209FC6010810B5046B0346C16853
:10143000406944B11A6C8C1A013A08BF0A46005D33
:101440001A64C0B210BD1A6A805C01328A4228BF99
:101450002246C0B21A6210BD436B13B190F844002B
:101460007047836A406A1B1A584258417047416A64
:10147000836A0269994238BF8918CB1A416B21B13E
:1014800049680B44511E8B4202D2501EC01A70474D
:1014900000207047036B4BB1026C5B689342A3EB77
:1014A00002032EBF1846C068C0187047C269036A9D
:1014B0009A422FBFD01AC0688018C01A70470A4BD2
:1014C00030B503F1100493F900205D78072AC8BFF6
:1014D000143A81180D739D780433855413F8012C48
:1014E000A3420A76EFD130BD08AF01082323037071
:1014F0002423437000238370C37070474171F7F752
:101500006BBE8160F7F768BE2DE9F0470646894655
:101510004FF000474FF00008038A8589ADB21D40A7
:101520000DB9BDE8F087B5FA85F327FA03F2D24387
:101530001B3B91B231821540042BF1D8DFE803F058
:101540002925211A0300D9F8244084B1013CA4B212
:10155000C9F82480D9F820A0BAF1000FE0D0DAF859
:101560000030504621469847DAF804A0F4E7B48DDD
:10157000A4B2EFE7D9F80000B18E036889B29847AA
:10158000CEE7D9F80400318FF7E7D9F80800B18F1A
:10159000F3E7D9F80C00B6F84010EEE71FB50023CA
:1015A000ADF80A30ADF806308DF80C30074B013934
:1015B0001B68ADF80810B3FBF2F204A9013A21F858
:1015C0000C2D03F006FF05B05DF804FB10000020B1
:1015D00073B504460068FFF7E1FF226817491388D6
:1015E0009BB243F001031380002351F8334001EB19
:1015F000C300A2421DD145790124002601A88DF81F
:1016000004508DF805408DF806608DF8074003F012
:10161000F9FD1B2D0BD1192301A88DF804308DF88D
:1016200005408DF806608DF8074003F0EBFD02B031
:1016300070BD0133042BD8D10025DDE700A20108DD
:101640000B4B800A98420FD004D8B0F5801F09D008
:10165000FE207047074B984208D049339842F7D193
:101660000020704701207047022070470320704718
:101670000100100002001000F8B50468054620467D
:10168000FFF7DEFF032841D86B794FEA930E39B993
:1016900075460227A689AF40B6B226EA0706A6819C
:1016A0000A2505FB00E51D4E46F82510043546F8D1
:1016B0002520324631B199080223A5898B402B435E
:1016C0009BB2A3812823434303F120011144EFF38C
:1016D0001286502585F312880425103313441F68A1
:1016E00017B10F6019680431013D03F10403F6D10D
:1016F0000D60F3B283F31188282303FB0020036AF3
:101700002BB1A3899BB243F00103A381F8BDA38948
:1017100023F001031B041B0CF7E700BF081C00208B
:101720001E4B30B55B681E4AC3F308039BB9EFF349
:10173000128383B91B4910688C6800BF13689842F4
:10174000F9D14FF47A72184B196802FB01F31B1B95
:10175000B3FBF1F31EE0EFF31281102383F3128841
:10176000104CA568236813F4803F18BF01200F4B6D
:101770001CBF1860A56814681868CAB282F3118883
:101780004FF47A72084B2044196802FB01F35B1B8B
:10179000B3FBF1F302FB003030BD00BF00ED00E011
:1017A000901B002010E000E0E00A0020A02D0020A7
:1017B00038B50446FFF7B4FF0546FFF7B1FF401BFD
:1017C000A042FAD338BD10B5044604B910BD4FF499
:1017D0007A70FFF7EDFF013CF7E7EFF31283102279
:1017E00082F312880649DBB20A6801320A600021DE
:1017F000044A1160044A126883F31188704700BFDD
:10180000901B0020A02D002010E000E0014B586844
:10181000F7F7B0BC400B0020014B1868F7F7AABCE3
:10182000400B0020836A8169426B1944D160416A90
:101830008B4229BF0169CB1ACB1A53602ABF002300
:10184000536083624FF0000380F84430136838BF60
:10185000816243F0010313607047436A8269D15487
:10186000436A02690133934228BF00234362436BFA
:101870001BB11B68DB0705D4D4E7026DD36843F0C6
:101880008003D360704703689B69184703685B69EE
:1018900018470368DB68184703685B6818470368E4
:1018A0001B68184703682DE9F041DB6904460E46C2
:1018B000174693B90D467B1B3344002B01DCBDE872
:1018C000F081236820469B6898470028F9D015F8D6
:1018D000011B2046FFF7E3FFEDE7BDE8F0411847A5
:1018E000E0E7064B53F8202032B193881268D168A4
:1018F0000B4218BF1B041361704700BFEC0A0020A5
:1019000010B50409013C022C00F00F0215D80C4B55
:1019100033F8141041FA02F313F001000ED0012045
:1019200090400138084005F069FB064B1C44237CBD
:101930000344054800EBC30010BD002010BD00BFEC
:10194000F8A1010808AF0108341600202DE9F04184
:101950000C460746002851D003682D4A03F1404346
:10196000A3F5843302EB9323D87C03F02DFCBD88D0
:10197000E20654BF04F00C0104F00F0115F0FF0F54
:1019800004F07C063B681AD000204FF0010E4FF0A7
:101990000F0C1A680EFA00F737EA05040BD1840021
:1019A0000CFA04F822EA080201FA04F4282E42EAAA
:1019B000040225D15F6101300828EBD11A60FF2DA8
:1019C0001CD900204FF0010E4FF00F0C5A6800F1A7
:1019D00008040EFA04F434EA05070BD187000CFA68
:1019E00007F822EA080201FA07F7282E42EA07025E
:1019F0000AD15C6101300828E9D15A60BDE8F08164
:101A0000482E08BF1F61D6E7482E08BF1C61F1E7CA
:101A100008AF010810B1036882885A61704710B19D
:101A2000036882881A61704738B1002914BF002109
:101A30001021838802688B40136170470F4B014669
:101A40001B883BB90E4B18680E4B1B780BB981F005
:101A50000101E9E70C4B5A6972B150B10B4A1968A0
:101A600010880B4A92FBF0F292B20A8001225A745B
:101A700070471A6810805874704700BF400C0020EF
:101A8000440C0020480C00204C0C0020640C00206A
:101A900020A107000123084A834012781340074A17
:101AA00052F8200019B1191C18BF0121BCE7B3FA84
:101AB00083F14909FAE700BFE60A0020EC0A00209A
:101AC00038B50D46012104460846FFF7E3FF002123
:101AD0000846FFF7DFFF04B938BD0120FFF701FF1B
:101AE0000020FFF7FEFE0120FFF7A8FF2846FFF7C2
:101AF0006AFE0120FFF7F5FE0020FFF7F2FE00204E
:101B0000FFF79CFF013C2846FFF75DFEE4B2E2E7E9
:101B100038B50D460130C4B205B938BD05203221B3
:101B2000FFF7CEFF4FF4FA70FFF74DFE1CB1FA211C
:101B30002046FFF7C5FF4FF47A70FFF744FE013DE2
:101B4000EAE708B50A21FFF7E3FF024A024BDA6031
:101B500008BD00BF0400FA0500ED00E0FBF746B940
:101B6000FBF744B9FBF742B9FBF740B9FBF73EB9C5
:101B7000FBF73CB9FBF73AB9037903F00C03042BEC
:101B800005D0082B0FD0BBB9B0F80B0070470B4B3A
:101B9000B0F80B001B7803EBC30203EB820300EBEE
:101BA000430080B27047054BB0F80B005B7803EB45
:101BB000430300EB8300F4E7002070470816002081
:101BC00010B4447A631CDBB204444372A172027AFB
:101BD0009A4202D810BCFBF711BA10BC704720B172
:101BE0000078B0FA80F0400970470120704708B5CE
:101BF000202108F081FA034618461BB10278013310
